:020000040800F2
:1040000000500020E1F800084DCA000851CA00081D
:1040100055CA000859CA00085DCA0008000000001F
:1040200000000000000000000000000065CA000859
:1040300061CA00080000000069CA00085198000821
:104040006DCA000871CA000875CA000879CA00085C
:104050007DCA000881CA000885CA000889CA00080C
:104060008DCA000891CA000895CA00080000000027
:104070000000000000000000000000000000000040
:104080000000000000000000B5CA0008B9CA00081E
:10409000C9CA0008D9CA0008E9CA0008B14900081D
:1040A000FDCA000801CB000805CB000809CB0008B9
:1040B0000DCB000811CB000815CB000819CB000868
:1040C0001DCB000821CB000825CB000829CB000818
:1040D0002DCB000831CB0008398D0008FD8D00087C
:1040E0003DCB000841CB000845CB00080000000094
:1040F00000000000000000000000000000000000C0
:0C41000000000000000000005FF800005C
:1041100030BF704720BF704740BF7047BFF36F8FFD
:104120007047BFF34F8F7047BFF35F8F704701DF5A
:104130007047EFF31480704780F31488BFF36F8FDC
:104140007047EFF30980704780F309887047EFF3F9
:104150000880704780F30888704772B6704762B66F
:10416000704771B6704761B6704780F31188704729
:10417000EFF31280704740BA704700BA70470000F2
:1041800010B500F03FFC0B4C0B490C4A0C4B48B1EE
:104190004FF0010C0B4884F800C00B4C1860146001
:1041A000086006E020700948086009491160094A62
:1041B0001A6010BD780B0020A00B0020840C00209A
:1041C000140C0020C9910008F99F00085D920008B6
:1041D00099970008E196000837B50AF053F86B4B41
:1041E00000254FF480301D700AF06CF80AF0D0F909
:1041F0000128044627D1102009F02EFB28460AF09A
:10420000B1F828460AF0C2F84FF480600AF0B4F81A
:104210004FF440304FF4E0110AF080F820460AF0E5
:1042200089F839200AF09EF90028FAD0022009F016
:10423000FBFA02200AF084F80AF08CF80828FBD177
:10424000524B01221A70042001210AF041F9032384
:104250008DF80630153301A94D488DF807304FF41D
:104260008073ADF8043009F02BFD06200AF074F9D4
:10427000012001460AF02CF9464C4FF480414FF0E2
:10428000006009F021FF4FF4407009F07FFE00F05C
:1042900001FC00F0B5FDFFF773FF00F0F3F805F047
:1042A0001BFC05F077FB04F021FC00F079F8207886
:1042B00004F0B6FEE07804F0A7FC207804F0F6FDE8
:1042C000E07804F0C9FC344B1B7823B9226960798B
:1042D000A16805F05DF8304B1B780BB105F03CFF91
:1042E00006F0C4FC00F016FA08F082F900F066F956
:1042F00001F0A0FE05F04CFF06F0FEFC274B4FF44A
:1043000000521A6105F040FB044603F0A5FC06F0DC
:1043100001FD05F077FF05F037FB001B0028B8BF53
:104320004042B0F57A7F24DD1B4D2B782C4683B1BB
:1043300000F068FB68B9287005F0CEFE05F0ACFD12
:10434000FFF71EFF134B1A695879996805F020F89A
:104350000CE0237853B900F055FB38B104F0DCFFD2
:1043600001232370FFF70CFF05F0F6FE05F00CFBB0
:10437000044600F05FF900F051F90028C5D006F0BE
:1043800075FC01F057FE06F0B7FCBEE7740C002088
:104390000008014008000020780B002000100140B8
:1043A000114B82B01B78E3B1104B08225A610422F2
:1043B0001A61002301E0019B01330193019A0C4B28
:1043C0009A42F8D9094B08221A6104225A61002343
:1043D00001E0019B01330193019A054B9A42E3D816
:1043E000F7E702B0704700BFB40B00200010014097
:1043F0003F0D030010B1012805D101E0402200E08B
:104400008022014B5A617047000C014010B1012815
:1044100005D101E0402200E08022014B1A61704783
:10442000000C014038B50546002455FA04F2E3B209
:1044300012F0010F184602D0FFF7E8FF01E0FFF786
:10444000D9FF0134082CF0D138BD00BF18B10128C4
:1044500006D0002008E0054BD868C0F3801003E0C8
:10446000024BD868C0F3C010704700BF000C014079
:1044700008B1002003E0024B9868C0F38000704749
:10448000000C014062B6704772B6704718B9024B13
:104490004FF400521A6170470010014018B9024BE6
:1044A0004FF400525A6170470010014010F0010FA4
:1044B00003D00E4B08221A6102E00C4B08225A610D
:1044C00010F0020F03D0094B10221A6102E0074BD3
:1044D00010225A6110F0040F03D0044B20221A61FD
:1044E00002E0024B20225A61704700BF000C0140DD
:1044F00008B1002005E0034BD3E90023100A40EA8D
:1045000003607047B80B0020F8B50D460446B8B9F3
:10451000FFF7BAFF0B492A464FEAE273C1E90023CD
:10452000D1E900673B0243EA16633202C1E9002386
:10453000054B1C60054B1C60054B9C84FFF7A2FFDC
:10454000F8BD00BFB80B0020C00C0020980B002065
:104550000004004010B9024B09011960704700BF08
:10456000C00B002020BB11F0040F10D011F0100F71
:1045700004D0104B9A6842F480720CE00D4B9A689C
:1045800022F480729A60DA6842F4807207E0094B84
:104590009A6822F480729A60DA6822F4807211F0CC
:1045A0000801DA60044B02D001221A7000E0197091
:1045B000704700BF0004014030020020084B4FF458
:1045C00000721A60074B10B50024204610211C60B1
:1045D000FFF7C0FF20462146FFF7C4FF10BD00BF14
:1045E000A80B0020A40B002010B9024B0901196090
:1045F000704700BF0400002008B9014B5970704794
:1046000030020020044B98780138C0B201288CBFDA
:1046100000200120704700BF30020020044B987832
:10462000012801D0002001E002229A70704700BFEB
:1046300030020020082008B505F0C2F9592804D935
:10464000064B9A784AB9013206E0082005F0B8F91D
:10465000542802D8014B00229A7008BD3002002075
:10466000012808B505D003D30A280AD000200CE0A1
:10467000002005F0A5F9B0F5006F94BF00200120DF
:1046800003E0024B9868C0F3402008BD00100140D1
:1046900038B500242546E0B2FFF7E2FF20B1012340
:1046A000A34043EA0505EDB20134082CF3D12846B6
:1046B00038BD00BF38B50D4B0D4C9A6812F00202A0
:1046C00001D0606810E0FF21032000F01FFBFF21F4
:1046D00005460122032000F019FBA36840EA0520EB
:1046E00003EA9000181A606038BD00BF000C01405A
:1046F0003002002008B5FFF7DDFF052801D80120B2
:1047000007E0FFF7D7FF40F2F933984294BF00204B
:10471000012008BD38B51E4C002021694909FFF76A
:1047200063FF2169002001F01F01FFF765FFFE21F3
:104730000022032000F0EAFA40210122032000F0C9
:10474000E5FA00210A46032000F0E0FA00210446C1
:104750000122032000F0DAFA082C0E4B05D14FF4A9
:104760000062DA6040F6FF7204E04FF40072DA6033
:1047700040F2FF329A60FFF79DFF064B0402244689
:104780004FEAE475C3E90845C3E90645186138BD39
:10479000180C0020300200202DE9F84305F0F4F851
:1047A000624CA062FFF786FF2369E06298423EDD1B
:1047B000E268C11A91420BDA5D4B256B1A684D19FC
:1047C0005143D4E90867721847EBE17325632BE086
:1047D00094F801C0564A1CF0040F12D0A368166862
:1047E000C31A5E432CF0040C36464FEAE677236387
:1047F00000220023C4E9086784F801C0C4E9062345
:104800004EE0A56816685A190132121A7243D4E9AB
:104810000867236BED43ED18B6EB020867EBE2790E
:1048200042464B4669182163C4E9082338E037DA69
:10483000E1681A1A8A420EDA3D4D216B2D68C91AB9
:104840006A43D4E90867B6EB020867EBE2794246AF
:104850004B460918E7E76178354A11F0040F0FD08D
:10486000126821F00401424312464FEAE273C4E9A0
:104870000823002200236170C4E9062320630FE0AF
:10488000A16812680131CB1A1B185A43D4E9086792
:10489000B61847EBE277226BC4E908679B182363DD
:1048A000224B1D6B5A6B996BAA1A82EAE27CACEB25
:1048B000E27C8C452CD942F210714A439E6ADC6B33
:1048C0003C21341B92FBF4F251434FF4807C91FB6A
:1048D000FCF181EAE172A2EBE172596440F6B83171
:1048E0008A42DE635D631C6401DDC82219E0B2F513
:1048F0007A7F01DD642214E0322A01DD0A2210E011
:104900000A2A01DD05220CE0012A0BDD012208E064
:10491000996ADA6B8A1AB2F5FA6F03D900225A64DF
:1049200001329A63014B1861BDE8F8833002002020
:104930000400002038B50D4618BB124CFFF72CFFC1
:10494000D4E90801002901DBA26803E0A268404223
:1049500061EB4101120212464FEAE2730DF0E0FDF5
:10496000C4E9062328464FEAE071064C0B02020216
:1049700043EA1063D4E90601801841EB0301C4E95E
:10498000080138BD3002002008B508B100200CE055
:10499000FFF702FF054BD3E90601D3E90823121AFA
:1049A00063EB0103100A40EA036008BD30020020F7
:1049B00008B54FF4807008F031FF0C4A00231360F3
:1049C0000B4A002013600B4A0021C2E900010A4A89
:1049D00093840A4B1B7843B9094B9A6822F480727E
:1049E0009A60DA6822F48072DA6008BDC00C002098
:1049F000980B0020B80B002000040040300200207B
:104A00000004014008B5084B587E10F0010005D0A5
:104A1000002007F0FFF980F0080001E007F0FAF944
:104A2000C0F3C00008BD00BF0800002010B5044658
:104A3000C0B1002007F050FC0221002007F0D4FA9A
:104A4000421E0020014607F081FB0020024601467D
:104A500007F0A4FA6821002007F0C6FA40F0080227
:104A6000002005E0682107F0BFFA20F00802204688
:104A7000682107F06BFB10BD08B510B109F02EFBE3
:104A800001E009F033FB08BD08B5C90805F058FD81
:104A900008BD00BF2DE9F04501218BB0DFF860A211
:104AA000914809AC09F09CF904200121032709F081
:104AB0000FFD1025214642F213035046ADF8243075
:104AC0008DF826708DF8275009F0FAF840F203238C
:104AD0000426DFF834822146CAF810505046CAF83E
:104AE00014304CF20063ADF824308DF826708DF848
:104AF000276009F0E5F80820012109F0E9FC4046AB
:104B0000214641F2F803ADF824308DF826708DF877
:104B1000275009F0D5F841F2380340462146C8F83D
:104B200010304FF00503ADF824308DF826708DF865
:104B3000276009F0C5F84823404621468DF8273004
:104B40004FF0020308F58068ADF824308DF8267028
:104B500009F0B6F82846012109F0BAFC4046214682
:104B60004EF20C038DF82750ADF824308DF82670E6
:104B700009F0A6F84CF20C03C8F8103042F23003EA
:104B800040462146C8F814304FF4FE53ADF82430A7
:104B90008DF826708DF8276009F092F82020012109
:104BA00009F096FC214651488DF82670ADF8246036
:104BB0008DF8276009F084F8022001214C4C09F09F
:104BC00087FC01214B4809F00BF90121022009F073
:104BD0008DFC03AD20460AF05BFC28460AF04EF837
:104BE000294620464FF000054FF0FF33ADF8103056
:104BF000ADF80C50ADF81250ADF80E5009F0E6FECD
:104C000000221346394620460AF0EEF868460AF0BC
:104C100049F84FF0080820466946ADF808800AF0C8
:104C2000D3FB20466946ADF800600AF0CDFB204674
:104C300041F65F610AF01EFB20460121A5840AF0BF
:104C400045F80821022009F0F9F801244FF4807397
:104C500006A806938DF81D808DF81C508DF81E4017
:104C600008F076FD244B08A89A688DF8234022F4BA
:104C700080729A60DA686F4622F48072DA601723D5
:104C80008DF820308DF822508DF8215009F088F9E8
:104C900021461A4809F0A4F800231A461946184C70
:104CA0004FF4005565612046A468013314F4804F29
:104CB0004FF400540461806808BF013110F4804F44
:104CC00018BF01320A2BEAD10A2903D10A2A01D1DD
:104CD000012200E000220B4B03481A70012109F069
:104CE0007FF80BB0BDE8F0850002300000140140F1
:104CF00000040040000C1A000004014000043000D1
:104D000000080140B40B0020000C014070B50446BF
:104D10000D461646032867D8DFE800F00206090EA4
:104D20004FF48052314B11E01022314B02E0314BF5
:104D30004FF480425A611BE02F4A138823F002038C
:104D40001B041B0C13802B4B4FF400425A612A4862
:104D5000022109F01FFD0028F9D02946264809F054
:104D6000BDFC2548012109F015FD0028F9D00FE010
:104D70002248022109F00EFD0028F9D029461F48DB
:104D800009F0ACFC1D48012109F004FD0028F9D010
:104D9000EEB1032C28D8DFE804F002070A0F134B0A
:104DA0004FF480521A611AE01022114B02E0114BAD
:104DB0004FF480421A6110E00E4A0F4B4FF400414D
:104DC00011611A8892B242F002021A8007E0032CA5
:104DD0000AD8DFE804F004020204084800E00648AC
:104DE00009F07EFCC0B200E0002070BD000C014064
:104DF0000008014000100140003800400030014030
:104E00002DE9F04F01218BB04FF4804009F06EFB8B
:104E1000494C012009AF014609F05AFB03264FF027
:104E2000180B204639464AF20003DFF81491ADF81A
:104E300024304FF0040A8DF826608DF827B008F072
:104E40003FFF204639464FF480430DF11008ADF87E
:104E500024308DF826608DF827A008F031FF4FF43C
:104E60008273002402224FF4007C0125484641460B
:104E7000ADF812304FF00803ADF81620ADF81AC0A7
:104E80000392CDF808C0ADF81C30ADF81040ADF875
:104E90001440ADF81850ADF81E40ADF8204009F0B0
:104EA000A9FB4846294609F0E1FB29464FF480500A
:104EB00009F00EFB09F550492846214608F090FFFD
:104EC000484639464FF0A003ADF824308DF827B09E
:104ED0008DF8266008F0F4FE484639464FF040034E
:104EE000ADF824308DF826608DF827A008F0E8FE94
:104EF000039ADDF808C04FF482734146ADF81230D2
:104F00000E484FF02803ADF81620ADF81AC0ADF8E2
:104F10002040ADF81040ADF81440ADF81850ADF891
:104F20001C30ADF81E4009F065FB0448294609F025
:104F30009DFB0BB0BDE8F08F000C0140003001403C
:104F400000380040014B1878704700BF78020020FD
:104F50002DE9F845054614460E4600294BD0002899
:104F600049D0814247D04FEA42185FFA88F848F0AA
:104F700006073946002007F037F848F00C01824652
:104F8000002007F031F8804628460DF08BF80546E2
:104F900030460DF087F8014628460DF08FF9064699
:104FA00050460DF07FF831460DF088F90DF098FA73
:104FB000054640460DF076F831460DF07FF90DF0CC
:104FC0008FFA0E49002814BF80464FF00108304682
:104FD000002D08BF01250DF05BFA18B141462046AF
:104FE00007F07CFA39462A46002007F0AFF8044B58
:104FF000E41801232371BDE8F88500BF0000A0413B
:105000007802002070B50D4D044645192B799BB1EF
:10501000C6B20B4B710141F0060153F8202001F09C
:10502000E601002007F026F9064B304653F824101D
:1050300007F054FA00232B7170BD00BF78020020E6
:10504000700B00206C07002013B5A14CA07800283D
:1050500040F031836378A62B00F06C825FD8852BFB
:1050600000F0F08027D8072B00F024810FD8032B05
:1050700000F0E88005D8012B00F0BC8000F2C4806D
:10508000B2E0052B00F0F68000F20981E0E0812B10
:1050900000F0B08009D80D2B00F03A81802B00F091
:1050A000A3800C2B40F0058320E1832B00F0D080FF
:1050B00000F2AA803EE1952B00F0708115D88C2B70
:1050C00000F05D8108D8872B00F03E81C0F0D280CF
:1050D0008A2B40F0EE823DE1932B00F0198100F223
:1050E00005818D2B40F0E58252E1A12B00F0F48187
:1050F00009D89A2B00F08281A02B00F0E781992B30
:1051000040F0D78265E1A32B00F0F081C0F0E88188
:10511000A42B00F0F181A52B40F0CB82FBE1B82B52
:1051200000F0818229D8AE2B00F0448211D8AA2B3E
:1051300000F01D8206D8A82B00F00E82644B00F20E
:10514000118204E2AC2B00F02482614B00F22D822C
:105150001AE2B22B00F0438206D8B02B00F0348262
:105160005B4B00F237822AE2B62B00F0448200F259
:105170005582B52B40F09D8235E2D12B00F057824D
:1051800016D8C32B00F05F8108D8C12B00F04F81E7
:1051900000F25281C02B40F08C828BE0C82B00F0D3
:1051A0005981CC2B00F06681C72B40F0828276E0DB
:1051B000D62B00F0748108D8D42B00F0638100F264
:1051C0006981D22B40F0758238E2D92B00F05482ED
:1051D00003D8D82B40F06D8245E2DA2B00F06182D3
:1051E000FE2B40F0668261E1394B00205A6801468F
:1051F000DB7804E0364B00205A68DB78022143EA72
:10520000022206F0A3FF59E2314C0020E3786268E5
:10521000082143EA022207F02DF8E378A1786268BA
:10522000490143EA0222002A41F00601B8BF524276
:1052300001F0E601002007F01DF8264AA378D318F4
:105240000122EEE1224B00205A680A21DB7876E049
:105250001F4C0020E3786268062143EA022207F02F
:1052600009F8E2786068A37842EA0020194A1A49EE
:105270009A180FE0164C0020E378616843EA012198
:1052800007F02CF9E2786068A37842EA0020114A1E
:1052900012499A1841F82300002313710EE20C4BB7
:1052A0000F4AD9780F4B01201B7810700E4A022B41
:1052B0005172D9E0064B0122D9780A4B1878084B75
:1052C0001A70094B9972002840F0F881CFE000BFB6
:1052D000E806002078020020700B00206C070020F8
:1052E0007C0C0020800C0020180C002014210020D1
:1052F00001AA06F0CBFEA04A9DF805305168D2788D
:1053000052EA012114BF43F0020323F0020354E0E8
:105310001421002001AA06F0B9FE974A9DF8053035
:105320005168D27852EA012114BF43F0010323F0FF
:10533000010342E0904B00205A68DB78042143EAE5
:10534000022206F097FFB9E18B4B00205A680E212C
:10535000DB78F4E701AC22461421002006F096FE2B
:10536000854B22469978DB78490141F0140101F020
:10537000F40100208DF8063007F024F89EE1E37870
:105380007E4AC3F10801C9B2D37205F0F3FB95E17F
:10539000794B00205A681A21DB78D0E7142101AA42
:1053A00006F074FE6168E2789DF8053052EA01214A
:1053B00014BF43F0040323F004038DF805306E4B53
:1053C0000020997801AA490141F0140101F0F4018B
:1053D000D2E701AC22461821002006F057FE664AAB
:1053E0009DF805309178D278490102F00F0223F040
:1053F0000F0341F0180142EA030311E001AC224619
:105400001821002006F042FE5B4A9DF80530917895
:10541000D278490103F00F0341F0180143EA021367
:1054200001F0F801224600208DF80530A4E7524B28
:10543000DA78524B1A7241E14F4B5A68DB7843EAF3
:1054400002224E4B33E1E378626843EA02224B4B7F
:105450005A6033E1484B4A4AD9784A4B01201B78BD
:105460001070464A032BD17740F028810138FFF7AE
:105470000BFB23E1404B5A68DB7843EA02223F4BA7
:10548000DA811BE13C4B5A68DB7843EA02223B4B52
:105490005A6113E1384BDA78384B9A770EE1E378AA
:1054A000626843EA0222354B9A8307E1324B334A62
:1054B0005968DB7843EA0121052904D8184613739B
:1054C000FFF7B4FAFAE000231373F7E02A4B002049
:1054D000D97805F041FBF1E0E17805F033FBEDE030
:1054E000254B0020D97805F00DFAE7E0224B00208B
:1054F000D97805F0FBF9E1E0002004F0B9FE1E4B7D
:1055000020B9D978987805F0D9F9D7E0D978987882
:1055100005F0A4F9D2E0002004F0AAFE164B20B951
:10552000D978987805F0BEF9C8E0D978987805F070
:105530007DF9C3E004F09CFEE178A37818B9184621
:1055400005F0A4F9BAE0184605F07CF9B6E0D97880
:10555000002005F08FF9B1E0074B0020D97805F065
:1055600093F8ABE0D978002005F082F8A6E0E17866
:1055700005F072F8A2E000BFE8060020180C002039
:105580007C0C0020800C0020D978002005F058F811
:1055900094E04B4C0020E17805F046F8A178494BA7
:1055A000E27803EBC1035A7188E0D978002004F057
:1055B000DFFF83E094F9031004F0CEFF7EE0D9789A
:1055C000002005F063FA79E03D4B0020D97805F022
:1055D00051FA73E0D978002005F040FA6EE0E178E6
:1055E00005F030FA6AE0364B5A68DB7843EA02226B
:1055F000354B9A6162E0324A324B5068D27842EAC7
:105600000020186010B9597905F00EF82C4B2F4A7C
:105610009878125C012A51D1D97828E7284BDA789A
:10562000284B1A714AE0E17805F054F946E06168C8
:10563000E37843EA0121FFF77DF93FE0204C0020A9
:10564000E378626803F01F0143EA02221E4B1A61ED
:10565000FEF7D2FFE3786168A07843EA012149119F
:10566000FEF7C2FF2AE0164B00205968DB7843EAB8
:105670000121FEF749FF21E0114C0020E378626828
:1056800003F01F0143EA0222114B1A60FEF76AFF82
:10569000E3786168A07843EA01214911FEF75AFFD7
:1056A0000CE0074B5A68DB7843EA0222094B1A6088
:1056B00004E0032200E00422074B1A701CBD00BF67
:1056C000E8060020880B0020180C0020800C002029
:1056D000A80B0020A40B00206007002013B5AD4CE0
:1056E000A078002840F072826378A62B00F0078231
:1056F000A94C7DD8852B00F00B813AD8092B00F0FE
:1057000032811CD8042B00F006810CD8012B00F04C
:10571000F680002B00F0F080022B00F0F680032BC7
:1057200040F05182F4E0062B00F0FA80C0F0F580E2
:10573000072B00F0F880082B40F04582F6E0802B24
:1057400000F0DA8009D80B2B00F01281C0F02E8116
:105750000C2B00F0F4800D2B24E0822B00F0338121
:10576000C0F0CD80832B00F0D680842B40F02B82BC
:10577000CBE09A2B00F055811ED88D2B00F039819B
:105780000BD8872B00F02481C0F0C7808A2B00F053
:1057900022818C2B40F0178225E1942B00F0CF80E2
:1057A00003D8932B40F00F82D3E0952B00F0258196
:1057B000992B40F008822AE1A12B00F077810BD8C9
:1057C0009C2B00F0F380C0F0D3809D2B00F0AE80C6
:1057D000A02B40F0F88165E1A32B00F06E81C0F0B2
:1057E0006881A42B00F06F81A52B40F0EC8178E15B
:1057F000C12B00F01E813BD8B02B00F0B0811BD82C
:10580000AB2B00F099810BD8A82B00F08981C0F058
:105810008381A92B00F08881AA2B40F0D48187E1F5
:10582000AD2B00F08F81C0F08A81AE2B00F08E810D
:10583000AF2B40F0C8818EE1B52B00F0A2810BD8D0
:10584000B22B00F09381C0F08D81B32B00F09281D8
:10585000B42B40F0B88191E1B72B00F09881C0F0F3
:105860009481B82B00F09681C02B40F0AC815AE0B7
:10587000D02B00F008811DD8C72B51D00BD8C32BDB
:1058800000F0DC80C0F0D880C42B00F0DA80C52B9B
:1058900040F09981D7E0CC2B00F0DA8003D8C82BF8
:1058A00040F09181D1E0CE2B00F0D580CF2B40F09D
:1058B0008A81D2E0D62B00F0EF800BD8D22B00F0FB
:1058C0007181C0F06B81D42B00F0E080D52B40F0CB
:1058D0007A81DEE0D92B00F06F8106D8D72B00F05B
:1058E0006481D82B40F06F8162E1DA2B00F0668191
:1058F000FE2B40F06881D2E00020014601E000204C
:10590000022106F071FB606063E10020082171E074
:1059100000200A2159E0214B00E0214B1B6832E1B5
:10592000204B5B7A2FE11F4B9B7A2CE1002006F085
:1059300071FA184B9B785B0050FA03F310E00020DB
:10594000142101AA06F0A2FB9DF80530C3F3400321
:1059500019E10020142101AA06F098FB9DF80530FA
:1059600003F001030FE1104B9B68C3F3C0330AE15E
:105970007C21002001AA06F089FB064B02219A78BF
:105980009DF80630520011FA02F21A420CBF0023B1
:105990000123F8E0E806002060070020700B0020DB
:1059A0006C070020180C00200008014001AA00200C
:1059B0007C2106F06BFB904B9DF806209B785B00EA
:1059C00052FA03F3CCE70020042106F047FB77E00E
:1059D00000200E21F9E701AA0020142106F056FB51
:1059E0009DF80620ECE0002004F022FCC0F1080045
:1059F00066E01A2106F032FB85E701AA0020142197
:105A000006F044FB9DF80520C2F38002D8E001AA0D
:105A10000020182106F03AFB9DF8052002F00F0245
:105A2000CEE0182101AA06F031FB9DF805301B09D4
:105A3000A9E0724B1B7AA6E0704BC0E06F4B5A682E
:105A4000BEE06F4BBBE06F4BB9E06C4BDA7FB7E069
:105A50006A4BDA89B4E06C4BB1E06C4A6C4B12785B
:105A6000002159600AB101225A606A4B674A1B78CB
:105A70000021117023B1664B5A6842F002025A604D
:105A80000022644BA4E0644B1B787CE05B4B5A69BA
:105A900096E05A4B9A7F93E0584B9B8B73E0574BA1
:105AA0001A7B8DE0002004F0CBFB09E004F0D0FB72
:105AB00029E7002004F0D4FB02E0002004F0D8FB2A
:105AC000534B586085E0002004F0D2FB504C4A4B09
:105AD00018B9987804F0DCFB15E7987804F0F8FB27
:105AE00011E7002004F0C4FB494C434B18B99878E7
:105AF00004F0D6FB07E7987804F0FAFB03E704F01C
:105B0000B7FBA378424C18B9184604F0D1FBFAE66B
:105B1000184604F0E5FBF6E6002004F0D1FBCFE7E1
:105B2000002004F0EDFBCBE7002004F0F1FBC7E719
:105B3000002004F0F5FBC3E704F0FAFBE3E6374B83
:105B40005A793DE0002004F003FCB9E7002004F09E
:105B500007FC40B2B4E7002004F014FCB0E704F006
:105B600019FCD0E6002004F01DFCA9E7002004F099
:105B700021FCA5E7002004F02DFCA1E7284B1A78B2
:105B80001EE01E4B9B69636023E0244B17E0234B10
:105B90001A7915E0002004F073FB91E70020FEF76E
:105BA000F3FE8DE7154B1A690AE0FEF783FD87E7E0
:105BB0000020FEF79DFC83E71A4B00E01A4B1A68A1
:105BC000134B5A6005E00323237002E0104B0422BC
:105BD0001A70164B1B786BB10D4B15495A68154B53
:105BE0000A601AB91A6842F0080202E01A6822F044
:105BF00008021A601CBD00BFE8060020180C002037
:105C00007C0B00203C0C0020B00B00200C0C002072
:105C100060070020940B0020100C0020880B00204F
:105C2000840B0020A80B0020A40B00205A070020A2
:105C300048070020F006002010B51B4A5378142BAB
:105C40002DD8917871B95468D078184A1849927E45
:105C500040EA042041F8230022B31BB303F5C270CD
:105C6000013013E0FF2918D163B94FF4C36411491F
:105C7000204609190422043402F070FDB4F5CD6FFA
:105C8000F5D10FE003F5C2700949013001EB830142
:105C90008000042202F062FD04E0042200E00322FE
:105CA000054B1A7010BD00BFE80600200800002058
:105CB000F4060020E00000206007002038B51F4CEB
:105CC0006578142D36D8A07810F0800F18D010F019
:105CD000010F06D00020022106F086F9184B43F888
:105CE0002500184B9B7E43B3144B5B782BB303F515
:105CF000C2701349013001EB83018000042214E0DB
:105D0000B0B9022106F070F90E4A0D4B927E43F8AD
:105D1000250092B1617881B1A0780422091801F5BB
:105D2000C270013003EB8101800002F017FD04E036
:105D3000042200E00322044B1A7038BDE80600205C
:105D4000F4060020080000206007002038B56E4CE3
:105D5000A07808B10422D3E063789A2B22D8992B3B
:105D600080F09B80822B00F081800BD8062B6ED0B8
:105D700003D8042B38D0052B0AE0072B6DD00C3B41
:105D8000012B0CE08C2B75D005D8832B2CD0862BC7
:105D900040F0B5803FE08D2B7DD0933B022B00F28D
:105DA000AE8060E0C72B52D00ED8C12B7AD005D878
:105DB000B52B74D0C02B40F0A2804EE0C22B77D020
:105DC000C32B40F09C8076E0D42B7DD005D8C82B27
:105DD00074D0CC2B40F0938073E0D62B7CD077D35B
:105DE000FE2B40F08C807DE0474D0020062106F020
:105DF00053FBAC780020610141F0060101F0E6019F
:105E000006F02CF9414AAB78D318414A42F82400F5
:105E100000221A7176E03C4D00200C2106F03CFB7C
:105E2000AC780020610141F00C0101F0EC0106F0BA
:105E300015F9AB78374A354942F8240018465B1803
:105E400052F8201000221A7106F048FB5AE049204F
:105E500002F06CFC304B587254E04A2002F066FCB1
:105E60002D4B98724EE00020142100E0042106F032
:105E700013FB47E04B200122284902F033FCA378B2
:105E8000254A184602EB4313D97AC1F10801C9B279
:105E900004F070FE36E01A21E9E71821E7E7582000
:105EA0001F4913E0482002F041FC1B4B187229E007
:105EB000402019490AE044201A4907E05F201A49A6
:105EC00008E04E20194909E019495420042206E04F
:105ED00018495E20012202E017495C20022202F0EC
:105EE00001FC0FE04C200122144902F0FBFBA278D8
:105EF000094B03EB4213187BFEF798FD02E00322E7
:105F00000F4B1A7038BD00BFE80600207802002051
:105F1000700B00206C070020180C0020230C0020C0
:105F2000300C00201C0C0020370C0020260C002018
:105F30002C0C0020360C0020340C0020240C0020F7
:105F40006007002010B51E4A5378142B34D892787D
:105F5000AAB91C4A1C4952F823201C4B4A601B78E2
:105F6000002B2CD01A491B4B0A601AB91A6842F050
:105F7000080202E01A6822F008021A601FE0FF2AF5
:105F800018D163B94FF4C364134920460919042298
:105F9000043402F0A7FBB4F5CD6FF5D10FE003F5A3
:105FA000C2700849013001EB83018000042202F035
:105FB00099FB04E0042200E00322034B1A7010BD99
:105FC000E8060020F4060020600700205A070020A1
:105FD00048070020F0060020E000002037B5134CF1
:105FE000657815B1012D1DD112E0042240F2FB703D
:105FF00001A902F077FBE378626843EA0222019B81
:106000009A420B4B02D101225A600EE05D600CE017
:10601000A3782A2B06D1E11C40F2FB70042202F087
:106020009DFB02E0024B03221A703EBDE8060020F1
:1060300060070020374938B500230B603649374ADE
:106040000B60374993740B609360D360137453747F
:10605000344A4FF0FF3142F82310334A0024D4541D
:1060600001332F2BF4D10731204605F0BDFF2F4B14
:106070000C211860204605F0B7FF2D4D2D4BE97A15
:106080001860C1F108012046C9B204F073FD287BF5
:10609000FEF7CCFC284B0022E2500434B4F5806FAC
:1060A000F8D1264B9B7E5BB104F50674244920464B
:1060B00009190422043402F015FBB4F5CD6FF5D1B3
:1060C0001E4BDB7E5BB94FF4A7641E4920460919BD
:1060D0000422043402F006FBB4F5C36FF5D1174B6C
:1060E0001B79012B03D0112B01D0212B01D10122CF
:1060F00000E00022094B83F8D020104B5B7D23B1D8
:10610000FEF780FA08B1012200E00022034B83F879
:10611000D12038BD48070020680700207802002001
:10612000F00600208C020020900C0020700B002054
:10613000180C00206C0700207007002008000020C9
:10614000E00000203802002008B50B4B5A7892B9C5
:10615000997881B95A68DB7843EA022240F2D24347
:106160009A4208D140F2FF7002F076FB02F038FC50
:106170000120FEF781FC08BDE806002010B59A4B0F
:106180009A78022A00F05A81032A00F06081002ADE
:1061900040F0F0815A784D2A00F0BD8023D8452A7E
:1061A00070D00ED8422A56D005D8402A45D0412A70
:1061B00040F0DE8146E0432A53D0442A40F0D881A3
:1061C00056E0482A7CD005D8462A61D0472A40F0BC
:1061D000CF816AE04B2A00F0858000F29580492A41
:1061E00040F0C68172E0542A00F0E48011D8512AB0
:1061F00000F0B18006D84F2A00F09380502A40F07A
:10620000B781A1E0522A00F0B880532A40F0B08153
:10621000BDE0832A00F0F58006D8552A00F0D7802B
:10622000572A40F0A581E5E0852A00F0FA80C0F009
:10623000F080FF2A40F09C81FCE06B4B40F2FF7045
:10624000D97805E0684B694ADB780020194613705D
:1062500002F002FB91E1DB78644A19460120537099
:10626000F6E7614B614ADB78042019461371EFE7CA
:106270005D4B5E495A68DB781C2043EA022341F8F3
:106280001C3F0EE0DB78594A194605205371DFE7C1
:10629000554B56495A68DB780C2043EA022341F8F3
:1062A0000C3F042202F05AFA67E14F4B4F4C5A68F8
:1062B000DB78214643EA022341F8083F082070E0DA
:1062C000DB784A49262001F8263F7EE0464A474BC4
:1062D000D27812B1464901224A60DA75434B172041
:1062E000D97DB5E7404B414CDB7803201946E3707C
:1062F00002F0B2FAE07802F087FCE07802F084FC69
:10630000E07802F0A9FC38E1374B384ADB7802200C
:10631000194693709CE7DB78344A1946152053756B
:1063200096E7314B314CDB7819201946637602F041
:1063300093FA607E10F0010002D00020012100E0FD
:10634000014605F085FF18E1274B284ADB78162027
:10635000194693757CE7254A127D12F0010F05D08E
:10636000DB7813F0010F01D102F03AFB1E4B1F4AFC
:10637000DB781420194613756AE71B4B1B495A68D2
:10638000DB78202043EA022341F8203F89E7164BBF
:10639000164C5A68DB78214643EA022341F8103F45
:1063A0001020042202F0DAF922696079A16802F073
:1063B000EFFFE2E05A68DB7843EA0222012A00F2AA
:1063C000D9800A491A2001F81A3F01226AE7064BD0
:1063D0005A68DB7843EA0222012A00F2CB800349A3
:1063E0001B2001F81B3FF0E7E80600200800002012
:1063F00060070020614B6249DB78272001F8273FC6
:10640000E3E75A68DB7843EA02225E4BC3F8D42004
:10641000B3E05A4B5A68DB7843EA02225A4B1A60BF
:10642000ABE0564B5A68DB7843EA0222554BC3F87F
:10643000D820A2E0514BDA78544B9DE05868D978C7
:106440005A78534B41EA002143F8221095E05A78DC
:10645000272A59D00ED8022A33D004D8CAB1012A2B
:1064600040F0868021E01B2A3ED01C2A44D0092A15
:106470007ED132E02B2A5FD005D8292A50D0D97896
:10648000444A54D847E02D2A64D05CD32E2A6FD1D9
:1064900067E05A68DB7843EA02223E4B1A6003F059
:1064A00073FA384BC3F8DC0067E05A68DB7843EADC
:1064B0000222384B5A6003F067FA324BC3F8E0000F
:1064C0005BE05A68DB7843EA0222324B9A6003F0C1
:1064D0005BFA2C4BC3F8E4004FE05A68DB7843EAE0
:1064E00002222C4BDA6048E05968DB78002043EA4E
:1064F000012105F0A7FF40E05968DB78002043EA5E
:10650000012105F073FF38E05A68DB7843EA022284
:10651000204B1A6131E05B6841EA032151612CE0B4
:106520005A68DB7843EA02221A4B9A6125E05B68DD
:1065300041EA0321D16120E05A68DB7843EA022274
:10654000144B1A6219E05A68DB7843EA0222114BB5
:106550005A6212E05A68DB7843EA02220D4B9A62D3
:106560000BE05A68DB7843EA02220A4BDA6204E065
:10657000032200E00422084B1A7010BDE806002038
:1065800008000020780200205C0700205907002046
:1065900070070020400C00206007002008B5824BE7
:1065A0009A78022A00F0B980032A00F0BB80002A02
:1065B00040F01E815B78502B6ED022D8462B54D0F1
:1065C0000ED8422B47D005D8402B3DD0412B40F070
:1065D0000D813EE0442B43D0744B754A43D83DE0D7
:1065E0004B2B4DD006D8482B43D040D3492B40F0FD
:1065F000FD8042E04D2B49D045D34F2B40F0F68033
:1066000047E0812B5FD010D8542B4ED005D8522BA9
:1066100047D0664B664A46D841E0572B4BD0802B7B
:106620004DD0552B40F0E28042E0852B5DD004D860
:10663000832B53D05D4B55D84DE0FE2B64D066D8EC
:10664000F02B40F0D3805FE040F2FF7002F06EF874
:106650009CE0574B59E0564B5A78C4E01279C3E09E
:10666000534BDA69BFE05279BEE0514B85E0504BA5
:1066700080E04F4B93F82620B5E04D4BDA7D48E0A3
:106680004B4BDA78AFE04A4B9A78ACE0484B5A7DF6
:10669000A9E0474B5A7EA6E0454B9A7DA3E0127DC8
:1066A000A2E0434B95E012699EE0414B9A7E9AE04E
:1066B0003F4BDA7E97E03E4B93F8272093E03D4B2B
:1066C00093F8D1208FE03B4B93F8D120042A14BFDC
:1066D0000022012287E0374A926885E0354BD3F8E3
:1066E000D42080E0344A12687EE0324A334BD2F83C
:1066F000D8104B4303F5405339332C4923F0004065
:106700004860C2F8D83076E02D4B1A786BE02D4BFC
:106710001A78003A18BF012265E05A782A4B53F8DC
:10672000222060E05B78272B33D00DD8022B20D0BD
:1067300003D8C3B1012B59D118E01B2B1FD01C2B40
:1067400021D0092B52D117E02B2B41D005D8292B72
:1067500024D0164B1D4A24D81EE02D2B3ED03AD310
:106760002E2B43D13DE0194B1A683CE0174B5A6879
:1067700039E0164B9A6836E0144BDA6833E00020B3
:1067800005F0AEFC02E0002005F096FC074B5860D7
:1067900031E00E4B1A6926E0526925E00B4B9A69ED
:1067A00021E0D26920E000BFE80600206007002059
:1067B00008000020780200205C0700206D4EC641D2
:1067C000740C00205907002070070020400C0020A6
:1067D000124B1A6A07E0114B5A6A04E00F4B9A6A8F
:1067E00001E00E4BDA6A0E4B5A6004E0032200E02F
:1067F00004220B4B1A700B4B1B786BB1084B0A49E8
:106800005A680A4B0A601AB91A6842F0080202E094
:106810001A6822F008021A6008BD00BF400C002070
:10682000600700205A07002048070020F0060020DB
:1068300010B5154CA07818BB6378012B16D003D384
:10684000022B124C19D114E004F07CFFA17839B16D
:106850000F4A937FBBB102EB4112927F9A4212D151
:106860000C4B01221A71013A0B4B0BE004F072FF42
:1068700009E004F077FF606005E00323237002E085
:10688000024B04221A7010BDE806002060070020A9
:10689000180C002078020020940B002037B5504BD4
:1068A0001A7CA2B94F494868CA7842EA0022B2F17C
:1068B000FF3F04BF4C4A12680A214A43C3F8E8204C
:1068C00003F062F8464B01221A74C3F8EC00454B02
:1068D0005B78042B00F28280DFE803F003353F4F42
:1068E000130003F051F83E4BD3F8EC10D3F8E82036
:1068F000411A0029B8BF494291426CD900221A744A
:106900006CE0384B364C987804F02CFF30B9374A9D
:106910002074136823F0100313605FE0D4F8E830AC
:10692000002B57D003F030F8D4F8EC20D4F8E8303E
:10693000821A002AB8BF52429A424BD92B4B0021EF
:106940001A68217442E0002005F064FA254B244CBB
:106950009D786D0050FA05F51CE000207C2101AA0D
:1069600005F094FB1F4B02229D789DF806306D00C8
:1069700012FA05F51A4C1D400EE001AA00207C21F8
:1069800005F084FB174A9DF806309578144C6D008D
:1069900053FA05F515F0010506D0144B00211A68CD
:1069A000217422F0100213E0D4F8E83093B102F021
:1069B000EBFFD4F8EC20D4F8E830821A002AB8BFF4
:1069C00052429A4206D9094B25741A6842F01002C5
:1069D0001A6003E0024B9A68013A9A603EBD00BF1C
:1069E00078020020E806002048070020F00600207A
:1069F00008B5184B9A7812B1022A26D106E05868D9
:106A0000DB7843EA0020FDF751FD21E058780728A4
:106A10000AD85A68DB7853EA022202D1FDF7EAFC71
:106A200016E0FDF7F3FC13E0FF280CD15868DB7883
:106A300043EA0020B0F1FF3F0ABF074BC0B218780D
:106A4000FDF7F0FC04E0032200E00422034B1A707F
:106A500008BD00BFE80600204807002060070020AE
:106A600010B5254B9A78012A28D003D3022A234C4B
:106A70002DD127E05878082802D8FDF7F1FD1AE05B
:106A80000A2804D11E4B9A68C2F340220CE00B285E
:106A900002D1FDF72FFE0EE00C2808D1184B9A68A2
:106AA00082F48052C2F30032144B5A6011E0FF2886
:106AB0000FD1FDF7EDFD114B58600AE0587802F058
:106AC0007FFFF8E75878FDF7C1FC606001E0042320
:106AD00023700C4B1B786BB1084B0B495A680B4B5E
:106AE0000A601AB91A6842F0080202E01A6822F035
:106AF00008021A6010BD00BFE806002060070020F1
:106B0000001001405A07002048070020F00600202E
:106B100010B5204B5A78812A3AD19A78922A37D1E7
:106B20009A79A32A34D15A79B42A31D11A79C52A4B
:106B30002ED1DB78D62B2BD1174B4FF400525A6154
:106B400003F0CAFA02F020FF044602F01DFF001B0A
:106B50000028B8BF4042B0F57A7FF6DBFDF794FC21
:106B600007F0E2F9002007F00FFF00210B4806F0C4
:106B700091FD0A4806F0EEFC094806F0A9F906F076
:106B8000D9FD4FF0804008F083FC0020FDF774FF32
:106B900010BD00BFE80600200010014008000240C0
:106BA000002401402DE9F3479D4A9E4DD07851685D
:106BB000137840EA01204FF0640C222B85F800C0C6
:106BC0006B70686000F0838554D80F2B00F03E8313
:106BD00024D8072B00F00A8210D8032B00F0F8808D
:106BE00006D8012B00F0A680022B40F0B187C8E048
:106BF000052B00F0F38100F2F58101E10B2B00F091
:106C0000E88205D8092B00F0DC8200F2DE82D4E2B3
:106C10000D2B00F0138300F21583F3E2192B00F023
:106C2000BD8412D8152B00F0C98306D8132B00F0B1
:106C30001183142B40F08C8774E3172B00F08E84A3
:106C4000794B00F29E8400F082BC1E2B00F0D084B1
:106C500009D81B2B00F0C484C0F0B0841C2B40F07A
:106C6000778700F0C0BC202B00F0C88400F2C984F4
:106C700000F0C1BC812B00F0D8852ED8412B00F04C
:106C8000BA8515D8252B00F0688507D8232B00F08E
:106C90002A85242B40F05C8700F031BD272B00F0C3
:106CA0009385C0F06585402B40F0528700F0A0BD71
:106CB000452B00F0AC8506D8432B00F0A28500F2EE
:106CC000A38500F09BBD472B00F0A785C0F0A285EF
:106CD000802B40F03D8700F0A3BD882B00F0478655
:106CE00012D8842B00F0EC8507D8822B00F0B585F4
:106CF000832B40F02D8700F0B5BD862B00F0FA8580
:106D000000F2558600F0F1BD8C2B00F09A8606D873
:106D10008A2B00F07D8600F28F8600F076BEF22B83
:106D200000F0E786FF2B00F005878D2B40F01087E1
:106D300000F08ABE9378FBB93B4B4FF0010C83F80F
:106D400004C03A4B00241C70394B21461C7020466D
:106D5000022205F023F92046062140F2FF7205F0D9
:106D600089FA2F4B20465A68DB78082143EA022231
:106D700005F080FA00F0EFBE2A4B04221A7000F0F2
:106D8000EABE274DAC78F4B9274B4FF0010C83F8DD
:106D900004C0264B21461C70254B20461C70022245
:106DA00005F0FCF82046062140F2FF7205F062FA79
:106DB0006A68EB78204643EA02225242082105F035
:106DC00059FA00F0C8BE174B04221A7000F0C3BE77
:106DD00094788CB9154B20461C70154B1C7004F030
:106DE000B9FC20462146022205F0D8F820460821A9
:106DF00005F054FA00F0AFBE04232B7000F0ABBED8
:106E0000074B9A78002A40F0E4805B78032B00F26D
:106E1000DB80DFE813F00F0049009400BA0000BFE8
:106E2000E806002060070020780200200C0C0020FB
:106E3000940B0020A64D0020FEF7E4F8A54EAB7899
:106E400000246868EA78F454A34E590142EA00220B
:106E5000F45401F0E001204605F078F9A9782246C3
:106E6000204605F09BF8A9789C4A02EB41139B7FD2
:106E7000002B00F07086002900F06D86927F9A4208
:106E800040F069862046FEF7BDF86A68EB78204638
:106E900043EA0222214605F059F9204621462246BE
:106EA00005F07CF800F057BE894D0020FEF7AAF8E7
:106EB000AB78884A00245901D454874A41F0020132
:106EC000D45401F0E201204605F08EF8EB786E68AC
:106ED000A97843EA06268619490101F0E001324605
:106EE000204605F033F92046A978224605F056F8E9
:106EF000A8787A4A7A4902EB40139B7F4E60002BB8
:106F000000F02986002800F02686927F9A4240F001
:106F10002286FEF777F80221204605F065F86A68B8
:106F2000EB78214643EA02228218204605F00EF94A
:106F300020462146224605F031F800F00CBE644C94
:106F4000E378626843EA0223142B19DC654A0020C7
:106F500052F82360FEF756F8A37832465D4E0025BE
:106F6000F5545D4E5901284601F0E001F55405F055
:106F7000EDF82846A1782A4605F010F800F0EBBDA0
:106F8000574B04221A7000F0E6BD514C0020E37804
:106F90006268002543EA0222524B53F82260FEF752
:106FA00031F8A37832464B4E5901F5544A4E2846E3
:106FB00001F0E001F55405F0C9F82846A1782A4609
:106FC00004F0ECFF00F0C7BD454B03221A7000F03F
:106FD000C2BD434B04221A7000F0BDBDFEF734F869
:106FE00000F0B9BDFEF77AFB00F0B5BD907818B19E
:106FF00004232B7000F0AFBD53789A2B21D8992B26
:1070000080F08480822B6FD00BD8062B4BD003D816
:10701000042B3CD0052B0AE0072B4BD00C3B012B5B
:107020000CE08C2B65D005D8832B30D0862B40F01C
:10703000BF8032E08D2B63D0933B022B00F2B880EF
:107040003FE0C82B00F083800FD8C12B6AD005D851
:10705000B52B60D0C02B40F0AB802BE0C32B6FD0A2
:1070600067D3C72B40F0A4801DE0D42B00F08480B0
:1070700005D8CC2B72D0D22B40F09A8075E0D62B5D
:1070800000F088807FD3FE2B40F0928089E00020C2
:10709000062105F039F800F05EBD00200C2105F056
:1070A00033F800F058BD0D4B4920597A01F0D4FB5C
:1070B00000F051BD094B4A20997A01F0CDFB00F058
:1070C0004ABD0020142105F01FF800F044BD00BFA8
:1070D000E8060020940B00200C0C0020180C002067
:1070E00060070020F4060020042105F00DF800F0F0
:1070F00032BD4B20A149012201F030FB00F02BBD35
:1071000000201A2105F000F800F025BD182104F038
:10711000FBFF00F020BD58209949042201F01EFB1E
:1071200000F019BD974B4820197A01F095FB00F04B
:1071300012BD40209349042201F010FB00F00BBD6A
:1071400044209149042201F009FB00F004BD5F20B6
:107150008E49012201F002FB00F0FDBC4E208C495B
:10716000022201F0FBFA00F0F6BC5020894904220B
:1071700001F0F4FA00F0EFBC54208749042201F03A
:10718000EDFA00F0E8BC5E208449012201F0E6FA45
:1071900000F0E1BC5C208249022201F0DFFA00F03D
:1071A000DABC4C207F49012201F0D8FA00F0D3BCB0
:1071B0007D4B03221A7000F0CEBCFEF7C7FD00F035
:1071C000CABCFEF7DBFF00F0C6BCFFF7E7F900F032
:1071D000C2BC9378022B11D15378372B0AD873494C
:1071E00003F5A77001EB83018000042201F0B6FAD9
:1071F00000F0B1BC03232B7000F0ADBC04232B7056
:1072000000F0A9BC6A4B9A78022A12D15B78372B1E
:107210000AD8664903F5A77001EB830180000232AA
:1072200001F060FA00F097BC5F4B03221A7000F087
:1072300092BC5D4B04221A7000F08DBCFFF7F8FA87
:1072400000F089BCFFF7D4FB00F085BCFFF708FC19
:1072500000F081BC5278574B092A53D8DFE802F07E
:10726000050D151D26313941494C514A19685068A0
:10727000D27842EA0022521843E04D4A1968506819
:10728000D27842EA00228A1A3BE0494A19685068DB
:10729000D27842EA00224A4333E0454A19685068EE
:1072A000D27842EA002291FBF2F22AE040481968C3
:1072B0004468C27842EA042291FBF2F002FB101209
:1072C0001FE03B4A19685068D27842EA00220A401F
:1072D00017E0374A19685068D27842EA00220A4318
:1072E0000FE0334A19685068D27842EA00224A40D7
:1072F00007E01A68D24304E02D4A5168D27842EA86
:1073000001221A602B4A2C4B12682AB91A6842F0E3
:1073100008021A6000F01FBC1A6822F008021A6006
:1073200000F019BC224B234A5968DB78126843EA03
:1073300001239A4206DD204B1A6842F0040222F033
:1073400003020CE01C4B05D11A6822F0060242F041
:10735000010204E01A6822F0070242F002021A60F9
:10736000144A154B126822B91A6842F008021A60D2
:10737000F1E31A6822F008021A60ECE3230C002003
:10738000300C0020180C00201C0C0020370C0020B2
:10739000260C0020280C00202C0C0020360C00208D
:1073A000340C0020240C002060070020700700200F
:1073B000E806002048070020F006002053780C2B38
:1073C00000F2C983DFE813F00D001B00290037002D
:1073D0004500530061006F007D008B009900A700FD
:1073E000B500944B1B6813F0080F00F0B483924B68
:1073F0005A68DB7843EA0222904B9A60ABE38D4BEC
:107400001B6813F0080F40F0A6838B4B5A68DB789B
:1074100043EA0222894B9A609DE3864B1B6813F076
:10742000010F00F09883844B5A68DB7843EA02220C
:10743000824B9A608FE37F4B1B6813F0010F40F083
:107440008A837D4B5A68DB7843EA02227B4B9A6041
:1074500081E3784B1B6813F0040F00F07C83764BBC
:107460005A68DB7843EA0222744B9A6073E3714BEB
:107470001B6813F0050F00F06E836F4B5A68DB78C2
:1074800043EA02226D4B9A6065E36A4B1B6813F076
:10749000020F00F06083684B5A68DB7843EA0222EF
:1074A000664B9A6057E3634B1B6813F0030F00F0C1
:1074B0005283614B5A68DB7843EA02225F4B9A6041
:1074C00049E35C4B1B6813F0100F00F044835A4BE8
:1074D0005A68DB7843EA0222584B9A603BE3554BEB
:1074E0001B6813F0200F00F03683534B5A68DB788B
:1074F00043EA0222514B9A602DE34E4B1B6813F076
:10750000400F00F028834C4B5A68DB7843EA022294
:107510004A4B9A601FE3474B1B6813F0800F00F043
:107520001A83454B5A68DB7843EA0222434B9A6040
:1075300011E3404B1B6813F4807F00F00C833E4B3B
:107540005A68DB7843EA02223C4B9A6003E33A4AEA
:107550005168D27842EA01229A60FCE2374BDA683D
:10756000072A00F2F88234499C684868C97841EAE1
:107570000020511C03EB8202C2F8F0409860D960F1
:10758000E9E2DA682D4B002A00F0E582013A03EBCC
:107590008201D1F8F010DA609960DCE253782E2B8A
:1075A00003D8274A0121D154D5E2FF2B03D1234B25
:1075B00001225A74CFE203232B70CCE21E4B5B787E
:1075C0002E2B03D81E4A0021D154C4E2FF2B03D135
:1075D0001A4B00225A74BEE21A4B03221A70BAE206
:1075E000FFF75CF9B7E2154B002283F8D120B2E235
:1075F000FEF722FBAFE2FEF7A5FCACE2FEF75EFB76
:10760000A9E20D4A104B52780A2A52D8DFE802F05C
:10761000060B20252B33393F45494C000B491A688E
:1076200009688A1803E0094A196812688A1A1A60F8
:107630003FE000BFF0060020E806002078020020AE
:10764000900C0020600700204807002068070020F9
:10765000934A196812684A43E9E7914A196812681F
:1076600091FBF2F2E3E78E4A1968126891FBF2F09F
:1076700002FB1012DBE78A491A68096801EA020274
:10768000D5E787491A68096841EA0202CFE78449C9
:107690001A68096881EA0202C9E7814B1A68D24375
:1076A000C5E71A687E4BC2E77D4A1868116810600A
:1076B00019607C4A7C4B126822B91A6842F00802B1
:1076C0001A6048E21A6822F008021A6043E2754B19
:1076D00001F07F4118681B7841EA10215160D37096
:1076E000FDF7B2FC37E26F4B01F07F4118681B7861
:1076F00041EA10215160D370FEF740FD2BE26B4B45
:107700005B78052B00F22782DFE803F003090F15F1
:107710001B21654B1A6802F00F021A601BE2624BD4
:107720001A6822F010021A6015E25F4B1A6822F004
:1077300020021A600FE25C4B1A6822F040021A60C5
:1077400009E2594B1A6822F080021A6003E2564B94
:107750001A6822F480721A60FDE153782E2B04D847
:10776000534A02EB83035861F5E103232B70F2E1E6
:107770004F4BDFF830C1D3F810914E4993F82C21CC
:10778000D3F814A1CCF80090DFF814C1D3F8187125
:10779000D3F81C81D3F82061D3F82451D3F82841C1
:1077A000CCF800A0885CDFF800C19F60CCF80080B6
:1077B0001E74C3F8EC50C3F8E84008B101238B54A1
:1077C0003B4B00229A74C6E193786BB9374B5B78D8
:1077D000142B05D8334A1168374A42F82310BAE10E
:1077E000364B03221A70B6E1344B04221A70B2E110
:1077F00002F0D0FCAFE102F0CFFCACE102F0CEFC35
:10780000A9E102F0CDFCA6E102F0CCFCA3E102F07C
:10781000CBFCA0E102F0CAFC9DE102F0C9FC9AE1B8
:10782000234B002283F8D12095E1537813B1012B2B
:1078300010D104E01E4B012283F8D1208BE1B0F57A
:10784000006F04D21A4A906082F8D13083E1042399
:107850002B7080E103232B707DE1154B022283F80E
:10786000D12078E1124B002199745974104A4FF0DD
:10787000FF3402F1140040F821400E480023435425
:1078800001312F29F2D1084913740B60054982F8A0
:10789000D1300B60024993600B60D3605BE100BFA5
:1078A0006807002048070020F0060020E8060020B6
:1078B00078020020900C0020F406002060070020D1
:1078C0008D4B1B7D13F0020F0CD1B0F5006F06D26B
:1078D0008A4B0422C3F8300183F8D1203BE1042312
:1078E0002B7038E108232B7035E1844B002283F89C
:1078F000D12030E1804B01219A78814BB0F5006FA7
:107900001970804B1A7028D27B4B1C7D0C4024D1FF
:10791000694601F0A9F87B4B9DF800709DF8016065
:107920009DF802509DF806C09DF805009DF80410D2
:107930009DF803201C725F709E70DD7083F804C098
:1079400058719971DA7101236E4A985C117A01338A
:107950004118082B1172F7D1FDE00123694A00217B
:1079600099540133082BF9D113781372F3E053784B
:107970008BB9614A01209178634A1468604A10709B
:10798000604A11700133E21812F8011C5D4A082B9D
:107990009954F7D1DFE0012B40F0DD801B222A71E2
:1079A0000422EA716FF07702AA716B71D3E0574B32
:1079B0005B78032B00F2CF80DFE803F002101D227A
:1079C0004E4A534BD2F8301192F8D1C0107C0A0ABB
:1079D000197183F807C098715A71BCE0474A4C4B43
:1079E000916892F8D1C0107C0A0A197183F807C017
:1079F00098715A71AFE0474B1A68454B5A60AAE03C
:107A0000454B1A68424B5A60A5E0FEF79DFBA2E089
:107A10005278424B02B101221A703C4B404AD8784E
:107A2000364B107093F834113E4A002311703E4AD1
:107A300013703E4A13708EE0304B012283F83521DB
:107A400089E0FEF7CBFA86E0304B5B78032B4CD80D
:107A5000DFE803F00C023C472C4B28495A68DB78DE
:107A6000D1F8381143EA022C00232BE0234BD3F842
:107A70003821092A0CD82549501C4C68C97803EBD9
:107A8000820241EA0421C2F83C11C3F8380162E0E5
:107A90001F4B09221A705EE052F82340581C6445BF
:107AA0000FD102EB8002013904E052F8040C0133DB
:107AB00042F8080C04328B42F7D3104BC3F838114C
:107AC00049E003468B421A4AE6D344E00B4A0023BE
:107AD000C2F83831164A0021D1500433282BF9D18D
:107AE00039E00B4B0A225A6035E0094B03221A7029
:107AF00031E0FFF70DF82EE00800002078020020AA
:107B00004C0700205007002000000020E80600205D
:107B1000600700204807002068070020800B002035
:107B2000AC0B00207E0C0020C40C00209C0B00201D
:107B3000B4030020094B5A68DB7843EA022240F282
:107B4000D2439A4207D1064B012283F8642102E016
:107B5000044B02221A70BDE8FC8700BFE806002033
:107B6000780200206007002073B5204B0246407861
:107B70001F4D1870907800265870D078EC46987099
:107B800010790C4698715079587192F806E095E892
:107B9000030083F804E0D2798CE80300DA70154B17
:107BA0001E70FEF7FFFF144B1B7873B963702370D0
:107BB0002B78A3706B78E370EB792371AB796371E9
:107BC0006B79A3712B79E37108E0012B06D10B4B84
:107BD0009B195B78A3550136082EF8D1044B6A46F1
:107BE00092E8030083E803007CBD00BFE8060020A4
:107BF000600700205A0700204C0700205007002093
:107C0000F7B5114D114C6F684FF0000C07F07F472E
:107C100047EA13276F600E4F6E4687F800C0287042
:107C20006970AA7094E80300EB7086E80300FEF721
:107C3000B9FF96E803006368227884E803000549E9
:107C400018460A70FEBD00BFE8060020600700204D
:107C50005A070020780200202DE9F04F834B9BB09B
:107C60001B781BB9824B93F865316BB1814B1B7844
:107C7000062B09D00A2B07D00F2B05D01F2B03D0C2
:107C80007B4B002283F83421794A92F83431591E13
:107C9000C9B2012946D892F866017749774ACC687B
:107CA0001278012B0CBF4FF0070C4FF0080C00238B
:107CB0000E948DF834C08DF835008DF83630CAB981
:107CC0006F4B8E681D7819795C7893F807C09879A6
:107CD0005B798DF83C608DF83D508DF83E408DF815
:107CE0003FC08DF840008DF841308DF842108DF87E
:107CF00043200AE0012A08D1624A0133995C1AA89C
:107D0000C218082B02F82D1CF6D15F4B1B78002BF4
:107D100040F024810DA801F059FA002840F01E819E
:107D200000F0DDBC032B25D192F8D040002C40F0B0
:107D3000E880524B1B7893B94F4D514CA8786E7820
:107D4000227863788619B618E279F618A379B618FE
:107D50006279F6182379B618F618F6B219E0012BF5
:107D600040F0FC80474BE05C013400F0B9FF092C87
:107D7000F8D1F3E0042B27D13F4D414CAB786E781E
:107D800018469E1901360023012222706360F6B264
:107D9000637000F0A5FF687800F0A2FF207800F083
:107DA0009FFF607800F09CFFE07900F099FFA079D8
:107DB00000F096FF607900F093FF207900F090FFCB
:107DC000304600F08DFFC9E0052B25D192F8D04058
:107DD000002C40F09680294B1B7893B9264D284CF7
:107DE000A8786E78227863788619B618E279F61842
:107DF000A379B6186279F6182379B618F618F6B290
:107E000019E0012B40F0AA801E4BE05C013400F029
:107E10004BFF092CF8D1A1E0062B37D1164D184C99
:107E2000AB786E7818469E19013600230122227025
:107E30006360F6B2637000F037FF687800F034FFDB
:107E4000207800F031FF607800F02EFFE07900F03C
:107E50002BFFA07900F028FF607900F025FF207942
:107E600000F022FF304600F01FFF77E059070020A6
:107E700078020020E8060020080000204C070020BF
:107E80006007002050070020780B0020072B3CD112
:107E900092F8D030002B34D1A74A127822BBA74ADF
:107EA000A74B557896781C7893F801C0AF19D8790C
:107EB000E719997967445A79C7191B79CF19D719E6
:107EC000DF198DF858708DF850608DF851508DF88D
:107ED00052408DF853C08DF854008DF855108DF830
:107EE00056208DF8573008E0012A06D1954A995C52
:107EF00014AAD1540133092BF8D1934B1B786BB3DF
:107F000028E08F4804F004FC28E0082B26D18B4B96
:107F10000022597898788C4B45181C78884B4FF084
:107F2000010C01355A608DF852C08DF85320164669
:107F30008DF854208DF855208DF856208DF8572057
:107F40008DF858505A7083F800C08DF850008DF8A5
:107F500051101CB114A8092101F08CFF7B4B1B7838
:107F6000002B00F081807A4A774B1278794C013AE5
:107F7000062A74D8DFE802F004042A7373734E00F3
:107F80006E4A94F800C0D068926819788DF82C2059
:107F90006FF07F028DF82D200A3200238DF82E20FD
:107FA0007D328DF832C08DF824208DF826300A906D
:107FB0008DF82F308DF830308DF831308DF8253038
:107FC00000294CD109A801F001F948E05B4D227865
:107FD000AB786E7818469E190A36B61800F080FE07
:107FE000687800F07DFE802000F07AFE8A2000F0A4
:107FF00077FE002000F074FE002000F071FE0020EB
:1080000000F06EFEF6B2207800F06AFE304600F016
:1080100067FE24E049482278417880786FF07F0538
:1080200000EB010C1C780CF10A0C002394448DF831
:1080300046500A358DF847508DF84A308DF84CC0BF
:108040008DF844008DF845108DF848308DF8493092
:108050008DF84B201CB111A8092101F00BFF3B4A00
:10806000002313703B4A13703B4B334893F8641161
:108070000022027083F8652183F8342111B10120B8
:10808000FCF7FAFC344B93F8352152B193F8D02029
:108090000021D2F1010238BF002283F8351183F8A4
:1080A000D020294B1B78002B5ED10DA801F06CF875
:1080B000002859D09DF83430062B55D9274B1F4A3C
:1080C0009DF83C709DF83D609DF83E509DF83F4006
:1080D0009DF840E09DF841C09DF84280116983F809
:1080E00003801F705E709D709C7183F805E083F8BB
:1080F00004C00E9B184A9DF835008B4282F8660139
:1081000002D1012382F8653101F03EFC9DF8343044
:108110004FF00002072B124B0F4C1860114B1A70D6
:1081200001D1012300E0022384F834310A4B93F893
:10813000D1305A1ED2B25FE14C0700200800002067
:108140006007002050070020780B0020C40C00209E
:108150007E0C00209C0B002078020020E806002006
:10816000700C0020790B0020A84C94F8D050002D02
:1081700072D10DF1670000F031FD00286CD000F0E5
:1081800049FD08B184F86751A04B9DF8670093F84A
:1081900067114A1CD2B2C918092A81F8680183F80C
:1081A000672140F05F819A4993F8682148784FF041
:1081B000000C904283F867C107D091F82730002B5C
:1081C00000F050819A4240F04D81914B93F8273056
:1081D000934203D18D4B012283F8652100231A4677
:1081E0008A4C04F5B471C95C01335218082BD2B221
:1081F000F6D194F8703193422CD1864B94F86D11DE
:1082000094F86E2194F86F5194F8696194F86AE1DA
:1082100094F86BC194F86C01DD7059711A711E707D
:1082200083F801E083F802C0987101F0ADFB7A4D4C
:1082300094F8D1302860591E78480022C9B20270E3
:108240000320012984F8340184F8672140F2D880A2
:10825000052B8AE00423D5E06C4C94F8D03083B130
:108260006C4804F09BFA60B101F08EFB6A4994F807
:10827000D130086069495A1E00200870D2B203212B
:10828000B8E0624C94F8D050002D73D10DF1670026
:1082900000F0CAFC00286DD000F0E4FC08B184F8BE
:1082A00067515A4B9DF8670093F867114A1CD2B288
:1082B000C918092A81F8680183F8672140F0D28043
:1082C000534993F8682148784FF0000C904283F8A6
:1082D00067C107D091F82730002B00F0C3809A4285
:1082E00040F0C0804A4B93F82730934203D1474B6C
:1082F000012283F8652100231A46444C04F5B47129
:10830000C95C01335218082BD2B2F6D194F87031FF
:1083100093422DD13F4B94F86D1194F86E2194F84F
:108320006F5194F8696194F86AE194F86BC194F81C
:108330006C01DD7059711A711E7083F801E083F8C9
:1083400002C0987101F020FB334D94F8D1302860C1
:10835000591E32480022C9B202700520012984F852
:10836000340184F867214BD9834249D0013272E04D
:10837000062347E0254B93F8D040002C52D1284BE0
:108380001B78002B4ED017A801F05EFD002849D0C5
:108390002346224617A9C95C01335218082BD2B2D2
:1083A000F8D19DF86410194C91422BD1194B9DF8CE
:1083B00061109DF862209DF85D609DF85EE09DF87B
:1083C0005FC09DF860009DF8635059711A711E706E
:1083D000DD7083F801E083F802C0987101F0D4FAEF
:1083E0000D4994F8D13008600C495A1E00200870DD
:1083F000D2B2072184F83411012A01D9052B29D1E1
:10840000002228E084F834312CE000BF78020020FC
:1084100008000020E8060020780C00207D0C0020D9
:10842000780B0020A14C94F8D130013BDBB2012B3A
:1084300018D8A368B3F5006F10D2FCF7E3F868B161
:10844000A3689B4918460133A36000F00DFB092384
:1084500084F834310122974B1A7003E0934B0022C9
:1084600083F8D120914C94F8D130042B05D1904E53
:10847000327812F0800F00F0EF808C4B93F834319B
:108480003BB1042B05D0082B03D0062B01D0FEF7FF
:1084900089FB864C94F83431092B40F0B28001F00E
:1084A00073FAD4F8DC30844AC31A002B1268B8BFC0
:1084B0005B4293420AD9814B1A78012A01D10132D9
:1084C0001A7001F061FA794BC3F8DC0001F05CFA34
:1084D000764BD3F8E020784B821A002A5B68B8BF4D
:1084E00052429A420AD9754B5A78012A01D1013277
:1084F0005A7001F049FA6D4BC3F8E00001F044FAFC
:108500006A4BD3F8E4206C4B821A002A9B68B8BFF0
:1085100052429A420AD9694B9A78012A01D1013212
:108520009A7001F031FA614BC3F8E4005F4A537C62
:10853000002B66D0937C002B63D19C46604BD2F815
:10854000EC001B68D2F8E81007935E4B04901B68A0
:10855000D2F8108106935C4BD2F814711B68D2F8E4
:108560001841059392F82C31D2F81C610293107CCB
:108570009368D2F82051D2F824B1D2F8282103917F
:1085800001926246DFF83491194619F802A0BAF157
:10859000020F18D14D4951F82210B1F1FF3F0ED012
:1085A0000546D0B202900398DDF810B00190059E08
:1085B000069FDDF81C804FF0010C002004E0002134
:1085C00009F802101946234601322F2A02D01C4610
:1085D0000B46D7E7354A9160C2F818310199029BE2
:1085E00082F812C0C2F81081C2F81471C2F81C617E
:1085F0001074C2F82051C2F824B1C2F8281182F8D0
:108600002C312A4B93F83421092A06D193F8D12032
:10861000022A02D1033283F8D120244BD3F8381137
:1086200000295CD093F83421092A58D193F8D1203D
:10863000012A54D19868002308E054F823400133FC
:10864000A04203D1052382F8D13048E0174A8B427B
:1086500002F59E74F1D342E094F83431002B3ED001
:10866000042B3CD0082B3AD0062B38D0F378716815
:10867000D4F83001164D43EA0123B0F5006F6A705B
:108680006B6027D2314600F01FF93146D4F8300133
:1086900000F042F930B1D4F830310133C4F8303150
:1086A000652300E007232B7019E000BF780200204B
:1086B000E80600205A070020400C0020900C002003
:1086C0004807002068070020F00600208C020020E8
:1086D0006007002007232B70002384F8D1301BB0E3
:1086E000BDE8F08F70B5044600200E461546032104
:1086F0000246FCF70BFB0020C4F307210246FCF7FF
:1087000005FB0020E1B20246FCF700FB002407E075
:10871000944214BF00220122FCF7F8FA30550134CC
:1087200000206A1EAC420146F2D370BD10B504466B
:10873000002003210246FCF7E9FA0020C4F30721D8
:108740000246FCF7E3FA0020E1B20246FCF7DEFA4B
:10875000002001460122FCF7D9FA10BD2DE9F041B5
:1087600004460F461646002006210122FCF7CEFAE9
:10877000002005210246FCF7C9FA0020012201462B
:10878000FCF7C4FA10F0020FF2D0002002210246DA
:10879000FCF7BCFA0020C4F307210246FCF7B6FA46
:1087A0000020E1B20246FCF7B1FA002543E00134B3
:1087B00014F03F08795D01D1012204E0721E954258
:1087C00014BF002201220020FCF7A0FAB8F1000F2C
:1087D00030D1731E9D422DD2002005210246FCF7A8
:1087E00095FA002001220146FCF790FA10F00100F2
:1087F000F2D106210122FCF789FA00200521024668
:10880000FCF784FA002001220146FCF77FFA10F001
:10881000020FF2D0002002210246FCF777FA002076
:10882000C4F307210246FCF771FA0020E1B20246C8
:10883000FCF76CFA0135B542B9D300200521024698
:10884000FCF764FA002001220146FCF75FFA10F001
:10885000010FF2D1BDE8F08138B5012204460D4682
:1088600000200621FCF752FA002005210246FCF701
:108870004DFA002001220146FCF748FA10F0020FE1
:10888000F2D0002002210246FCF740FA0020C4F397
:1088900007210246FCF73AFA0020E1B20246FCF753
:1088A00035FA294600200122FCF730FA0020052184
:1088B0000246FCF72BFA002001220146FCF726FABB
:1088C00010F0010FF2D138BD38B50725454305F545
:1088D00000650C46284609780135FFF7BDFF28469C
:1088E00061780135FFF7B8FF2846A1780135FFF719
:1088F000B3FF2846E1780135FFF7AEFF284621791E
:108900000135FFF7A9FF28466179FFF7A5FF681C2D
:10891000A179FFF7A1FF38BD2DE9F34707254543AE
:1089200000200C4602460321FCF7F0F905F500652E
:108930000020C5F307210246FCF7E8F90020E9B260
:108940000246FCF7E3F9002001460246FCF7DEF997
:108950008246002001460246FCF7D8F980460020F6
:1089600001460246FCF7D2F90746002001460246BE
:10897000FCF7CCF98146002001460246FCF7C6F917
:108980000646002001460246FCF7C0F905460020D5
:1089900001220146FCF7BAF9237853451DD16378CB
:1089A00043451AD1A378BB4217D1E37821798DF8DA
:1089B00004608DF805508DF80600627943EA0123C2
:1089C00043EA0243A079019A43EA006049EA022996
:1089D000814514BF0020012000E00020BDE8FC8795
:1089E00038B54FF40064002006210122FCF78EF90F
:1089F000002005210246FCF789F9002001220146EA
:108A0000FCF784F910F0020FF2D000200221024698
:108A1000FCF77CF90020C4F307210246FCF776F945
:108A20000020E1B20246FCF771F9002500203F2D3D
:108A300014BF0022012201460135FCF767F9402DE1
:108A4000F4D1002005210246FCF760F90020012244
:108A50000146FCF75BF910F0010FF2D14034B4F598
:108A6000804FC0D138BD00BF38B507254543002031
:108A70000C4602460321FCF749F905F50065002084
:108A8000C5F307210246FCF741F90020E9B202468E
:108A9000FCF73CF9002001460246FCF737F920704C
:108AA000002001460246FCF731F9607000200146C3
:108AB0000246FCF72BF9A070002001460246FCF7A5
:108AC00025F9E070002001460246FCF71FF92071ED
:108AD000002001460246FCF719F9607100200146AA
:108AE0000122FCF713F9A07138BD00BF37B5002093
:108AF00005210246FCF70AF9002001220146FCF795
:108B000005F910F07104F2D100F03EFF054605E0D2
:108B1000FFF70CFE422814BF0024012400F034FFAC
:108B2000431B002BB8BF5B42B3F5FA6F40F2FF70F6
:108B300002DA002CECD000E01CB1234B1B78002B98
:108B400036D040F2FF700021FFF786FEFFF748FFA6
:108B500000201E494022FFF701FE4FF480701C499F
:108B6000B422FFF7FBFD40201A492022FFF7F6FD53
:108B7000002301934FF4C36401AD20460422043462
:108B80002946FFF7EBFDB4F5FF6FF5D10023019304
:108B9000A4F530742046042204342946FFF7DEFD94
:108BA000B4F5C36FF6D140F2FF704221FFF754FED7
:108BB000002040220549FFF795FD4020064920226C
:108BC000FFF790FD3EBD00BFB40B00200800002061
:108BD000102C0108402C0108180C0020094B1968C2
:108BE0005A68914201D100200BE01A68D118097A25
:108BF000013201701A601A68202A01D100221A601D
:108C000001207047EC030020014B9862704700BFC1
:108C1000EC030020034B1A78104612B100221A70A0
:108C200001207047D80C00200A4BD96A1A6B914278
:108C300001D100200CE0DA6AD11891F83410013229
:108C40000170DA62DA6A202A01D10022DA62012098
:108C5000704700BFEC030020014B5865704700BF10
:108C6000EC030020034B1A78104612B100221A7050
:108C700001207047D90C002008B5FBF705FC034B19
:108C80000022DA621A63FBF7FDFB08BDEC0300204B
:108C900008B5FBF7F9FB034B00221A605A60FBF79B
:108CA000F1FB08BDEC03002038B50B4B84469C6DEE
:108CB000DA6D0134202C08BF002494420AD09D6D47
:108CC0000648ED1885F860C040F2277101229C65C6
:108CD00006F076FC38BD00BFEC03002000440040E5
:108CE00038B50D4B8446D3F88040D3F88420013446
:108CF000202C08BF002494420CD0D3F880500748A1
:108D0000ED1885F888C040F227710122C3F8804031
:108D100006F056FC38BD00BFEC03002000480040C0
:108D200038B50546002401E0FFF7DAFF2B5D01347A
:108D30001846002BF8D138BD2B4910B50B8813F01D
:108D4000200F1DD0294BDB6813F0020F01D08B8858
:108D500016E0274B1A6BD86A0132202A08BF00227E
:108D6000824206D01C6B8888E118C0B281F83400BA
:108D70001A63204B0A221A601D4B5A6D1E4B1A6053
:108D80001948038813F0800F1BD01B4B1A68C2B917
:108D9000174B9C6DD96D8C420FD0144902240C6185
:108DA000D96DCC1894F860C00131A0F804C0D96521
:108DB000D96D202905D1DA6503E040F2277106F06C
:108DC000FFFB0948038813F0400F0BD040F22661E7
:108DD00006F0EEFC064BDA6D9B6D9A4202D1034B16
:108DE00002225A6110BD00BF00440040000801404B
:108DF000EC030020C80C0020D00C0020274910B53F
:108E00000B8813F0200F15D0254B5A6818680132D3
:108E1000202A08BF0022824205D05C688888E118B9
:108E2000C0B208725A601F4B0A221A601C4B9A6A21
:108E30001D4B1A601948038813F0800F1ED01A4B7F
:108E40001A68DAB9164BD3F88040D3F884108C42F4
:108E500010D0D3F88410CC1894F888C00131A0F851
:108E600004C0C3F88410D3F88410202906D1C3F8B5
:108E7000842003E040F2277106F0A2FB0748038834
:108E800013F0400F08D040F2266106F091FC044B2D
:108E9000D3F88420D3F8803010BD00BF00480040D4
:108EA000EC030020D40C0020CC0C002030B505468B
:108EB00087B0564806F0CCFC4FF40030012105F095
:108EC00015FB0420012105F003FB0420002105F01F
:108ED0001BFB0820002104F083FF06AC4FF00403C5
:108EE00024F8083D03234A4821468DF812301533F3
:108EF0008DF8133004F0E4FE482345488DF8133014
:108F000021464FF00803ADF8103004F0D9FE684652
:108F100006F020FB0B2D25D8DFE805F02406090C10
:108F20000F1215181B1E20224FF461531CE04FF442
:108F3000964319E04FF4E14316E04FF4164313E073
:108F40004FF4614310E04FF496330DE04FF4E133FA
:108F50000AE04FF4613307E02E4B05E02E4B03E0AF
:108F60002E4B01E04FF416530093009B06A95B08BB
:108F700041F8183D2548694606F022FC26230024C6
:108F8000012505A88DF8143007238DF815308DF8CC
:108F900016408DF8175005F003F81C4840F2FF31D9
:108FA00006F0E2FB28212246184806F009FB2A4673
:108FB000164840F2277106F003FB2A46134840F298
:108FC000266106F0FDFA2A46104840F2255106F0C7
:108FD000F7FA22460D4840F2244106F0F1FA224603
:108FE0000A4840F6460106F0EBFA2246074840F6EA
:108FF0006A1106F0E5FA60212246044806F0E0FA1C
:109000002946024806F0CEFA07B030BD00440040C1
:109010000008014090D0030020A1070040420F004B
:1090200030B5054687B0524806F012FC4FF4802058
:10903000012105F05BFA4F48002104F0D1FE06AC97
:109040004FF4806324F8083D03234B4821468DF8F4
:10905000123015338DF8133004F032FE48234648A1
:109060008DF8133021464FF40063ADF8103004F052
:1090700027FE684606F06EFA0B2D25D8DFE805F0CE
:109080002406090C0F1215181B1E20224FF46153E1
:109090001CE04FF4964319E04FF4E14316E04FF41F
:1090A000164313E04FF4614310E04FF496330DE0A4
:1090B0004FF4E1330AE04FF4613307E02F4B05E052
:1090C0002F4B03E02F4B01E04FF416530093009B0E
:1090D00006A95B0841F8183D2548694606F070FB73
:1090E00027230024012505A88DF8143007238DF8C7
:1090F00015308DF816408DF8175004F051FF1C48BC
:1091000040F2FF3106F030FB28212246184806F0D5
:1091100057FA2A46164840F2277106F051FA2A46B5
:10912000134840F2266106F04BFA2A46104840F2F6
:10913000255106F045FA22460D4840F2244106F03A
:109140003FFA22460A4840F6460106F039FA22461E
:10915000074840F66A1106F033FA602122460448B7
:1091600006F02EFA2946024806F01CFA07B030BD78
:109170000048004010001400000C014090D0030093
:1091800020A1070040420F0030B50C4B0C4C844628
:1091900022681B689A4201D100200EE02368094A28
:1091A0005D1C02EB03130FCB8CE80F0025602368D6
:1091B000082B01D100232360012030BD680D002061
:1091C000DC0C0020E80C0020704700BFF0B54378AD
:1091D00087B00646426833B104238DF80C30002373
:1091E0000292019303E0019202938DF80C30B37860
:1091F00003B102238DF80D30327800238DF80E2054
:10920000F21801A8117AC2180133082BD172F7D1D4
:1092100003F098FF042818D10D4D0E4B2C681B68E5
:109220000134082C08BF00249C4201D100200DE02D
:1092300096E80F002F68084E06EB071C8CE80F001D
:10924000012001462C6003F06FFF012007B0F0BD44
:10925000E00C0020E40C00206C0D00207FB52B4BAF
:109260002B4A19681268914204D10120002103F0B1
:109270005BFF48E01968274A02EB0111487850B1BA
:109280001B6802EB0312536804228DF80C200022A5
:109290000192029307E01B68029002EB03125368ED
:1092A0008DF80C000193194B1A681A4B03EB02134B
:1092B0009B781BB102238DF80D3001E08DF80D3045
:1092C000124B00221968134B0901CB5C8DF80E304C
:1092D0000E4B0DF1180C18680CEB020102EB001C90
:1092E0000C4801326044007A082A01F8090CEFD1D9
:1092F0001A6801321A601A68082A01D100221A601D
:1093000001A803F01FFF07B000BD00BFE40C002060
:10931000E00C00206C0D002073B50220002103F04A
:1093200003FF1020002103F0FFFE01AC002101200B
:1093300003F0FAFE00250726142320468DF804309A
:109340008DF805608DF806508DF8075004F028FE62
:10935000152320468DF804308DF805608DF80650F1
:109360008DF8075004F01CFE204613238DF80430BE
:109370008DF805608DF806508DF8075004F010FE4A
:1093800004F0DCF829464FF0007005F0AFF87CBD22
:109390002DE9F04101388AB00C46154607285BD804
:1093A000DFE800F04C4034281C5A10040C238DF8E0
:1093B0001C3003238DF81D3000238DF81B304FF037
:1093C000020354E00C238DF81C3003238DF81D306C
:1093D00000238DF81B304FF004023AE00C238DF887
:1093E0001C3003238DF81D3000238DF81B304FF007
:1093F00010022EE00C238DF81C3003238DF81D3055
:1094000000238DF81B304FF0140330E00C238DF84F
:109410001C3003238DF81D3000238DF81B304FF0D6
:10942000280216E00C238DF81C3003238DF81D3024
:1094300000238DF81B304FF0640318E00C238DF8E7
:109440001C3003238DF81D3000238DF81B304FF0A6
:10945000C802ADF81E200CE00C238DF81C3003234D
:109460008DF81D3000238DF81B304FF00803ADF848
:109470001E3004F063F801214FF0007005F036F85B
:109480000120014605F024F80820012105F020F80C
:109490000820002105F038F801214FF4EA1004F00B
:1094A0009FFC0AAE4FF4007226F8042D03233146C8
:1094B0008A488DF8263015338DF8273004F000FCEB
:1094C0000423314685488DF827304FF480730026F9
:1094D0000127ADF8243004F0F3FB05A88DF81A60DD
:1094E0008DF814608DF815708DF816608DF8176082
:1094F0008DF818708DF8197003F014FDB4F5006F35
:1095000001A815DA4FF0FF326301ADF80830ADF86D
:1095100010608DF812708DF804608DF805608DF87C
:109520000670ADF80A60ADF80C20ADF80E2013E01F
:109530004FF0FF338DF80670ADF810608DF81260B3
:109540008DF804608DF80560ADF80860ADF80A602C
:10955000ADF80C30ADF80E3003F056FDDDB1B5F5C9
:10956000006F18DA002201236901ADF80A208DF896
:1095700005204FF0FF3201A8ADF808108DF8123029
:109580008DF804308DF80630ADF80C20ADF80E20C3
:10959000ADF8103016E000230122ADF80A308DF846
:1095A00012308DF80530ADF808304FF0FF3301A8C8
:1095B000ADF810208DF804208DF80620ADF80C30A1
:1095C000ADF80E3003F020FDE30043F004030DF18D
:1095D00004080027012602226413ADF80A30404631
:1095E0004FF0FF338DF80420ADF808408DF805707A
:1095F0008DF80660ADF80C30ADF80E30ADF8107097
:109600008DF8126003F000FDBD421ADDEB0043F05F
:1096100004036D130322ADF80A304FF0FF334046C8
:109620008DF804208DF80570ADF808508DF81260A3
:109630008DF80660ADF80C30ADF80E30ADF8106066
:1096400017E003238DF804304FF004024FF0FF338E
:109650004046ADF80870ADF810608DF812708DF8C6
:1096600005708DF80660ADF80A20ADF80C30ADF845
:109670000E3008AF03F0C8FC012407260025142390
:1096800038468DF820308DF821608DF822508DF805
:10969000234004F085FC152338468DF820308DF8E2
:1096A00021608DF822508DF8234004F079FC1323BB
:1096B00038468DF820308DF821608DF822508DF8D5
:1096C000234004F06DFC0220214603F02DFD2146CD
:1096D000102003F029FD0AB0BDE8F081000C014024
:1096E00030B52A4D2A4B2C681B680134082C08BF62
:1096F00000249C4287B044D0012001A903F0FEFD64
:109700009DF80C20234B042A09D12A68012103EB80
:10971000021251702A6803EB0213029A08E02A68C9
:10972000002103EB021251702A6803EB0213019A25
:109730005A609DF80D30154A022B164B04D1126861
:1097400003EB0213012203E0126803EB0213002271
:109750009A700E4B9DF80E101A680E4B1201D154E0
:1097600000230A4A06A9C81811680A4D03EB011123
:1097700010F8090C01334919082B0872F1D1146053
:1097800002E0012003F09EFD07B030BD680D00200F
:10979000DC0C0020E80C002030B52A4D2A4B2C6848
:1097A0001B680134082C08BF00249C4287B044D0B9
:1097B000002001A903F0A2FD9DF80C20234B042AF0
:1097C00009D12A68012103EB021251702A6803EBC8
:1097D0000213029A08E02A68002103EB021251707A
:1097E0002A6803EB0213019A5A609DF80D30154A5E
:1097F000022B164B04D1126803EB0213012203E083
:10980000126803EB021300229A700E4B9DF80E10A3
:109810001A680E4B1201D15400230A4A06A9C8182F
:1098200011680A4D03EB011110F8090C01334919B5
:10983000082B0872F1D1146002E0002003F042FD11
:1098400007B030BD680D0020DC0C0020E80C0020C3
:10985000F0B5404B1A78AAB159683F4A01315960B6
:1098600011683E4B013111601A6812B11A68013A51
:109870001A603B4B1A6812B11A68013A1A6000224A
:10988000344B00E001221A70364B1A683AB11A685C
:10989000013A1A601B6813B9334B01221A70334B1B
:1098A0001A683AB11A68013A1A601B6813B9304B4A
:1098B00001221A702F4B304A9B8C30499BB21360A7
:1098C00010680B68984218DD146808682C4B201A41
:1098D000B0F5004F2B4806DAD3E900451668096851
:1098E0000268701A29E0D3E900450E68116806F590
:1098F000803C0268C1EB0C0011E010680B689842D4
:1099000023DA0C6810681E4B201AB0F5004F1D4872
:109910000ADAD3E900450E6811680268701A5043EC
:10992000261A65EBE0770CE0D3E900451268096878
:1099300002F5803C0268C1EB0C005043261845EB51
:10994000E07730463946C3E900010B4B1A680B4BF0
:109950001A60F0BD940400205C070020CC0C0020AD
:10996000D00C0020D40C0020D80C0020C80C002003
:10997000D90C002000040040C00C0020980B0020EF
:10998000B80B0020C00B0020014B5868704700BF87
:109990009404002008B5042004F0CAFF48F6A04053
:1099A00004F0D6FF012004F0D9FF0448032100226F
:1099B00004F0C4FB012004F0E7FF08BD9AC30200D5
:1099C000F8B5092806D8DFE800F0070A05050505FF
:1099D00005050E1600205CE03B4B188801E03A4B71
:1099E000588880B255E0384B988840F2F72380B20F
:1099F000584300134DE0344BD88880B208F052FB36
:109A000007F034FF0022314B07F084FF22A3D3E993
:109A1000002306460F4607F07DFF21A3D3E900236C
:109A200007F0C6FD1EA3D3E9002304460D463046C9
:109A3000394607F06FFF0022254B07F06BFF024607
:109A40000B462046294608F08FF808F025FA07F063
:109A50000DFF00221F4B08F087F807F0AFF912A3A3
:109A6000D3E9002307F056FF11A3D3E9002307F041
:109A70009FFD02460B4610A1D1E9000108F074F8E1
:109A80000FA3D3E9002307F091FD08F005FA08F0D1
:109A900027FDF8BDAFF300806666666666660AC09D
:109AA0006666666666660A40C3F5285C8FA27240E9
:109AB0000000000000FEAA409A999999FD6F2F417D
:109AC000C3F5285C8F1271409C0400200000303FD9
:109AD0000000E03F00002440F0B593B000240325CF
:109AE0004FF03303404811A9ADF844308DF846508B
:109AF0008DF8474004F0E4F80120014604F0DAFC58
:109B000001214FF4007004F0E3FC384803F022FD1B
:109B1000374B04270193374B344802938023069335
:109B2000DB18079303F540730893A3F578730DEBE7
:109B30000701099303F5FF530A93039404970594CF
:109B40000B9403F077FD2948012103F0A3FD0126C2
:109B50004FF4602328480CA90E930C948DF83460C0
:109B60008DF835600F948DF8407003F00FF822489F
:109B70000E2132462B4603F08BF81F480F2102229C
:109B80002B4603F085F81C480A212A462B4603F091
:109B90007FF82B463A4618480B2103F079F8224605
:109BA00015484FF4FC6103F035F81348314603F0D3
:109BB00027F81148314603F019F80F4803F034F83C
:109BC0000D4803F037F80028FAD10B4803F036F8B7
:109BD000094803F039F80028FAD10748012103F0B9
:109BE00037F813B0F0BD00BF00100140080002407C
:109BF0004C2401409C04002000240140AFF300806D
:109C0000014B03221A607047A4040020044A054B4C
:109C1000927A0AB1052200E001221A60704700BF63
:109C2000F80D0020A4040020704700BF014B002263
:109C30005A607047A404002008B5074B1A6892B216
:109C400042F008021A601A6892B242F004021A60E6
:109C5000FFF7D6FF08BD00BF405C004010B5064CC2
:109C60004FF6FB73226802EA03032360FFF7CEFF7F
:109C70004FF40643236010BD405C0040072818BF26
:109C80001F4B10B51E4C18BF18702378052B33D806
:109C9000DFE803F003060A0E1621FFF7DFFF2BE0D3
:109CA000FFF7DCFF042328E002236370013324E084
:109CB0006378013BDBB263706378FBB9042218E080
:109CC000104B1A6892B242F010021A6005232370FA
:109CD000DB18637012E06378013BDBB2637063787A
:109CE00063B9084A4FF6EF73116801EA0303136082
:109CF0000622034B1A7001E00623237010BD00BF3B
:109D00005C0E0020405C0040034B9B7A13B1034B78
:109D100005221A60704700BFF80D0020A40400203F
:109D2000014B04221A607047A4040020034B1A7AE6
:109D3000202A01D100221A72704700BFA40400201B
:109D4000704700BF212808B508D1124B1B681B784B
:109D500003F07F03212B1AD10F4B0EE0202816D1E0
:109D60000C4B0E4A1B681B7810720D4A03F07F03E0
:109D7000212B0CBF134600234BB1064A4FF00001C4
:109D800012680020518293619847002000E0022071
:109D900008BD00BF580E0020D99D0008A404002073
:109DA000F59D0008074B1B681B7803F07F03212BF0
:109DB00005D1022801D0222801D1002000E0022094
:109DC000704700BF580E002019B9012801D8084675
:109DD00000E00220704700BF28B9044B4FF0080292
:109DE0001B681A8200E00248704700BF580E00202E
:109DF0004800002028B9044B4FF008021B681A8263
:109E000000E00248704700BF580E002048000020C4
:109E10000B4B10B5DA6882B11B68052B01D000220C
:109E20000BE0002303E00749595CC15401330449A6
:109E3000CC68A342F7D30023CB60104610BD00BF0F
:109E4000A4040020600E0020084BDB68082B01D81A
:109E500000200AE00023064A9A5CC2540133092B11
:109E6000F9D1024B0022DA6001207047A4040020DF
:109E7000600E002010B5074C0B468AB2C02163600B
:109E800006F0C2FA0120A18806F0CCFC012006F001
:109E900097FB10BDA404002007B5142200238DF801
:109EA000042001A801228DF806308DF807208DF8D6
:109EB000053004F075F80EBD07B5142200238DF8A7
:109EC000042001A801228DF806308DF807208DF8B6
:109ED000053004F065F80EBD08B5064B1B68DB784D
:109EE000042B01D9002004E0034901EBC30105F074
:109EF00033FE08BD580E00205000002008B502496E
:109F000005F02AFE08BD00BF7000002008B5024918
:109F100005F022FE08BD00BF78000020334B10B5CD
:109F20001B686FF03F0200245A72DC729C7220465C
:109F300006F0BEFA20464FF4007106F0D7FA102161
:109F4000204606F0E9FA4021204606F03FFC802139
:109F5000204606F02BFC204606F068FB244B2046EA
:109F600093F8641006F080FC204606F037FB0120D1
:109F7000214606F0BBFA0120C02106F017FC0120A3
:109F8000202106F0C9FA0120214606F0DDFA022060
:109F90004FF4C06106F0AAFA02204FF4807106F077
:109FA00005FC0220214606F0CFFA0220202106F00F
:109FB000B3FA0320214606F099FA03204FF4887182
:109FC00006F004FC0320402106F04EFC03204FF471
:109FD000405106F0B9FA2146032006F09DFA2046CA
:109FE00005F0C8FD034B01221A6010BD580E002079
:109FF00048000020A404002008B5174B174A196830
:10A0000089B2118016491288098801EA020212F405
:10A01000806F05D04FF6FF321A60124BDB6B98470A
:10A020000E4B1A880E4B1B8803EA020212F4007FC3
:10A0300008D009490C4A4FF6FF500860117C0131E5
:10A04000C9B21174054A1288134013F4004F01D0AD
:10A0500006F016F908BD00BF445C0040EE0D00207C
:10A06000A00E002048000020A404002010B503200A
:10A0700006F02AFC064C034602464FF48871054858
:10A08000E36006F0D9F9032006F0A8FA10BD00BF7E
:10A09000A4040020600E002008B520B1044801216E
:10A0A00003F074FE03E00248012103F071FE08BDD5
:10A0B0000008014038B5064D01232B60054B0024F4
:10A0C00020461C60FFF7E8FF03232B60204638BDC5
:10A0D000405C0040445C004008B5FFF7EBFF08BD62
:10A0E00008B50120FFF7D8FF064B0121196006498A
:10A0F0004FF4E0520A8005490020186008601A6099
:10A1000008BD00BF405C0040A00E0020445C004041
:10A11000084B10B51B6800249C72FFF7E1FF064A4C
:10A120004FF406431460043A1360044A1460044A6E
:10A13000138010BD580E0020445C0040A404002091
:10A14000A00E0020002008B504F038F94FF40000FC
:10A15000012104F0CBF908BD07B5FFF7F3FFFFF7C6
:10A16000ABFE06F02FF80420012104F0B1F903231F
:10A170008DF806300D338DF8073004484FF0010399
:10A1800001A9ADF8043003F09BFD0EBD00080140AD
:10A19000704700BF704700BF704700BF704700BFE7
:10A1A000704700BF704700BF704700BF704700BFD7
:10A1B00008B5FAF77FFA052805D9FAF77BFA40F2D5
:10A1C000F933984201D9012200E00022094B5A607C
:10A1D000094B1B786BB1074B08495A68084B0A605A
:10A1E0001AB91A6842F0080202E01A6822F008025E
:10A1F0001A6008BD600700205A07002048070020A9
:10A20000F006002010B5FFF7BFFB074C2368C31A08
:10A21000B3F5FA7F07D9054BDA6882F00802DA60F5
:10A22000FFF7B2FB206010BDA40E0020001001401B
:10A23000024B03EBC003D879704700BFB80400207D
:10A24000024B03EBC0035879704700BFB8040020ED
:10A25000024B03EBC0039879704700BFB80400209D
:10A26000024B0B2202FB0033187A7047B80400201F
:10A27000024B0B2202FB0033587A7047B8040020CF
:10A28000024B0B2202FB0033D87A7047B80400203F
:10A29000024B0B2202FB0033987A7047B80400206F
:10A2A000024B0B2202FB0033187B7047B8040020DE
:10A2B000024B0B2202FB0033587B7047B80400208E
:10A2C000024B0B2202FB0033987B7047B80400203E
:10A2D000024B0B2202FB0033187C7047B8040020AD
:10A2E000024B0B2202FB0033587C7047B80400205D
:10A2F000024B0B2202FB0033987C7047B80400200D
:10A30000024B052202FB0033187D7047B804002081
:10A31000024B052202FB0033587D7047B804002031
:10A32000024B052202FB0033987D7047B8040020E1
:10A33000024B052202FB0033D87D7047B804002091
:10A34000024B052202FB0033187E7047B804002040
:10A35000024B032202FB0033187F7047B804002031
:10A36000034B032202FB003393F91D00704700BF2B
:10A37000B8040020024B032202FB0033987F704791
:10A38000B8040020024B03EBC00393F82000704791
:10A39000B8040020024B03EBC00393F82100704780
:10A3A000B8040020024B03EBC00393F8220070476F
:10A3B000B8040020024B03EBC00393F8230070475E
:10A3C000B8040020024B03EBC00393F8240070474D
:10A3D000B8040020024B03EBC00393F8250070473C
:10A3E000B8040020024B03EBC00393F8260070472B
:10A3F000B8040020024B03EBC00393F8270070471A
:10A40000B804002006281AD8DFE800F004070A0D77
:10A41000101316000A4B9B6A10E0094BDB6A0DE033
:10A42000074B1B6B0AE0064B5B6B07E0044B9B6B17
:10A4300004E0034BDB6B01E0014BDB7B0B607047FF
:10A44000B804002070B5C0F3074105460022012082
:10A45000FAF75CFC0A4C0602C5F307210022012032
:10A46000A662FAF753FC064301203602E9B202461F
:10A47000A662FAF74BFC06433609A66270BD00BF20
:10A48000B80400202D4B032202FB003310B51C330F
:10A4900093F901203F2A01DD3F225A70274B032206
:10A4A00002FB00331C3393F9012012F13F0FBCBFB4
:10A4B0006FF03E025A70214B032202FB00331C3323
:10A4C0009A781F2A01D91F229A701C4B032202FB83
:10A4D00000324FF440211964127F012A04BF4FF467
:10A4E00050221A64154B03EBC00292F827203AB9A8
:10A4F000033202FB0032527F196C02F07F020BE044
:10A50000032101FB003191F81DC002F003020CF0A1
:10A510007C0C196C4CEA0202084C41EA02221A64D3
:10A52000032303FB0040236C827F42EA03031846A7
:10A530002364FFF787FF236CA36310BDB8040020DA
:10A5400008B5044B032202FB00339977FFF79AFF0B
:10A5500008BD00BFB804002008B5044B032202FB6D
:10A5600000335977FFF78EFF08BD00BFB804002005
:10A5700008B5044B032202FB00331977FFF782FF73
:10A5800008BD00BFB8040020264B052210B502FB11
:10A5900000331A7D012A01D901221A75214B0522A7
:10A5A00002FB003314335A78032A01D903225A706C
:10A5B0001C4B052202FB003314339A780F2A01D971
:10A5C0000F229A70174B052202FB00331433DA78FE
:10A5D000032A01D90322DA70124B052202FB003351
:10A5E00014331A790F2A01D90F221A710D4C052341
:10A5F00003FB004000F114021379017D43F4202392
:10A60000507843EAC133917843EA4033D27843EA41
:10A61000012343EA421318462364FFF713FF236C18
:10A62000636310BDB804002008B5044B052202FB8B
:10A6300000331976FFF7A8FF08BD00BFB80400205B
:10A6400008B5044B052202FB0033D975FFF79CFFC8
:10A6500008BD00BFB804002008B5044B052202FB6A
:10A6600000339975FFF790FF08BD00BFB8040020C4
:10A6700008B5044B052202FB00335975FFF784FF30
:10A6800008BD00BFB804002008B5044B052202FB3A
:10A6900000331975FFF778FF08BD00BFB80400202C
:10A6A000514B0B2210B502FB00331A7A032A01D951
:10A6B00003221A724C4B0B2202FB003308339A78A8
:10A6C000032A01D903229A70474B0B2202FB003365
:10A6D00008331A790F2A01D90F221A71424B0B2223
:10A6E00002FB003308335A79072A01D907225A712D
:10A6F0003D4B0B2202FB003308339A790F2A01D914
:10A700000F229A71384B0B2202FB003310335A7818
:10A710000F2A01D90F225A70334B0B2202FB003350
:10A7200010339A780F2A01D90F229A702E4B0B22E0
:10A7300002FB0032117AC90341F400241C64527AEE
:10A7400012B141F404211964274B0B2101FB0031A4
:10A75000C97A19B1196C41F400511964224B8AB9B4
:10A760000B3202FB0032083292F804C091784FEAB3
:10A77000CC1C1C6C4CEAC12C51794CEA040242EA14
:10A7800001121DE00B2202FB0032127C1AB11A6C7E
:10A7900042F480521A64144B0B2101FB003110313A
:10A7A00091F801E01A6C897842EACE1201F0070CA8
:10A7B00042EA0C1211F0080F1A6402D042F400624F
:10A7C0001A64094B0B2202FB00300830C27922B90F
:10A7D00081791A6C41EA02021A64034C206CFFF77B
:10A7E00031FE236C236310BDB804002008B5064B6E
:10A7F0000B2202FB00330833DA791AB10022DA7136
:10A80000FFF74EFF08BD00BFB804002008B5064B97
:10A810000B2202FB00330833DA791AB90132DA71FC
:10A82000FFF73EFF08BD00BFB804002008B5044B89
:10A830000B2202FB00339974FFF732FF08BD00BF03
:10A84000B804002008B5044B0B2202FB00335974F6
:10A85000FFF726FF08BD00BFB804002008B5044B71
:10A860000B2202FB00331974FFF71AFF08BD00BF6B
:10A87000B804002008B5044B0B2202FB0033997387
:10A88000FFF70EFF08BD00BFB804002008B5044B59
:10A890000B2202FB00335973FFF702FF08BD00BF14
:10A8A000B804002008B5044B0B2202FB00331973D7
:10A8B000FFF7F6FE08BD00BFB804002008B5044B42
:10A8C0000B2202FB00339972FFF7EAFE08BD00BFBE
:10A8D000B804002008B5044B0B2202FB0033D972E8
:10A8E000FFF7DEFE08BD00BFB804002008B5044B2A
:10A8F0000B2202FB00335972FFF7D2FE08BD00BFE6
:10A90000B804002008B5044B0B2202FB0033197277
:10A91000FFF7C6FE08BD00BFB804002010B5254BE8
:10A920004FF460221A6403EBC00292F8272012B1A0
:10A930004FF470221A641F4B03EBC00292F82110EF
:10A9400092F820C01C6C090341EA8C312143196440
:10A9500092F82220012A04BF41F480611964154B4A
:10A9600003EBC00191F823C01A6C42EA0C221A646E
:10A9700091F82410012904BF42F080021A640D4BA3
:10A9800003EBC00292F82520012A03D11A6C42F091
:10A9900040021A64074C04EBC00090F82620236C98
:10A9A00043EA021318462364FFF74CFD236CE3636C
:10A9B00010BD00BFB804002008B5044B03EBC00372
:10A9C00083F82610FFF7AAFF08BD00BFB8040020D7
:10A9D00070B50F4B064603EBC00393F82650032DCA
:10A9E00002D00321FFF7E8FF3046FFF797FF084B3F
:10A9F0009C6A14F4002F1CBF6FEA04346FEA14340D
:10AA0000032D03D030462946FFF7D6FF204670BD00
:10AA1000B804002008B5044B03EBC00383F82510ED
:10AA2000FFF77CFF08BD00BFB804002008B5044B49
:10AA300003EBC00383F82410FFF770FF08BD00BFCD
:10AA4000B804002008B5044B03EBC00383F82310BF
:10AA5000FFF764FF08BD00BFB804002008B5044B31
:10AA600003EBC00383F82210FFF758FF08BD00BFB7
:10AA7000B804002008B5044B03EBC00383F8211091
:10AA8000FFF74CFF08BD00BFB804002008B5044B19
:10AA900003EBC00383F82010FFF740FF08BD00BFA1
:10AAA000B8040020064B10B503EBC003044683F83E
:10AAB0002710FFF733FF2046FFF7E4FC10BD00BF6F
:10AAC000B804002010B5144B00221A6403EBC00236
:10AAD000527912B14FF400721A640F4B03EBC002AB
:10AAE00092791AB11A6C42F480721A640A4B03EB21
:10AAF000C003DA790F2A01D90F22DA71064C04EB70
:10AB0000C000C279236C42EA030318462364FFF7AE
:10AB100099FC236CE36210BDB804002070B5084DA9
:10AB20009DF810E09DF8146005EBC004267162707A
:10AB3000A37084F803E005F83010FFF7C3FF70BD81
:10AB4000B804002008B5034B03EBC0039971FFF76D
:10AB5000B9FF08BDB804002008B5054B03EBC003DE
:10AB6000597109B10422DA71FFF7ACFF08BD00BFCB
:10AB7000B804002008B5054B042903EBC003D971C4
:10AB800001D000225A71FFF79DFF08BDB8040020D4
:10AB90002DE9F047344D0446401990F844000E4624
:10ABA00017469846DDF82090DDF824A004281FD829
:10ABB000DFE800F003090F151B002046FFF770FDCA
:10ABC0006519012316E02046FFF7A8FE6519022348
:10ABD00010E02046FFF7D8FC651903230AE0204661
:10ABE000FFF750FC6519042304E02046FFF76AFFD5
:10ABF0006519002385F844301B4B03EBC40494F81B
:10AC00002620012A0DD002D3022A23D111E016B149
:10AC10009B6A9B0C3370EFB1134B9B6A9B0A3B7092
:10AC200018E0B8F1000F15D09B6A9B0AC8F80030F5
:10AC300010E0B8F1000F04D09B6ADB0B5B01C8F891
:10AC40000030B9F1000F05D0074B9B6AC3F3842392
:10AC500089F80030BAF1000F03D0034B9B6A8AF8E1
:10AC60000030BDE8F08700BFB8040020214B10B5CC
:10AC7000032200244FF0050C02214FF0010E83F84F
:10AC800025E0197383F80EC09A745C7483F81CE095
:10AC900083F81DC083F81EC083F8202083F821208C
:10ACA00083F8224083F8234083F8244083F8261059
:10ACB00083F827401C755C759C75DC751C765C718F
:10ACC0009C71DC7119725C72DC729C725A73DC7359
:10ACD0001C742046FFF758FC2046FFF7D3FB2046A4
:10ACE000FFF71CFE2046FFF7EDFE2046FFF7D8FCDD
:10ACF00010BD00BFB804002008B5044A0023917AB3
:10AD0000034A18461370F9F7BFFE08BD180C00205F
:10AD1000800C00202DE9FF417E4B1A7822B90132C8
:10AD20001A706FF000425A607A4B1C7A5CB9E0B23C
:10AD3000F9F796FC774B03F10C0210550134082CFF
:10AD4000F5D101221A7227240025E8B2F9F788FC10
:10AD5000714A535D834219D0704B291D53F821303D
:10AD60005055022B05D0032B0AD0012B0ED168B110
:10AD700006E058B96A4A115D012907D1135505E06B
:10AD8000674B1A5D012A01D101321A550135013490
:10AD9000082DDAD1634EF36993B1634C25787DB900
:10ADA000FEF7F2FD614AF3691268821A002AB8BF01
:10ADB00052429A4204D9284601F08EFA01232370A8
:10ADC000584E336A93B15A4C25787DB9FEF7DCFDB5
:10ADD000584A336A1268821A002AB8BF52429A420D
:10ADE00004D9284601F078FA01232370494C524DCA
:10ADF000207D830005EBC302127B002A00F0268130
:10AE00004E4A4F4F4F4E0021D3183F1836180A466E
:10AE100000970196FFF7BCFE237D05EB43152A7BC7
:10AE2000013A042A00F20181DFE812F005004E0029
:10AE3000D2004E00D200444A364D926812F4805F30
:10AE40001BD15D192A7E022A04D1404AD25C002A15
:10AE500000F0EB80384A2F4C02EB43121846517A2F
:10AE6000F9F712FE207DFFF7C1FC237D374A002150
:10AE7000E418D15402232376D7E05D192A7E012AF3
:10AE800004D1324AD25C002A00F0CF802A4C184606
:10AE900004EB4313997AF9F7F7FD1E4B187D04EB89
:10AEA0004014A37A13B9FFF7B1FC04E0274B1B5CF5
:10AEB0000BB1FFF79BFC174A2449137D0020D218E1
:10AEC000C85401231376B0E01E4A124DD256002A10
:10AED0003EDB5D192A7E022A02D11C4AD25C8AB16D
:10AEE000154A0C4C02EB43121846517AF9F7CCFD87
:10AEF000207DFFF77BFC237D144A0021E418D15408
:10AF000002232376034C257DFEF73EFD04EB8504EA
:10AF1000606055E0000500200C050020400C00207A
:10AF2000900C0020080000207D0C0020780C0020F0
:10AF3000790B0020700C0020180C0020B00B0020B2
:10AF4000840B0020100C0020001001407C0C00201D
:10AF50005B191B7E012B11D0FEF716FD2B7D8C4A51
:10AF600005EB830502EB43139B8B0A2253436A686C
:10AF7000821A002AB8BF52429A4204DC854B864AA4
:10AF80001B7DD35CE3B1834D814C287D04EB4013E2
:10AF9000997AF9F779FD287D04EB4014A37A13B967
:10AFA000FFF734FC04E07C4B1B5C0BB1FFF71EFC8D
:10AFB000784A7949137D0020D218C85401231376AA
:10AFC000744B1A7D724B03EB42131B7B042B20E066
:10AFD000704A9A18127E022A02D16F4AD25C8AB154
:10AFE0006B4A6C4C02EB43121846517AF9F74CFD50
:10AFF000207DFFF7FBFB237D674A0021E418D15435
:10B0000002232376634B1A7D614B03EB42131B7BB8
:10B01000052B0AD1614B9A6812F4805F0BBF4FF485
:10B0200000524FF400521A615A61FEF7ADFC594CC0
:10B03000E369C31A002BB8BF5B420A2B40F36F834E
:10B04000F9F7AAFBFEF7A0FCE06168E3F9F7A4FBBF
:10B05000FEF79AFCE369C31A002BB8BF5B420A2BC8
:10B0600005DC4F4B9B6813F0040F40F05883494DAB
:10B070000020297D490141F00A0101F0EA0100F0B8
:10B08000EDFF0446287D01F04BF92B7D0C20584341
:10B0900044494218157A0DB1455800E05568424AB6
:10B0A000D25C032A00F2E680DFE802F002821C4B49
:10B0B000002C00F0DF80364A364D02EB4311C97F89
:10B0C000394E29B11846F9F7DFFC2B7D032207E042
:10B0D00002EB43121846517AF9F7D6FC2B7D022277
:10B0E000F254C7E04CB95B0143F0080101F0E801FC
:10B0F000204600F0B3FF002864D0264E244B307D5C
:10B1000003EB4013D97F002900F0AD80002D84EAC5
:10B11000E472B8BF6D42A2EBE472AA4202D0002CE6
:10B1200040F09B80214B53F830108A4280F09B8086
:10B1300003EBC0031979F9F7A7FC164B01211B7D1E
:10B140008FE0002D84EAE471B8BF6D42A1EBE47199
:10B15000A94202D0002C40F08680144A0D4D52F8CE
:10B160003300114E814208D202EBC3021846117916
:10B17000F9F78AFC2B7D012208E0054A184602EB0C
:10B180004313597AF9F780FC2B7D0222F2546AE0CE
:10B19000180C0020000500207C0C0020001001404D
:10B1A00000140140C40B0020800C0020880B0020FC
:10B1B00044BB5B0143F0080101F0E801204600F0C8
:10B1C0004DFFF8B9FEF7E0FB1F4D204A2B7D4FF0F5
:10B1D0000A0E02EB4311B1F81CC099004E197668B3
:10B1E0000EFB0CFC861B002EB8BF7642664541DD87
:10B1F00002EBC1021846917AF9F746FC2B7D144AFE
:10B20000D45437E0104E114A337D02EB4312D17F04
:10B2100049B3002D84EAE472B8BF6D42A2EBE47238
:10B22000AA4200D0C4B90B4951F833108A421AD34C
:10B23000064A184602EB4313597AF9F725FC024BEC
:10B2400002211B7D0DE000BF00050020180C00202E
:10B25000800C0020880B00201846F9F715FC337D80
:10B260000321A34AD154A34D2E7DFEF78DFB05EBA0
:10B27000860568609F4DA04F2B7DA04E1846F6189E
:10B28000FF189F4B002103EB80030A4601960097AD
:10B290009C4EFFF77DFC287D06EB40139B6943B372
:10B2A000F9F7E6F828B3287D84EAE47206EB401348
:10B2B0009B69A2EBE4729A421BD901F00DF82A7D3A
:10B2C000914906EB42139B7F0120885443B1B27F22
:10B2D0009A4205D1013800F0FFFF002000F03AFA51
:10B2E000844B8A4A1B7D0F33D15C012901D1013186
:10B2F000D154804D2B7D022B25D8002000F08AFDF3
:10B3000095F8203010F0010F03F0F80385F8203095
:10B310001CBF43F0010385F8203010F0040F8DF8B6
:10B320000C0006D0734B93F8202042F0020283F801
:10B33000202010F0100F06D06E4B93F8202042F022
:10B34000040283F82020724A137853B1694991F8B6
:10B3500020100B4205D16F496F480978037001B97D
:10B3600011706D4B1B784BB1624A92F8202003EAB2
:10B3700002029A4202D1694B01221A705D4B93F886
:10B38000202012F0010F0AD093F8213013F0010FA2
:10B3900005D15E4BDA78012A01D10132DA70554BC2
:10B3A00093F8202012F0020F0AD093F8213013F006
:10B3B000020F05D1554B1A79012A01D101321A71B8
:10B3C0004C4B93F8202012F0040F0AD093F8213050
:10B3D00013F0040F05D14D4B5A79012A01D10132E6
:10B3E0005A71444D03222B7D04A8B3FBF2F282185C
:10B3F00012F9042C95F82010002A85F821104ADA59
:10B400005B0143F01601002001F0F60102AA00F0F2
:10B410003DFE9DF80A3013F0400F08D02A7D3B49CD
:10B4200052001B32885C012801D10130885413F08E
:10B43000800F0AD02F49354A097D0E3112F81100CC
:10B44000012802D1013002F8110013F0100F09D0C9
:10B45000284A2E49127D52001B32885C012801D1F6
:10B460000130885413F0200F0AD0224A274B127D56
:10B470000E3213F81210012902D1013103F8121013
:10B480001C4B0020197D02AA490141F0160101F070
:10B49000F60100F097FF174F1A4E3B7D06EB431263
:10B4A0005269002A00F081801D4AD55C002D7CD1B4
:10B4B000002C7AD05B0143F0020101F0E201284642
:10B4C00000F092FD8046387DF9F75EFA397DC0EBD9
:10B4D000080806EB41135B69B8F1000F83EAE372D9
:10B4E000B8BFC8F10008A2EBE37290455DDD19E03A
:10B4F000800C002000050020840B0020100C002090
:10B50000B00B0020180C00200C0C0020900C002028
:10B51000AC0B0020800B00209C0B0020C40C0020F2
:10B52000940B0020002B0EDD084600F0D5FE3B7D7D
:10B5300006EB43139B7F3BB3B27F9A4224D128464C
:10B5400000F0CAFE1DE02846022200F027FD397DEA
:10B550002846490141F0080101F0E80100F09EFE93
:10B560003B7D06EB43139B7F73B1B27F9A420BD1B5
:10B5700029462846022200F011FD2846082100F045
:10B580008DFE284600F0E6F8664B674A1B7D1533B2
:10B59000D15C012901D10131D154624B634A1B7D39
:10B5A00001211846D15400F0D5F8614F3B68002BBB
:10B5B00047D05C4E5D4A337DD55C002D41D1002CD7
:10B5C00040D05B0143F0020101F0E201284600F0A7
:10B5D0000BFD8046307DF8F78BFF3B68C0EB080819
:10B5E000B8F1000F83EAE372B8BFC8F10008A2EB1C
:10B5F000E372904531DD002B317D03DD084600F01C
:10B600006BFE0CE02846022200F0C8FC317D284683
:10B61000490141F0080101F0E80100F03FFE414B13
:10B62000414A1B7D1533D15C012901D10131D1542F
:10B630003C4B3E4A1B7D01211846D15400F08AF84C
:10B640000BE054B9374B0020197D490141F0080146
:10B6500001F0E80100F002FD20B1324D354B2E7DA6
:10B660009B5D43B32F4B344A1B7D02EB4312D289BF
:10B6700012B9304AD35C1BB3FEF786F9294D2E4927
:10B680002B7D4FF00A0C9A0001EBC201C9895219B7
:10B69000526A0CFB01F1821A002AB8BF52428A4258
:10B6A0000EDD264EF25C5AB91846FFF7AFF82B7D37
:10B6B0000122F25404E0FEF767F905EB86056862A3
:10B6C000184E1F4D307D002C55F83030B8BF644205
:10B6D0009C420AD2FEF734FE337D05EBC3056A793E
:10B6E00082420DD11846002108E0FEF729FE337D85
:10B6F00005EBC3056979884202D01846FEF794FF2E
:10B70000084C207D00F034F8237D0133DBB2237533
:10B710000BB100232375FEF737F9024BD861BDE862
:10B72000FF8100BF00050020900C0020940B00203A
:10B73000A40B0020880C0020180C00208C0C00208A
:10B74000880B0020024B1A5C0AB901321A54704768
:10B7500028050020024B1A5C0AB10F221A547047C8
:10B7600028050020014B185C704700BF2805002009
:10B770002DE9F3474601F5B2044645F07C0100206F
:10B7800001AA00F083FCB74A610002EB4413187A67
:10B7900006EB020710F0400F9DF8063012D04FF074
:10B7A00001084FF0020C08FA01F80CFA01FCB1583C
:10B7B0007E680CEA030208EA0307C1F10009C6F13A
:10B7C000000A0FE04FF0010C4FF002080CFA01FCE8
:10B7D00008FA01F156F80290D7F804A00CEA030227
:10B7E00001EA030710F0800F00F03F0606D09E4BE1
:10B7F0009B6883F40048C8F3C03803E09A4B9B6809
:10B80000C3F3C038731E072B00F2D182DFE813F0B8
:10B8100008000800080008006E016E016E016E014C
:10B82000924B1B5D013B0E2B00F2C182DFE813F04F
:10B830000F003D00530062007A0082008E00A000DD
:10B84000D10014012401BF0243014E01A60201AA46
:10B8500045F014010020854F00F018FC9DF80530DC
:10B8600045F0060507EB8408C8F804302946002097
:10B8700000F0F4FB0222C8F808002146002000F086
:10B880008DFB023E0020294640F2FF7200F0F2FCE0
:10B89000F6B200200322214600F05AFB012E01D807
:10B8A000022300E004233B5581E2704E002006EBAA
:10B8B00084035A68214602F00402824214BF052222
:10B8C000012200F045FB45F008014A46002000F047
:10B8D000D1FC032324E0002A00F0698245F0020134
:10B8E000002000F081FB614B04221A55604B43F8A5
:10B8F00024005CE25D4E002006EB84035A6821467A
:10B9000002F00402824214BF0622022200F020FB51
:10B9100045F00801C9F10002002000F0ABFC05234E
:10B92000335544E2002F00F04282204600F0D4FC60
:10B9300006222FE200202146032200F009FB45F0F9
:10B9400008015246002000F095FC68E1002F40F00D
:10B950002E8245F008053A463846294600F08AFC12
:10B96000CAF100023846294600F084FC082211E2A0
:10B97000002F00F01C8245F00201002000F034FB93
:10B9800006460020024645F0080100F073FC384BE3
:10B99000002053F824702146BF1B43F82470032273
:10B9A00000F0D6FA8AEAEA7245F00601A2EBEA72E2
:10B9B000002000F05FFC610101F0E0013246002050
:10B9C00000F0C4FB00200246214600F0E7FA0922FD
:10B9D000E0E1002000F01EFA630050FA03F313F0D8
:10B9E000010F00F0E48145F002073946002000F025
:10B9F000FBFA204B45F0080543F8240000200246DE
:10BA0000294600F037FC00200222214600F0C6FA49
:10BA100000200246394600F099FB002061010246F1
:10BA200001F0E001033E00F091FBF6B20021204658
:10BA3000F8F780FF012E0D4E0CD80020214602227F
:10BA400000F0ACFA2946CAF10002002000F012FC16
:10BA50000A2365E70E2363E7002F00F0A8810B227D
:10BA600098E100BF180C00200008014028050020C4
:10BA70007C0B00203C0C0020002F40F0988145F00A
:10BA80000201384600F0B0FA45F0080106463A4691
:10BA9000384600F0EFFB6101022296FBF2F201F062
:10BAA000E001384600F052FB3A463846214600F0A5
:10BAB00075FA0D226EE1002000F0ACF9630050FA37
:10BAC00003F313F0010F00F0728162E1A84E45F01C
:10BAD000060106EB84050020AA6800F0CBFB2A795A
:10BAE0000020214600F034FA002319E7A04B1B5D2B
:10BAF000013B0E2B00F25B81DFE813F00F003400F6
:10BB00005200620081005901930059015901CC0093
:10BB1000DC00AD0008014F01400145F0140101AA0D
:10BB20000020934F00F0B2FA9DF805C007EB8403A4
:10BB300000200222C3F804C0214600F02FFA0020A2
:10BB400045F0060140F2FF7200F094FB0020032252
:10BB5000214600F0FDF9062E02D0082E7FF4A2AE99
:10BB6000022217E1062E0CD1814B002003EB840347
:10BB70005A68214602F00402824214BF05220122C3
:10BB800004E0082E04D100202146032200F0E0F951
:10BB90004A4645F00801002000F06CFB0322F9E062
:10BBA000731FDBB2012B05D822B1062E704E30D1A7
:10BBB0000423B5E6B8F1000F00F0F9800C22E9E0AB
:10BBC000052E0CD16A4B002003EB84035A682146F2
:10BBD00002F00402824214BF0622022204E0072E71
:10BBE00004D100202146032200F0B2F9C9F100027D
:10BBF00045F00801002000F03DFB0522CAE0731F5C
:10BC0000DBB2012B07D837B1052E594E01D10223E3
:10BC100086E60F2384E6B8F1000F00F0C880072203
:10BC2000B8E0B8F1000F40F0C280073EF6B2012E36
:10BC30000DD94F4B404603EB84035A68214602F06E
:10BC40000402002A14BF0522012200F081F945F008
:10BC50000801524619E0B8F1000F40F0A880073EF5
:10BC6000F6B2012E0DD9424B404603EB84035A68CD
:10BC7000214602F00402002A14BF0622022200F02C
:10BC800067F945F00801CAF10002002000F0F2FA5D
:10BC90000A227FE0B8F1000F00F0898045F0020130
:10BCA000002000F0A1F9324B0B2103EB840219555F
:10BCB000D0607CE0B8F1000F79D145F00201404638
:10BCC00000F092F92B4BA700294E03EBC7038AEA39
:10BCD000EA72814645F00601A2EBEA72404683F81B
:10BCE0000D80BF1900F032FAFB686101994402230C
:10BCF00099FBF3F201F0E001404600F027FA4046DC
:10BD00002146424600F04AF90D2309E6002000F0E2
:10BD100081F8630050FA03F313F0010F47D0144B7E
:10BD20000E2245F002061A553146002000F05CF95B
:10BD3000114B45F0080143F824000020024600F0B2
:10BD400099FA21460020022200F028F9002031460D
:10BD5000024600F0FBF900206101024601F0E0011B
:10BD600000F0F4F920460021F8F7E4FD1FE000BFE1
:10BD700028050020180C00203C0C00200020214643
:10BD8000022200F00BF9002045F00801024600F005
:10BD900071FA0E22074B1A5509E0064D002005EBFB
:10BDA00084031A79214600F0D3F800232B55BDE80F
:10BDB000FC8700BF28050020154B10B503EB0012CF
:10BDC000926891420EDD8A1AC2F18074A2424FEA53
:10BDD000001C03DC63445C6812190EE063445A687B
:10BDE000141B0FE00FDA521AC2F18074A2424FEA1C
:10BDF000001C04DC63445C68A21A5A6003E06344DC
:10BE00005A68A4185C60024B03EB0010816010BDFF
:10BE1000A80E0020012108B502200A46F8F776FF97
:10BE200008BD00BFF8B51378144613F0600F06463E
:10BE30000D4627D1414A127B22BB13F0010F21D1BD
:10BE40005F2B1FD83E4A1278E2B913F09F0301D04E
:10BE5000082B17D13B4F387860B9384BD97F19B1CF
:10BE6000F8F712FE032304E00846597AF8F70CFEAF
:10BE700002233B70344F3B7823B10020FEF7B6FC21
:10BE800000233B70002221780220F8F73FFF287042
:10BE9000002261780220F8F739FF68700022A1784B
:10BEA0000220F8F733FFA87001220220E178F8F7AA
:10BEB0002DFFE870237813F0010F3ED15F2B3CD8A3
:10BEC00003F01E02082A04D0142A2CD0062A34D1EA
:10BED0001BE0242171435B090C2000FB0313A578B0
:10BEE00094F803C0194A4CEA05259D50A37813F035
:10BEF000080F22D02678760900FB0616B3586FEAA1
:10BF000003536FEA1353B35017E0242256435B09DF
:10BF10000C22A17802FB0363E27842EA01220B497A
:10BF20005B185A6009E0242256435B090C2202FB8D
:10BF300003630649E2785B181A72F8BD180C0020FA
:10BF4000880C0020800C00208C0C0020C40B0020EA
:10BF50002DE9F3414901CEB201AC46F01503174675
:10BF6000694622468DF804308046FFF75BFF9DF856
:10BF700001C09DF8033046F014064046694622464B
:10BF80006D468DF804608DF805C08DF806708DF84B
:10BF90000730FFF747FFBDE8FC8100BF2DE9F34103
:10BFA0004901CEB201AC46F0150317466946224658
:10BFB0008DF804308046FFF735FF9DF801C09DF8ED
:10BFC000023046F014064046694622466D468DF81A
:10BFD00004608DF805C08DF806308DF80770FFF706
:10BFE00021FFBDE8FC8100BF37B541F001030C46DD
:10BFF0006A4601A98DF800300546FFF713FF9DF84A
:10C0000006009DF8052000029DF8073040EA024036
:10C01000184310F4000F18BF40F07F405F2C1AD86F
:10C02000C4F3411314F01E0402D0022C13D106E015
:10C03000032202FB0535084A2D01A8580BE0032214
:10C0400002FB053520F07F41E8B2FFF7B5FE024B59
:10C0500003EB051568683EBDA80E002007B541F04A
:10C0600001036A4601A98DF80030FFF7DBFE9DF859
:10C0700006009DF8073043EA002010F4006F1CBF53
:10C080006FEA00506FEA10500EBD00BF13B541F0CB
:10C090000103144601A96A468DF80030FFF7C2FE7D
:10C0A0009DF805109DF806309DF807202170A270BC
:10C0B00063709DF804001CBD07B5410141F01601F5
:10C0C00001F0F601002001AAFFF7E0FF9DF805301E
:10C0D000D80913F0200F18BF40F002000EBD00BFBA
:10C0E00007B5410141F0160101F0F601002001AA57
:10C0F000FFF7CCFF9DF80530C3F3801013F0100F4D
:10C1000018BF40F002000EBD37B50C4641EA4011A1
:10C1100001AA0546C9B20020FFF7B8FFB4235D436A
:10C120006408032305F5807503FB04549DF804108F
:10C130002046FCF791FB601C9DF80510FCF78CFB7A
:10C14000A01C9DF80610FCF787FB3EBD5F292DE97A
:10C15000F3410D460646144662D8C1F3411811F06A
:10C160001E0102D002295BD11EE0032202FB0088DF
:10C17000344A4FEA081083185B688450E01A00289C
:10C18000B8BF4042B0F5000F0ADB9C42CCBF2E4C3A
:10C190002E4C2C4A1C1902EB0812012313733FE0AA
:10C1A00002EB081211733BE0032707FB0087254BC6
:10C1B0003801C1587A00C4EB010C0132BCF1000F08
:10C1C000B8BFCCF1000C00EB030EBCF5000F24F05F
:10C1D0007F40CEF8044043F832001DDBA142CCBFC3
:10C1E000194B1A4B4FEA4818E3184FEA234E4FEA0F
:10C1F000232C3046694601AA8DF807308DF804805B
:10C200008DF805E08DF806C0FFF70CFE0D4B03EB33
:10C21000071701233B7303E003EBC20300221A71EB
:10C220004FEA244C23123046694601AA8DF8045087
:10C230008DF805C08DF806308DF80740FFF7F2FD48
:10C24000BDE8FC81A80E0020FFFF7F00010080FFF9
:10C2500038B50D4668210446FFF7C6FE15B140F01B
:10C26000010201E020F0010220466821FFF76EFF85
:10C2700038BD00BF07B513464FEA222C8DF80410D5
:10C280004FF0000E694601AA8DF805E08DF806C052
:10C290008DF80730FFF7C6FD0EBD00BF07B50B4692
:10C2A00011F01E01024601D0022905D1104619469F
:10C2B0000022FFF74BFF0DE04FF0000C694601AA8A
:10C2C0008DF804308DF807C08DF805C08DF806C0D4
:10C2D000FFF7A8FD0EBD00BF10B5C4B22146640132
:10C2E00000200222E4B2FFF759FE002044F00801CA
:10C2F000FFF7D4FF44F00A010020FFF7CFFF10BD85
:10C3000007B59DF810C08DF804108DF8052069461A
:10C3100001AA8DF806308DF807C0FFF783FD0EBD2A
:10C3200030B5430185B0044643F00303002003A960
:10C3300002AA8DF80830FFF775FD9DF80E109DF8E4
:10C340000D209DF80F30090241EA024119432046B1
:10C35000FFF732FD174B03EB041108310A7932B3B2
:10C36000154A0C2000FB0422107A00BB2201D518CC
:10C37000D2586B68C3EB020CBCF1000FB8BFCCF114
:10C38000000CBCF5000F05DB9A42CCBF0B4A0C4AEF
:10C390009A1800E008716101C2F30723D4B201F0DA
:10C3A000E0010020C2F307420094FFF7A9FF05B0A7
:10C3B00030BD00BFA80E0020C40B0020FFFF7F008F
:10C3C000010080FF07B5937892F800E092F801C071
:10C3D0008DF8041001AA69468DF805E08DF806C0B5
:10C3E0008DF80730FFF71EFD0EBD00BF37B54401C5
:10C3F00044F01604E4B20D4601AA21460020FFF7DE
:10C4000045FE9DF8053015F0010F1ABF6FEA436332
:10C410006FEA536303F07F038DF805309DF8053014
:10C4200015F0020F14BF43F0200323F020038DF812
:10C43000053000231846214601AA8DF80630FFF783
:10C44000C1FF3EBD37B5440144F01604E4B20D46C9
:10C4500001AA21460020FFF719FE9DF8053015F0CE
:10C46000010F14BF43F0400323F040038DF8053063
:10C470009DF8053015F0020F14BF43F0100323F0B0
:10C4800010038DF8053000231846214601AA8DF8C7
:10C490000630FFF797FF3EBD73B5B42545434B0803
:10C4A000032205F5807502FB0355044628460E4617
:10C4B000FCF73CF98DF80400681CFCF737F98DF89F
:10C4C0000500A81CFCF732F946EA44148DF8060072
:10C4D000E1B2002001AAFFF775FF7CBD2DE9F74FFF
:10C4E0004001C7B24C05002047F0180101AAFFF730
:10C4F000CDFD9DF80560640D06F00F053609B542C7
:10C500000EDB204605F090F9AD1B80460120A840C7
:10C51000894605F099F90022334B05F0FBF90FE04D
:10C52000204605F081F9751B80460120A840894608
:10C5300005F08AF902460B4600202B4905F014FB52
:10C5400002460B464046494605F00EFB05F0A4FCAA
:10C5500005F08CF922A3D3E9002305F0DBF905F0FF
:10C560009BFC05F083F90022204B05F0D3F94FF036
:10C57000FF36B046002582468B460120A84005F0D4
:10C5800063F902460B465046594605F0C3F905F0DB
:10C590005BFCA0F180027F2A98BF2E46034605F17E
:10C5A000010588BF43460E2D01D09846E5E70025DA
:10C5B00047F0120101AA28468DF805308DF8066073
:10C5C0008DF80450FFF7FEFE284647F00C01224686
:10C5D000FFF750FE2846BDE8FE8F00BFAFF3008096
:10C5E00004560E2DB29DEF3F000060400000204039
:10C5F00013B5154B587E10F0010003D000206821C0
:10C60000212201E0682120220024FFF79FFD20461F
:10C610007E21202223460094FFF772FEE1B2002023
:10C620000134FFF739FF1D2CF8D10C210020FFF752
:10C63000DBFC01460020FFF751FF0020162143F2EA
:10C64000FF12FFF717FE1CBD08000020AFF30080AB
:10C65000084B1868034605E02C2A02D100221A7004
:10C6600003E001331A78002AF6D1024A013313603D
:10C67000704700BF3805002010B50E4B02461B78EE
:10C68000ABB10D4B1C7994B19C68601CE4180D2A69
:10C690002273986002D03F2800D851B9064C014659
:10C6A00004F10C00FDF7E6FB0023A36001E0FCF7BA
:10C6B00017FB10BD780B00203805002030B5012194
:10C6C000044687B02020FFF7D7FF002C04DA2D2086
:10C6D0000121FFF7D1FF644200230A2194FBF1F20C
:10C6E00001FB124101AD3031E954591C141E01DD2A
:10C6F0000B46F2E7ED181C460121013C15F8010933
:10C70000FFF7BAFFB4F1FF3FF6D107B030BD00BF6D
:10C7100038B50C4D0446A87801214030C0B2FFF76F
:10C72000ABFF687801214030C0B2FFF7A5FF207849
:10C73000FFF7C4FF6068FFF7C1FF0D200121FFF77D
:10C740009BFF38BD0800002070B5124B06461B78D1
:10C75000EBB1FCF743FA104C054618B100232371E6
:10C76000012016E0E36C226D934208D21A1992F868
:10C770005420013301203270E364207109E004F198
:10C780005400FDF745FBE5642065284601E0FCF711
:10C7900025FA70BD780B0020380500202DE9F34103
:10C7A00004460DF10700FFF7CFFF002800F0CB8013
:10C7B0008B4B8C4A93F8941019BB51789DF8070065
:10C7C000403188420DD1D3F89810002940F0BB8049
:10C7D0001179012231F0010183F8942040F0B380F7
:10C7E000AFE00D2801D01B2802D100227C4B05E0D0
:10C7F000D3F898207E2A00F2A6800132C3F8982050
:10C80000A1E0117931F0010103D19DF80700FFF794
:10C8100033FF9DF807301F2B0BD9714AD2F89810BF
:10C820007E297FD8481C891881F89C30C2F898006E
:10C8300078E0082B08D16A4BD3F89820002A71D0F1
:10C84000013AC3F898206DE00D2B6BD1644BD3F8FF
:10C850009830002B66D0634B1A79112A15D158787D
:10C8600001214030C0B2FFF707FF002503E0585D0B
:10C87000FFF702FF01355A4B0121D3F898209C3372
:10C880009542F4D30D20FFF7F7FE554A00231568B3
:10C89000D2F8987019461A4633E001290FD002D316
:10C8A00002292DD122E04E4E06F19C00805C20280A
:10C8B00026D09E1986F81C010133012120E048484A
:10C8C00000F19C0C1CF802C0BCF1200F0AD1012B16
:10C8D00004D91818002180F81C110133424D02219F
:10C8E000ED180DE0181880F81CC108E03C4E06F168
:10C8F0009C00805C202803D09E1986F81C0101331F
:10C900000132BA42C9D3364A0021981880F81C1166
:10C910000120C2F89810156082F8A001C2F89C317D
:10C9200082F894109DF807301B2B0CD12D4A2C4B0C
:10C9300012790021012A83F89410C3F8981002D1CB
:10C940000D20FFF799FE264B93F8A001002878D020
:10C950000022164683F8A0211546DFF8A880072795
:10C9600007FB058720483946013504F03BF930B90B
:10C97000BE797B7916F0010F237049D007E018F8D3
:10C9800006300736002B5ED0FF2DE6D15BE0FFF7C7
:10C990005FFE23780546042B0CD1144904F022F9DC
:10C9A0000346D8B12846124904F01CF970B1284654
:10C9B00010490FE00D2B28D10F4904F013F903465D
:10C9C00060B128460D4904F00DF908B9012305E0CE
:10C9D0000B49284604F006F9B0B90223637017E04A
:10C9E000380500200800002054060020212F0108EF
:10C9F000252F0108292F01082F2F0108352F0108A5
:10CA00003A2F0108182D0108284604F0E5F8607057
:10CA100016F0020F04D0FFF71BFE04F0DDF8A07043
:10CA200016F0040F0CD0FFF713FE04F0D5F8010E3A
:10CA3000C0F30722C0F30743A17122716371E07054
:10CA40000120BDE8FC8100232370F9E7704700BF97
:10CA5000FEE700BFFEE700BFFEE700BFFEE700BF46
:10CA6000704700BF704700BF704700BF704700BFEE
:10CA7000704700BF704700BF704700BF704700BFDE
:10CA8000704700BF704700BF704700BF704700BFCE
:10CA9000704700BF704700BF704700BF704700BFBE
:10CAA000704700BF704700BF704700BF704700BFAE
:10CAB000704700BF704700BF08B5024B1B6898471E
:10CAC00008BD00BFA00B002008B5024B1B689847AB
:10CAD00008BD00BF840C002008B5024B1B689847B6
:10CAE00008BD00BF140C002008B5024B1B68984716
:10CAF00008BD00BF380C0020704700BF704700BF62
:10CB0000704700BF704700BF704700BF704700BF4D
:10CB1000704700BF704700BF704700BF704700BF3D
:10CB2000704700BF704700BF704700BF704700BF2D
:10CB3000704700BF704700BF704700BF704700BF1D
:10CB4000704700BF704700BF704700BF704700BF0D
:10CB5000704700BF704700BF704700BF704700BFFD
:10CB6000704700BF704700BF704700BF704700BFED
:10CB7000704700BF704700BF704700BF704700BFDD
:10CB8000704700BF704700BF704700BF436830B5B3
:10CB900023F470230C680A7923F48073234343EA57
:10CBA0000223436082688D68CC680A4B45EA040C16
:10CBB00002EA03034A794CEA030343EA420383602F
:10CBC0000B7CC26A013B22F47002DBB242EA0353DF
:10CBD000C36230BDFDF7F1FF002301220274C36080
:10CBE0000360037143718360704700BF19B18368AC
:10CBF00043F0010302E0836823F001038360704780
:10CC000019B1836843F4807302E0836823F480736E
:10CC100083607047C9B212B14368194302E04368A8
:10CC200023EA010141607047836843F00803836091
:10CC3000704700BF8068C0F3C0007047836843F04E
:10CC400004038360704700BF8068C0F380007047B2
:10CC500019B1836843F4A00302E0836823F4A003BE
:10CC6000836070478068C0F3805070474368013923
:10CC700023F4604343EA41334360704719B143688A
:10CC800043F4006302E0436823F4006343607047A9
:10CC9000092930B511D94FF0030C0CFB01FC072515
:10CCA000ACF11E0C05FA0CF503FA0CFCC46824EA7E
:10CCB000050343EA0C03C3600EE04FF0030C0CFBCA
:10CCC00001FC072505FA0CF503FA0CFC046924EABB
:10CCD000050343EA0C030361062A0DD80523013A34
:10CCE0005A434FF01F0C0CFA02FC9140436B23EAAD
:10CCF0000C020A4342631CE00C2A0DD805235A4358
:10CD00004FF01F0C233A0CFA02FC9140036B23EA0C
:10CD10000C020A4302630CE005235A434FF01F0C38
:10CD2000413A0CFA02FC9140C36A23EA0C020A431E
:10CD3000C26230BD19B1836843F4801302E0836896
:10CD400023F4801383607047C06C80B2704700BFCB
:10CD5000014B1868704700BF4C24014019B143686B
:10CD600043F4806302E0436823F4806343607047C8
:10CD700019B1436843F4805302E0436823F48053BD
:10CD800043607047836823F4E04341EA0303836010
:10CD9000704700BF19B1836843F4004302E0836821
:10CDA00023F400438360704719B1836843F402138E
:10CDB00002E0836823F40213836070478068C0F345
:10CDC00040507047092930B511D94FF0030C0CFBC6
:10CDD00001FC0725ACF11E0C05FA0CF503FA0CFC5E
:10CDE000C46824EA050343EA0C03C3600EE04FF075
:10CDF000030C0CFB01FC072505FA0CF503FA0CFCEF
:10CE0000046924EA050343EA0C030361836BC3F35B
:10CE1000015CCCEB020202324FF0050CD2B20CFBEB
:10CE200002F20CF11A0C0CFA02FC914023EA0C03FA
:10CE30000B43836330BD00BF836B013923F4401380
:10CE400043EA0153836370470A50704728304058C3
:10CE500080B27047436823F4400323F4007341EA2F
:10CE600003034360704700BF41628262704700BFA6
:10CE7000436823F01F0341EA03034360704700BF88
:10CE800020B1054B9A6842F4000203E0024B9A6815
:10CE900022F400029A60704700240140036819429E
:10CEA0000CBF002001207047C9430160704700BFDC
:10CEB0004368006810EA112004D0C9B219420CBFBF
:10CEC00000200120704700BF6FEA11210160704708
:10CED00008B5134B98420FD003F5A053984213D0D6
:10CEE000A3F5C053984219D14FF40070012101F00D
:10CEF0000BFB4FF400700EE04FF48060012101F055
:10CF000003FB4FF4806006E04FF40040012101F084
:10CF1000FBFA4FF40040002101F0F6FA08BD00BF13
:10CF200000280140374B01221A605A6812F00102B2
:10CF300001D1104664E00278012A0BBF1A681A6812
:10CF400042F0800222F080021A604378012B04D163
:10CF50002C4B1A6842F0400203E02A4B1A6822F078
:10CF600040021A608378012B04D1264B1A6842F0E4
:10CF7000200203E0234B1A6822F020021A60C378D3
:10CF8000012B04D11F4B1A6842F0100203E01D4B25
:10CF90001A6822F010021A600379012B04D1194B90
:10CFA0001A6842F0080203E0164B1A6822F00802E1
:10CFB0001A604379012B04D1124B1A6842F0040223
:10CFC00003E0104B1A6822F004021A608279C379D8
:10CFD00090F808C0920742EA03624189437A42EA24
:10CFE0000C4242EA03520139064B0A43DA611A68DD
:10CFF00022F001021A60586880F0010000F0010080
:10D00000704700BF0064004090F800C0012202FA9F
:10D010000CF23B4B2DE9F045D3F8004292B244F0BC
:10D020000104C3F80042D3F81C42D14301EA0404CE
:10D03000C3F81C428478A4B90CF1480CD3F80C72E4
:10D04000B0F80AA0C688B0F8088085884FEACC04FA
:10D0500004F1804446EA0A4645EA084501EA070722
:10D0600015E0012C1AD10CF1480CD3F80C72B0F871
:10D0700004A0C688B0F8088045894FEACC0404F1C2
:10D08000804446EA0A4645EA084542EA070704F5AD
:10D09000C844C3F80C7243F83C60656043782BB910
:10D0A000174BD3F8044201EA040404E0144BD3F80C
:10D0B000044242EA0404C3F80442838923B9104BB2
:10D0C000D3F81442214006E0012B06D10C4BD3F8D3
:10D0D000141242EA0101C3F81412837B012B05D11B
:10D0E000074BD3F81C120A43C3F81C22044BD3F895
:10D0F000002222F00102C3F80022BDE8F08500BF43
:10D100000064004003220272013A002342724FF091
:10D110000102C3714281037043708370C370037155
:10D1200043718371704700BF19B1054B5A691043B1
:10D1300003E0034B5A6922EA00005861704700BFC0
:10D1400000640040364B70B59968024611F0806F5C
:10D1500001D000200CE0996811F0006F01D001208F
:10D1600006E09B6813F0805F01D1042056E00220A6
:10D170002B4B00F118010901CC5804F00104CC50EC
:10D18000157A92F809C035B9146864051460CD5851
:10D190004CEA050C07E0546845EA0C0CE4005460C6
:10D1A000CE584CEA060C4CEA0404CC50947A00F1B8
:10D1B000180C4FEA0C1C04F00F040CF1804394721D
:10D1C00003F5C8435D68010125F00F055D605D68EA
:10D1D00001F180412C435C60537B947BD57A1B0426
:10D1E00043EA0463147B2B4343EA042301F5C8415B
:10D1F000C1F88831557C937CD47B2D0445EA0365C6
:10D20000137C45EA040242EA0322054BC1F88C2153
:10D210005CF8032042F001024CF8032070BD00BF0F
:10D2200000640040012810D002D302282CD11AE05B
:10D23000164A91689368926801F0010103F00203B5
:10D2400043EA8103C2F380621AE0104A936891684E
:10D2500003F48073926801F400719B0943EA11237F
:10D26000C2F3C0620CE0094A9368916803F480330A
:10D27000926801F400319B0B43EA1143C2F3007240
:10D280001343034AD05C70470023FAE70064004070
:10D29000F82D0108012808D002D302280FD109E097
:10D2A000074B9A6842F0800208E0054B9A6842F406
:10D2B000004203E0024B9A6842F400029A60704711
:10D2C0000064004018B9044B2022DA6002E0024BEF
:10D2D00020221A61704700BF0064004010B9064B5D
:10D2E000D86805E0012801D0002003E0024B18694E
:10D2F00000F00300704700BF00640040254B00F1C0
:10D300001B02120110B5D45804F004040C721CB9AD
:10D31000D3585B0D0B6002E0D358DB084B6000F183
:10D320001B021C4B1201D35802F1804203F002038E
:10D330004B7202F5C8425468030104F00F0C81F8E7
:10D340000AC0526803F18043120ACA7403F5C84345
:10D35000D3F8B821CA72D3F8B821120A0A73D3F8E5
:10D36000B821120C4A73D3F8B821120E8A73D3F87D
:10D37000BC21CA73D3F8BC21120A0A74D3F8BC21A9
:10D38000120C4A74D3F8BC311B0E8B74FFF79AFF52
:10D3900010BD00BF00640040044B1A6842F0020256
:10D3A0001A601868C0F34000704700BF0064004076
:10D3B000054B1A6822F002021A60186880F0020019
:10D3C000C0F34000704700BF00640040034B9B69FE
:10D3D00018420CBF00200120704700BF00640040CD
:10D3E000024B9A6922EA00029A6170470064004089
:10D3F000202831D00CD8062820D004D8042825D0E5
:10D40000052844D118E007281DD008283FD11FE087
:10D41000B0F5007F2BD005D840281FD0B0F5807F15
:10D4200035D11FE0B0F5803F2CD0B0F5003F2BD0B8
:10D43000B0F5806F2BD11FE0012201E04FF4807224
:10D44000134B9A6023E04FF48032F9E7082200E0A2
:10D4500010220F4BDA601AE0082200E010220C4B79
:10D460001A6114E00A4B9A6922F0010208E0084BA5
:10D470009A6922F0020203E0054B9A6922F0040245
:10D480009A6104E0082200E01022014B5A607047C4
:10D490000064004001420CBF00200120704700BF23
:10D4A000202808B532D00CD8062821D004D804286A
:10D4B00026D0052818D119E007281ED0082813D136
:10D4C00020E0B0F5007F29D005D8402820D0B0F565
:10D4D000807F09D120E0B0F5803F27D0B0F5003F34
:10D4E00022D0B0F5806F1BD0002024E0012101E0A4
:10D4F0004FF48071104B98681BE04FF48031F9E7CE
:10D50000082100E010210C4BD86812E0082100E04F
:10D510001021094B18690CE0012102E0022100E012
:10D520000421054B986904E0102100E00821024B1A
:10D530005868FFF7AFFF08BD00640040012108B53F
:10D540004FF0007000F0EEFF4FF00070002100F08F
:10D55000E9FF08BD0268002322F0010202600360B7
:10D5600043608360C3602D4B984233D011D83C3B5D
:10D57000984229D006D8283B984221D014339842AB
:10D580004BD11FE0264B984220D01433984244D10F
:10D590001EE0244B98422CD008D8A3F5677398421C
:10D5A0001DD003F56273984237D11DE01E4B98429F
:10D5B00029D0143398422BD0283B98422DD11DE01E
:10D5C0001A4B12E0194B15E0184B18E0174B1BE0F3
:10D5D000164B1EE0154B5A6842F470021CE0134BC8
:10D5E0005A6842F0706217E0114B5A6842F00F021D
:10D5F00012E00F4B5A6842F0F0020DE00C4B5A68F3
:10D6000042F4706208E00A4B5A6842F4704203E048
:10D61000074B5A6842F470225A6070476C0002400F
:10D62000440002401C040240440402400000024046
:10D63000000402408A6870B50C6A0B6944EA020271
:10D640004C691A438B692243CC6905684E6A42EAE9
:10D65000030323438C6A334325F4FE4C23432CF00D
:10D66000F00C43EA0C030360CB6843600B688360F3
:10D670004B68C36070BD00BF0023836203604360DA
:10D680008360C360036143618361C361036243627A
:10D69000704700BF19B1036843F0010302E003685B
:10D6A00023F001030360704712B10368194302E0DD
:10D6B000036823EA01010160704700BF406880B23F
:10D6C000704700BF10F0805F14BF044B044B1B6811
:10D6D00003420CBF00200120704700BF000402403D
:10D6E0000000024010F0805F14BF024B024B5860F4
:10D6F000704700BF000402400000024010F0805F4D
:10D7000014BF044B044B1B6803420CBF00200120D4
:10D71000704700BF000402400000024010F0805F2C
:10D7200014BF024B024B5860704700BF0004024018
:10D7300000000240044B00221A605A609A60DA60CE
:10D74000024A5A61704700BF00040140FFFF070012
:10D75000837930B5016802794BB3184BCC431D680F
:10D7600090F805C004EA05051D605D682C405C600A
:10D77000D45844EA0101D15002689868D14301EAC3
:10D7800000009860D8680140BCF1100FD96007D143
:10D79000996811439960D96841EA0202DA600BE0A6
:10D7A0005CF8031041EA02024CF8032004E0034B4A
:10D7B000D05820EA0101D15030BD00BF0004014023
:10D7C00000230C228371427103600371704700BF14
:10D7D000024B1A6940EA02021A61704700040140D4
:10D7E000034B5B6918420CBF00200120704700BF4B
:10D7F00000040140014B5861704700BF0004014024
:10D80000054B1A685B69034001D1184603E01042DA
:10D810000CBF00200120704700040140014B5861FB
:10D82000704700BF00040140044B1A6802F0380240
:10D830001A601A6840EA02021A607047002002402B
:10D84000044B1A6822F008021A601A6840EA0202C1
:10D850001A60704700200240044B1A6822F0100240
:10D860001A601A6840EA02021A60704700200240FB
:10D87000034B044A5A6002F188325A60704700BF75
:10D880000020024023016745024B1A6942F08002E2
:10D890001A61704700200240014BD8698008704728
:10D8A00000200240014B186A704700BF0020024070
:10D8B000024BD869C0F34000704700BF002002400F
:10D8C000024B1868C0F34010704700BF00200240B0
:10D8D00019B1054B1A69104303E0034B1A6922EA98
:10D8E00000001861704700BF00200240012804D1E9
:10D8F000054BD86900F0010005E0034BDB681842D6
:10D900000CBF00200120704700200240014BD8606E
:10D91000704700BF00200240094BDA6812F0010F87
:10D9200001D001200BE0DA6812F0040F01D00220D0
:10D9300005E0DB6813F0100F14BF032004207047CC
:10D940000020024013B504460AE000230193FF3390
:10D9500001E0019B013B0193019B002BF9D1013CAC
:10D96000FFF7DAFF012802D1002CEED100E004B964
:10D9700005201CBDF8B5124C124B0546A36003F1FF
:10D9800088330F20A3600E461746FFF7DBFF0428FD
:10D9900014D1236945F0F80543F0100323612E43A9
:10D9A000094B37430B305F80FFF7CCFF012805D0D0
:10D9B000226941F6EF7302EA03032361F8BD00BF59
:10D9C000002002402301674500F8FF1F38B50546D7
:10D9D00040F6FF70FFF7B6FF04283CD11E4C1F4BEA
:10D9E00040F6FF70A36003F18833A360236943F01E
:10D9F00020032361236943F040032361FFF7A2FF63
:10DA0000042820D1226941F6DF7302EA030323616F
:10DA1000236943F0100323611DB1114B4FF0000245
:10DA200002E00F4B4FF0A5021A8040F6FF70FFF79F
:10DA300089FF01280FD0084A41F6EF73116901EA06
:10DA40000303136107E0012805D0226941F6DF7363
:10DA500002EA0303236138BD002002402301674529
:10DA600000F8FF1F10B504460F20FFF76BFF0428D6
:10DA70003DD11F4A1F4BE443936003F18833936009
:10DA80001169E3B241F01001FF2B116106D01A4A6F
:10DA90000B301381FFF756FF04281FD1C4F307236F
:10DAA000FF2B06D0144A0F205381FFF74BFF0428A9
:10DAB00014D1C4F30743FF2B06D00F4A0F209381E4
:10DAC000FFF740FF042809D1240EFF2C01D10420C8
:10DAD00006E0094B0F20DC81FFF734FF012806D058
:10DAE000034A41F6EF73116901EA0303136110BDA4
:10DAF000002002402301674500F8FF1F70B504466F
:10DB00000F200E46FFF71EFF042815D10B4D0C4BBE
:10DB10000B30AB6003F18833AB602B6943F010032B
:10DB20002B612680FFF70EFF012805D02A6941F6F8
:10DB3000EF7302EA03032B6170BD00BF00200240B7
:10DB40002301674570B504460F200E46FFF7FAFE25
:10DB5000042810D1084D0B302B6943F001032B61D1
:10DB60002680FFF7EFFE012805D02A6941F6FE73F3
:10DB700002EA03032B6170BD0020024070B5044629
:10DB80000F200E46FFF7DEFE042818D10C4DB3B26D
:10DB90002A690B3042F001022A612380FFF7D2FE8E
:10DBA000042804D1360C66800B30FFF7CBFE012829
:10DBB00005D02A6941F6FE7302EA03032B6170BDAA
:10DBC0000020024010B540F6FF70FFF7BBFE0428AE
:10DBD0002CD1174C174B40F6FF70A36003F188332C
:10DBE000A360236943F020032361236943F04003CA
:10DBF0002361FFF7A7FE042810D1226941F6DF73E5
:10DC000002EA0303236123694FF0A50243F01003E6
:10DC10002361094B0B301A80FFF794FE012805D0D1
:10DC2000226941F6EF7302EA0303236110BD00BFCE
:10DC3000002002402301674500F8FF1F10B540F6A1
:10DC4000FF70FFF77FFE042814D10B4C40F6FF70E5
:10DC5000236943F004032361236943F040032361F4
:10DC6000FFF770FE012805D0226941F6FB7302EA36
:10DC70000303236110BD00BF0020024038B50546F4
:10DC800040F6FF70FFF75EFE042815D10B4C40F6FE
:10DC9000FF70236943F0020323616561236943F048
:10DCA00040032361FFF74EFE012805D0226941F6AB
:10DCB000FD7302EA0303236138BD00BF0020024068
:10DCC000CB78F0B513F0100F18BF8A78098803F0ED
:10DCD0000F0C18BF4CEA020C11F0FF0F1AD00468A9
:10DCE00000220126964006EA0105B5420ED19600B3
:10DCF0000F27B7400CFA06F624EA07043443282B12
:10DD000001D1456102E0482B08BF05610132082AB4
:10DD1000E7D10460FF291CD94468002202F10805FC
:10DD20000126AE4006EA0105B5420ED196000F2746
:10DD3000B7400CFA06F624EA07043443282B01D135
:10DD4000456102E0482B08BF05610132082AE5D190
:10DD50004460F0BD0423C370022383704FF0FF338F
:10DD600003807047836819420CBF00200120704770
:10DD7000806880B2704700BFC36819420CBF0020A2
:10DD800001207047C06880B2704700BF01617047D2
:10DD9000416170470AB1016100E04161704700BF15
:10DDA000C160704741F4803383618161836183691D
:10DDB00083697047064A10B514684FF6807341EACC
:10DDC000001104EA030341EA0303136010BD00BF1E
:10DDD00000000140014B1860704700BF1C0020424A
:10DDE0000304154A00F4401C1B0CBCF5401F30B561
:10DDF000546806D1556824F0706425F0706555604C
:10DE000011E010F4801F06D0C0F303424FF0030C62
:10DE10000CFA02F203E0420D120113FA02F224EAB4
:10DE2000020444F0706419B1400D000183401C43AA
:10DE3000014B5C6030BD00BF0000014001F00303F6
:10DE40009B000F229A4010FA03F310B58908074C83
:10DE5000023154F8210020EA020244F8212054F84B
:10DE60002120134344F8213010BD00BF00000140C1
:10DE70000120014608B500F047FB0120002100F019
:10DE800043FB08BD08B5264B98422BD00CD8A3F510
:10DE9000006398421AD003F5806398421CD0A3F522
:10DEA000006398423AD10BE01E4B984226D003F50E
:10DEB0008063984228D0A3F5006398422ED117E0E2
:10DEC0000420012100F020FB042024E0082001218F
:10DED00000F01AFB08201EE01020012100F014FBC6
:10DEE000102018E02020012100F00EFB202012E07D
:10DEF0004020012100F008FB40200CE0802001219F
:10DF000000F002FB802006E04FF48070012100F059
:10DF1000FBFA4FF48070002100F0F6FA08BD00BF54
:10DF200000140140001C01400B4B4FF0FF316FF01B
:10DF30007042C3F88010C3F88420C3F88011C3F87E
:10DF40008421002303F1C001034A013300200F2B79
:10DF500042F82100F6D1704700E100E0094B4FF094
:10DF600020605860084800224FF0FF319A60D86066
:10DF70001A615A619A61DA611A625A629962D962C7
:10DF80001963704700ED00E00000FA0540F0BE6044
:10DF9000024B40F42020D860704700BF00ED00E045
:10DFA00030B5C27803787AB31C4A4178D2684FF012
:10DFB0000F0CD243C2F302222CFA02FCC2F104027B
:10DFC0009140807803F003020CEA000C4CEA010C4B
:10DFD000D2004FEA0C1CFF2090400CFA02FC0124F6
:10DFE00003F01F02944099080D4AC03152F82150A5
:10DFF0000CEA000C25EA00004CEA00005B0942F83C
:10E00000210042F8234008E003F01F020121914063
:10E010005B09034A203342F8231030BD00ED00E0D5
:10E0200000E100E00023C370037043708370704709
:10E03000024B5868C0F30930704700BF00ED00E0A4
:10E04000012200F01F0312FA03F34009044A403092
:10E0500052F820001840984214BF00200120704759
:10E0600000E100E0014B1860704700BF00EF00E0E6
:10E0700000F01F0301229A404009024B603043F830
:10E080002020704700E100E0024B58688005800DB9
:10E09000704700BF00ED00E0012200F01F0312FAFC
:10E0A00003F34009044A803052F820001840984297
:10E0B00014BF00200120704700E100E0014B186808
:10E0C000704700BF00ED00E021F0604121F07F01CA
:10E0D000014B01439960704700ED00E0014A024B9B
:10E0E000DA6070470400FA0500ED00E0014A024BD7
:10E0F000DA6070470100FA0500ED00E019B1054B48
:10E100001A69104303E0034B1A6922EA0000186100
:10E11000704700BF00ED00E000F01F00012313FA7C
:10E1200000F019B1044B5A6A104303E0024B5A6ADB
:10E1300022EA00005862704700ED00E0144B70B511
:10E14000DC684FF0FF0CE443C4F302242CFA04F51E
:10E15000C4F1040411FA04F4C0F30126F6000CFA29
:10E1600006FC02EA050545EA0404240114FA06F651
:10E17000C0F38110063053F8202022EA0C0243F845
:10E18000202053F82020164343F8206070BD00BFC4
:10E1900000ED00E0C0F3832001238340044A506A6D
:10E1A00003EA0000984214BF00200120704700BF1E
:10E1B00000ED00E000F01F0001228240024B596890
:10E1C0000A435A60704700BF00ED00E000F01F02F4
:10E1D0000123013A13FA02F2024B59680A435A60CA
:10E1E000704700BF00ED00E0C0F38330012383409F
:10E1F000044A506A03EA0000984214BF002001203C
:10E20000704700BF00ED00E0C0F3814313B90A4B33
:10E21000D86A10E0012B0CD1074AC0F30153906A71
:10E22000DA00D040022B14BF00F00F0000F0FF0016
:10E2300001E0014B186B704700ED00E010F4800F17
:10E240000BBF024B014B586B986B704700ED00E021
:10E2500008B5F5F78DFF08BD08B50001F5F785FF96
:10E2600008BD00BF08B5F5F77EFF08BD08B5F5F796
:10E2700078FF08BD08B5F5F772FF08BD08B5F5F7DA
:10E280006CFF08BD0D4B0E4A196841F00101196081
:10E29000596801EA02025A601A6822F0847222F474
:10E2A00080321A601A6822F480221A605A6822F4B6
:10E2B000FE025A6000229A60704700BF00100240C0
:10E2C0000000FFF80C4BB0F5803F1A6822F4803252
:10E2D0001A601A6822F480221A6003D0B0F5802FE9
:10E2E00008D103E01A6842F4803202E01A6842F46E
:10E2F000A0221A60704700BF00100240034B1A684A
:10E3000022F0F80242EAC0021A6070470010024090
:10E31000014B1860704700BF00004242044B5A682E
:10E3200022F47C1240EA02020A435A60704700BF9E
:10E3300000100240014B1860704700BF600042426D
:10E34000034B5A6822F0030240EA02025A60704707
:10E3500000100240024B586800F00C00704700BFEC
:10E3600000100240034B5A6822F0F00240EA020219
:10E370005A60704700100240034B5A6822F4E06272
:10E3800040EA02025A60704700100240034B5A688C
:10E3900022F4605242EAC0025A6070470010024004
:10E3A00019B1054B1A78104303E0034B1A7822EA9F
:10E3B00000001870704700BF09100240014B186040
:10E3C000704700BFD8004242034B5A6822F44042D3
:10E3D00040EA02025A60704700100240064B0022D9
:10E3E00001281A701A7002D0042804D101E01870B4
:10E3F00001E005221A70704720100240014B18609E
:10E40000704700BF80044242024B1A6A40EA02028F
:10E410001A62704700100240014B1860704700BF3D
:10E420003C0442421F4B10B55A6802F00C02042A09
:10E4300013D0082A11D15A685968C2F383420232B4
:10E4400011F4803F03D05B6813F4003F01D0164BFA
:10E4500000E0164B5A43026001E0144B0360114A7E
:10E46000134B51680468C1F30311595C34FA01F18C
:10E4700041605468C4F3022C13F80C4031FA04F4E0
:10E4800084605468C4F3C22C13F80CC021FA0CF158
:10E49000C1605268C2F381329B181B7CB1FBF3F15F
:10E4A000016110BD0010024000093D0000127A0019
:10E4B000002E010819B1054B5A69104303E0034BC4
:10E4C0005A6922EA00005861704700BF00100240FC
:10E4D00019B1054B9A69104303E0034B9A6922EA8C
:10E4E00000009861704700BF0010024019B1054B51
:10E4F000DA69104303E0034BDA6922EA0000D861CD
:10E50000704700BF0010024019B1054BDA68104394
:10E5100003E0034BDA6822EA0000D860704700BFCE
:10E520000010024019B1054B1A69104303E0034B78
:10E530001A6922EA00001861704700BF001002400B
:10E54000014B1860704700BF40044242014B186005
:10E55000704700BF4C004242014B1870704700BF2B
:10E56000071002404309012B02D1084B1B6805E04C
:10E57000022B0BBF054B054B1B6A5B6A00F01F00AB
:10E5800033FA00F000F00100704700BF00100240B5
:10E5900008B53120FFF7E6FF094B18705A680132C1
:10E5A0005A601A7822B95A6840F2FF139A42F0D1A1
:10E5B0003120FFF7D7FF003818BF012008BD00BF8A
:10E5C000DC060020024B5A6A42F080725A627047A1
:10E5D00000100240034B9B6818420CBF0020012032
:10E5E000704700BF00100240014B1870704700BF19
:10E5F0000A1002400B884A88B1F804C01A43CB883D
:10E6000042EA0C02B1F808C01A434B8930B542EA1D
:10E610000C028D89B0F800C0CC891A432A432243EA
:10E620000CF4415313439BB20380838B23F40063A8
:10E630001B041B0C83830B8A038230BD00234FF025
:10E640000702C3810282038043808380C3800381E9
:10E6500043818381704700BF00234381038043804F
:10E660008380C3804FF002030381704721B1038888
:10E670009BB243F0400304E0038823F040031B04F3
:10E680001B0C0380704700BF21B1838B9BB243F406
:10E69000806304E0838B23F480631B041B0C83835F
:10E6A000704700BF0909012313FA01F189B21AB1B9
:10E6B00083889BB2194303E083889BB223EA01015C
:10E6C000818070471AB183889BB2194303E0838825
:10E6D0009BB223EA01018180704700BF81817047AE
:10E6E000808980B2704700BF4FF6FF63994205D022
:10E6F00003889BB243F48073038002E003881940CF
:10E700000180704721B183889BB243F0040304E089
:10E71000838823F004031B041B0C8380704700BF15
:10E72000038823F400631B041B0C038003889BB243
:10E7300041EA03030380704703889BB243F480538C
:10E740000380704721B103889BB243F4005304E077
:10E75000038823F400531B041B0C0380704700BF85
:10E76000012914BF008B808A80B27047008A80B272
:10E77000704700BFB1F5804F04D103889BB243F4CA
:10E78000804304E0038823F480431B041B0C0380B4
:10E79000704700BF038919420CBF00200120704759
:10E7A000202906D1038903889BB243F040030380EC
:10E7B00008E0402901D0082901D1038902E0C943BA
:10E7C00089B20181704700BF012301F00F0213FAE3
:10E7D00002F2B0F804C000891FFA8CFC80B210402D
:10E7E00006D009098B401CEA030F0CBF0020012052
:10E7F000704700BF552906D1038903889BB243F0B7
:10E80000400303800DE0562901D0532901D103892B
:10E8100007E001F00F01012313FA01F1C94389B2A6
:10E8200001817047838BF0B523F47A6323F01F03D3
:10E830001B041B0C83834FF0020303840B89868B1C
:10E84000022B87B004460D46B6B201D1002225E066
:10E8500001A88F88FFF7E6FDEB88002F0CBF01278A
:10E860000227B3F5007F2989019A06D1A3F5FB732E
:10E8700053430902B3FBF1F305E00A2349015A436C
:10E880004F43B2FBF7F305330A229BB2B3FBF2F31B
:10E8900003F001021202C3F34F0392B2991E89B230
:10E8A000FE2928BF002228BF0223E98842EA030389
:10E8B0000B439BB223842B886A8846EA0303A9880A
:10E8C00043F4006313436A890B4313439BB2A3834E
:10E8D00007B0F0BD08B5154B98421BD003F5744343
:10E8E000984204D0A3F5784398421DD10AE0012153
:10E8F0004FF48050FFF708FE4FF480500021FFF7DF
:10E9000003FE11E04FF480400121FFF70BFE4FF4AE
:10E91000804006E04FF400400121FFF703FE4FF472
:10E9200000400021FFF7FEFD08BD00BF003C004095
:10E93000042804D1054B1A6842F0040203E0034B9B
:10E940001A6822F004021A60704700BF10E000E06D
:10E95000014B5860704700BF10E000E0012804D16F
:10E96000084B1A6842F0010206E010F1020F05D1CF
:10E97000044B1A6822F001021A6002E0014B0022E7
:10E980009A60704710E000E020B1054B1A6842F031
:10E99000020203E0024B1A6822F002021A6070477A
:10E9A00010E000E0014B9868704700BF10E000E005
:10E9B000C308022B0BBF044B034B1B68DB6833FA05
:10E9C00000F000F00100704710E000E0038803F061
:10E9D0008F0303800388B1F806C04A889BB243EADC
:10E9E0000C0313439BB203808B8883850B880385BC
:10E9F000064B984203D003F50063984201D10B7A8D
:10EA000003864FF001038382704700BF002C014052
:10EA1000038C2DE9F04123F001031B041B0C03843C
:10EA2000038C0A894C8823F002031C4E14431B04F8
:10EA30008288B1F806C0058B1B0CA4B2B04244EA30
:10EA4000030392B20C88ADB2A0F834C003D006F52F
:10EA50000066B04218D18E894F89B1F80E804FF60A
:10EA6000F77C03EA0C0C4CEA070748EA06064FF667
:10EA7000FB73898847F6FF4C02EA0C0C07EA030394
:10EA8000B2B20B4342EA0C024FF68F7105EA010164
:10EA90002143828001830384BDE8F081002C014082
:10EAA000038C2DE9F04123F010031B041B0C03849D
:10EAB000028CB1F808C022F0200212048488120CE3
:10EAC0004B8842EA0C1242EA0313A2B21B4C068B9B
:10EAD000B1F806C0A0420D88B6B29BB2A0F838C00B
:10EAE00003D004F50064A0421BD1B1F80A804FF6B0
:10EAF0007F748F8903EA040447F2FF3C02EA0C0C9E
:10EB000044EA0814CA894FF6BF73898804EA0303EC
:10EB10004CEA870C43EA01134CEA82023C469BB262
:10EB200092B248F6FF7106EA010141EA052189B275
:10EB3000828001830384BDE8F08100BF002C014086
:10EB4000038C2DE9F04123F480731B041B0C038418
:10EB5000028CB1F808C022F4007212048488120CEE
:10EB60004B8842EA0C2242EA0323A2B21A4C868B5B
:10EB7000B1F806C0A0420D88B6B29BB2A0F83CC066
:10EB800003D004F50064A0421BD1B1F80A804FF213
:10EB9000FF748F8903EA040444F6FF7C02EA0C0C3C
:10EBA00044EA0824CA894FF6FF33898804EA03033C
:10EBB0004CEA071C43EA01234CEA02123C469BB292
:10EBC00092B24FF68F7106EA010129438280818358
:10EBD0000384BDE8F08100BF002C0140038CF0B538
:10EBE00023F480531B041B0C0384B1F806C0078C6C
:10EBF0000C8882880D89868B4B88A0F840C0DFF88E
:10EC000048C0BFB2604592B2B6B203D00CF5006CFA
:10EC1000604505D192048989920C42EA811292B230
:10EC20004DF6FF7C07EA0C0C48F6FF7106EA01017D
:10EC30004CEA053C41EA04214CEA033389B29BB219
:10EC4000828081830384F0BD002C0140B1F802C0B2
:10EC50000B888A884CEA0303B1F806C013430A897B
:10EC600043EA0C03B1F80AC013438A8943EA0C0350
:10EC700013439BB2A0F84430704700BF00234FF00D
:10EC8000FF320372438082800380C380704700BFDD
:10EC90000023C381038043808380C3800381438139
:10ECA0008381704700234FF001020381038043807A
:10ECB0008280C380704700BF00238381038043802C
:10ECC0008380C38003814381704700BF21B10388E3
:10ECD0009BB243F0010304E0038823F001039B058A
:10ECE0009B0D0380704700BF39B1B0F844306FEA24
:10ECF00043436FEA53439BB203E0B0F844305B04F4
:10ED00005B0CA0F8443070471AB183899BB2194359
:10ED100003E083899BB223EA01018181704700BF30
:10ED2000818270470A43A0F8482070471AB183894E
:10ED30009BB2194303E083899BB223EA01018181DD
:10ED4000704700BF038923F007031B041B0C0381DA
:10ED5000704700BFB0F808C05FFA8CFC41EA0C0CA9
:10ED600042EA0C0C4CEA032C1FFA8CFCA0F808C0F9
:10ED7000704700BF10B50446FFF7ECFF23899BB234
:10ED800043F48043238110BD10B50446FFF7E2FF32
:10ED9000238923F077031B041B0C43F077032381A3
:10EDA00010BD00BF01858282704700BF038823F039
:10EDB00070039B059B0D41EA03030380704700BF6E
:10EDC000038923F070031B041B0C41EA0303038136
:10EDD000704700BF10B50446FFF7F2FF23899BB2CE
:10EDE00043F00703238110BD30B50489B0F818C083
:10EDF000058C2CF4407CADB22CF0030C24F00704FD
:10EE00004FEA0C4C25F0220542EA050524044FEA9E
:10EE10001C4C45EA0315240C4CF4807C21434CF037
:10EE2000010CADB20181A0F818C0058430BD00BF4F
:10EE3000038B23F070031B041B0C41EA03030383C1
:10EE4000704700BF038B23F4E0431B041B0C43EA11
:10EE500001239BB203837047838B23F070031B0451
:10EE60001B0C41EA03038383704700BF838B23F4A9
:10EE7000E0431B041B0C43EA01239BB283837047CE
:10EE800021B103889BB243F0800304E0038823F0A0
:10EE900080039B059B0D0380704700BF21B18388D1
:10EEA0009BB243F0040304E0838823F004031B04B3
:10EEB0001B0C8380704700BF21B183889BB243F055
:10EEC000080304E0838823F008031B041B0C8380E1
:10EED000704700BF21B183889BB243F0010304E077
:10EEE000838823F001031B041B0C8380704700BF41
:10EEF000038B23F008031B041B0C41EA0303038369
:10EF0000704700BF038B23F400631B041B0C43EA10
:10EF100001239BB203837047838B23F008031B04F8
:10EF20001B0C41EA03038383704700BF838B23F4E8
:10EF300000631B041B0C43EA01239BB283837047CD
:10EF4000038B23F004031B041B0C41EA030303831C
:10EF5000704700BF038B23F480631B041B0C43EA40
:10EF600001239BB203837047838B23F004031B04AC
:10EF70001B0C41EA03038383704700BF838B23F498
:10EF800080631B041B0C43EA01239BB283837047FD
:10EF9000038B23F080031B041B0C41EA0303038350
:10EFA000704700BF038B5B045B0C43EA01239BB2F9
:10EFB00003837047838B23F080031B041B0C41EAFF
:10EFC00003038383704700BF838B5B045B0C43EABE
:10EFD00001239BB283837047038C23F002031B043D
:10EFE0001B0C41EA03030384704700BF038C23F02A
:10EFF00008031B041B0C41EA03030384704700BF92
:10F00000038C23F020031B041B0C43EA01139BB267
:10F0100003847047038C23F080031B041B0C43EA1A
:10F0200001139BB203847047038C23F400731B0409
:10F030001B0C43EA01239BB203847047038C23F427
:10F0400000631B041B0C43EA01239BB2038470473B
:10F05000038C23F400531B041B0C43EA01339BB2C3
:10F060000384704701238B408A40018C89B221EAD6
:10F0700003030384018C0A4392B20284704700BFE9
:10F0800004238B408A40018C89B221EA0303038464
:10F09000018C0A4392B20284704700BF01238B4067
:10F0A000B0F820C010B51FFA8CFC2CEA03030384CF
:10F0B00009B1082909D11830490844584FF68F730F
:10F0C00004EA0303435043580CE004391830C1F3F9
:10F0D0004E01445848F6FF7304EA030343501202FA
:10F0E000435892B243EA0202425010BD21B1038854
:10F0F0009BB243F0020304E0038823F002039B0564
:10F100009B0D0380704700BF21B103889BB243F081
:10F11000040304E0038823F004039B059B0D038094
:10F12000704700BF21B183889BB243F0800304E0A5
:10F13000838823F080031B041B0C8380704700BF6F
:10F14000038823F008039B059B0D038003889BB273
:10F1500041EA030303807047838823F070031B0494
:10F160001B0C838083889BB241EA03038380704732
:10F17000038923F007031B041B0C038103899BB243
:10F1800041EA030303817047038923F080031B04D2
:10F190001B0C038103899BB241EA0303038170477F
:10F1A00081847047818570478186704701877047E9
:10F1B00081877047A0F84010704700BF038B23F091
:10F1C0000C031B041B0C0383038B9BB241EA030358
:10F1D00003837047038B23F440631B041B0C0383DE
:10F1E000038B9BB243EA01239BB20383704700BFAA
:10F1F000838B23F00C031B041B0C8383838B9BB238
:10F2000041EA030383837047838B23F440631B0429
:10F210001B0C8383838B9BB243EA01239BB28383C2
:10F22000704700BF0388DBB2038003889BB241EACA
:10F2300003030380704700BF808E80B2704700BF19
:10F24000008F80B2704700BF808F80B2704700BFD0
:10F25000B0F8400080B27047808C80B2704700BF29
:10F26000008D80B2704700BF038A19420CBF002096
:10F2700001207047C94389B201827047038A82899D
:10F2800011EA030092B203D011420CBF002001200A
:10F29000704700BFC94389B201827047B0F820C0EF
:10F2A00010B52CF0010C4FEA0C4C4FEA1C4CA0F8A6
:10F2B00020C0048BB0F820C0A4B21FFA8CFC24F04C
:10F2C000F30442EA04042CF0020C44EA03144CF068
:10F2D000010C4CEA010CA4B20483A0F820C010BDBC
:10F2E000B0F820C010B52CF0100C4FEA0C4C4FEACF
:10F2F0001C4CA0F820C0B0F818C0048C2CF4407C42
:10F30000A4B24FEA0C5C4FEA1C5C24F020044CEAE7
:10F31000022C44F010044CEA033C44EA01141FFAA6
:10F320008CFCA4B2A0F818C0048410BD38B50D46FA
:10F33000602D1146044603D10122FFF7D1FF02E000
:10F340000122FFF7ABFF29462046FFF739FD23894D
:10F350009BB243F00703238138BD00BFF8B50C46CC
:10F36000A2884988B4F800C0054600290CBF0227CE
:10F370000027012A0CBF022601262389BCF1000FB9
:10F3800010D1FFF78BFF2846E188FFF717FF2846CB
:10F39000394632462389FFF7A3FF2846E188FFF765
:10F3A00019FF0FE0FFF79CFF2846E188FFF712FFE7
:10F3B0002846394632462389FFF770FF2846E18800
:10F3C000FFF7FCFEF8BD00BF38B50B880C460546BC
:10F3D0004BB94988A2882389FFF760FF2846E18856
:10F3E000FFF7ECFE53E0042B09D14988A28823895A
:10F3F000FFF776FF2846E188FFF7ECFE47E0082B91
:10F40000B1F802C0B1F804E0098920D1028C22F4DD
:10F4100080721204120C0284838B028C9BB292B213
:10F4200023F0F30322F4007243EA011142EA0C2CA8
:10F4300089B21FFA8CFC41EA0E0E4CF4807CA0F8D5
:10F440001CE0A0F820C0E188FFF7D2FE1FE0028C8C
:10F4500022F480521204120C0284838B028C23F457
:10F46000407392B21B051B0D22F4005243EA0E2397
:10F4700042EA0C3C43EA01331FFA8CFC9BB24CF489
:10F48000805C8383A0F820C0E188FFF7BDFE38BD13
:10F4900008B52D4B984237D00BD8A3F5006398429E
:10F4A00026D003F58063984228D0B0F1804F4AD12E
:10F4B00018E0264B984233D004D8A3F580639842D5
:10F4C00041D127E0224B984204D003F500639842D3
:10F4D00039D12EE04FF400600121FFF715F84FF409
:10F4E00000602DE001200146FFF71CF801201CE020
:10F4F00002200121FFF716F8022016E00420012166
:10F50000FFF710F8042010E008200121FFF70AF8A7
:10F5100008200AE010200121FFF704F8102004E081
:10F5200020200121FEF7FEFF20200021FEF7FAFF38
:10F5300009E04FF400500121FEF7E6FF4FF40050C0
:10F540000021FEF7E1FF08BD000C00400014004060
:10F55000002C0140002383814FF416528380C38026
:10F5600003814FF00C030260438170470A8810B595
:10F570004C88B1F804C0038AC98844EA020242EA0E
:10F580000C0223F470630A431B041B0C92B242EA80
:10F590000303038210BD00BF0023C38003804380A8
:10F5A0008380704721B183899BB243F4005304E008
:10F5B000838923F400531B041B0C8381704700BF15
:10F5C00001F01F034FF0010CC1F3421161450CFA29
:10F5D00003F301D10C3004E0022901D1103000E026
:10F5E00014301AB1026842EA030302E0026822EA18
:10F5F00003030360704700BF1AB1838A9BB21943AB
:10F6000003E0838A9BB223EA01018182704700BF35
:10F61000038A23F00F031B041B0C0382038A9BB293
:10F6200041EA030303827047838923F400631B04C8
:10F630001B0C838183899BB241EA0303838170475A
:10F6400021B183899BB243F0020304E0838923F054
:10F6500002031B041B0C8381704700BF038A23F045
:10F6600020031B041B0C0382038A9BB241EA0303A1
:10F670000382704721B1038A9BB243F4804304E0C4
:10F68000038A23F480431B041B0C0382704700BFD2
:10F69000C905C90D818070478088C005C00D7047BD
:10F6A00083899BB243F0010383817047038BDBB2F4
:10F6B0000383038B9BB243EA01230383704700BF9C
:10F6C000038B03F47F430383038B9BB241EA030361
:10F6D0000383704721B1838A9BB243F0200304E087
:10F6E000838A23F020031B041B0C8382704700BF16
:10F6F00021B1838A9BB243F0100304E0838A23F094
:10F7000010031B041B0C8382704700BF21B1838A46
:10F710009BB243F0080304E0838A23F008031B0430
:10F720001B0C8382704700BF838A23F004031B04F1
:10F730001B0C8382838A9BB241EA03038382704756
:10F7400021B1838A9BB243F0020304E0838A23F051
:10F7500002031B041B0C8382704700BF03881942FD
:10F760000CBF002001207047C94389B20180704757
:10F770004FF0010CC1F3421201F01F0362450CFA75
:10F7800003F301D1828903E0022A0CBF028A828A34
:10F7900092B21340028892B20BB9184607E0090AE8
:10F7A000012313FA01F111420CBF00200120704720
:10F7B000090A01238B40DB439BB20380704700BFE3
:10F7C000038ACA8823F440531B041B0C134303828F
:10F7D00083898A8830B5044608890D4623F4B053DE
:10F7E000498940EA020223F00C030A431B041B0C64
:10F7F00092B242EA0303A381A38AAA8923F4407345
:10F800001B041B0C134387B0A38201A8FEF70AFE5A
:10F810000E4B2A689C420CBF049B039B1921594341
:10F8200092006423B1FBF2F1B1FBF3F21201100973
:10F8300003FB101109013231B1FBF3F303F00F03A5
:10F8400043EA020292B2228107B030BD0038014083
:10F8500008B5214B98422BD008D8A3F500639842F5
:10F8600016D003F58063984234D119E01B4B9842BF
:10F8700026D003F5684398422CD101214FF48040F3
:10F88000FEF742FE4FF480400021FEF73DFE21E0EE
:10F890004FF400300121FEF745FE4FF4003016E032
:10F8A0004FF480200121FEF73DFE4FF480200EE052
:10F8B0004FF400200121FEF735FE4FF4002006E052
:10F8C0004FF480100121FEF72DFE4FF4801000212F
:10F8D000FEF728FE08BD00BF004C0040005000406D
:10F8E000684620F007018D4601B5002303E00B496F
:10F8F0005958995004330A4A0A4998188842F6D34D
:10F90000094B02E0002243F8042B084A9342F9D342
:10F91000F4F762FCBDE8014085467047582F0108A6
:10F92000000000203002002030020020C00E002025
:10F9300010B5074C20B922684FF00103138205E08F
:10F94000044B1B681B68984720680A3010BD00BF35
:10F95000580E0020140E002010B50A4B0A4A1B68EE
:10F960005178DA7891420AD3997841B99C8834B9B0
:10F970009A72064B1B685B689847204600E002209D
:10F9800010BD00BF580E002004010020140E0020FE
:10F9900010B5074C20B922684FF00103138205E02F
:10F9A000044B1B689B68984720680C3010BD00BF53
:10F9B000580E0020140E002038B50E4C0E4B226855
:10F9C0001B68D1789B695079984723689A7A7AB1F5
:10F9D00070B91A7962B99D7855B9084B1B68DB6814
:10F9E0009847236828465979DA78D9721A7300E063
:10F9F000022038BD580E0020F00D0020140E00200B
:10FA000008B50246244B20B91B684FF00201198249
:10FA100040E0224A4FF000011B681180197811F074
:10FA20007F0113D15B7A13F0200F03D0117841F0DE
:10FA30000201117013F0400F184B15BF1A781A7895
:10FA400022F0010242F001021A701EE0012921D0C9
:10FA5000022901D000221DE0597911F0800F01F038
:10FA60000F0306D00E4951F8233003F03003102B5A
:10FA700006E00B4951F8233003F44053B3F5805F9F
:10FA800003D1137843F001031370064B1B681B6905
:10FA90009847024A104608BD580E0020B80E0020B4
:10FAA000005C0040140E002010B51E4B19684A7906
:10FAB00012F0800F22F0800305D01B4850F823007D
:10FAC00000F0300004E0184850F8230000F44050E3
:10FAD000164C94F800C0634522D24C8804BBF8B1A0
:10FAE000897AE9B112F0800F09D00F4948F6BF7248
:10FAF00051F8230000EA020282F0100208E00A49ED
:10FB00004BF68F7251F8230000EA020282F4805211
:10FB100041F82320064B1B689B699847002000E0B2
:10FB2000022010BD580E0020005C0040040100209F
:10FB3000140E002008B5064B1B685A7A42F02002CA
:10FB40005A72044B1B68DB699847002008BD00BF50
:10FB5000580E0020140E0020054B1A68538A18B95D
:10FB60008988CB1A138201E008681818704700BF13
:10FB7000580E002030B50E4B1C78002310E05FFAC1
:10FB800083FC4FEA8C0202F1804202F5B84215680C
:10FB900048F68F7105EA010141EA0C011160013359
:10FBA000A342ECD3034B40F08000186030BD00BF8F
:10FBB000040100204C5C0040704700BF08B50C4BAE
:10FBC000002093F82C1000F04FFE0A4B1B68187AA7
:10FBD000082807D1084B4FF480521A80074B4FF08A
:10FBE00010021A80092814BF0020012008BD00BFA0
:10FBF00080000020580E0020BA0E0020BC0E00200D
:10FC000070B52D4B1C68237A032B01D0052B46D1F0
:10FC1000A369228AABB1A2B1A58A954228BF154635
:10FC200028469847228A638A521BEB18064622828E
:10FC30006382002000F0E8FD2A460146304600F0CD
:10FC4000FBFB238A5BB11D4B4FF4405200201A800E
:10FC5000014600F0E7FD1A4B4FF030021A80A28AED
:10FC6000238A9A4203D8144B03221B6803E0124AEA
:10FC70001BB1136805221A720DE012680621117279
:10FC8000104A1168104A89B28A18520013600C4B4E
:10FC90004FF030021A80084B1B681B7A06E0072BD6
:10FCA00003D10A4B1B68DB6898470823024A126895
:10FCB0001372FFF783FF70BD580E0020BA0E0020AC
:10FCC000BC0E0020505C004002300020F00D0020EF
:10FCD000F8B5244B1C68238A267ABBB9042E15D1AB
:10FCE000214822490278012A0BD1214C214A24685B
:10FCF0000370A0B28218520013604FF030020A80E5
:10FD00002BE04FF010030B80072626E0A68AA2699D
:10FD10009E4234BF35461D462846B34294BF042652
:10FD2000022690470746002000F060FD2A46014663
:10FD3000384600F069FB2946002000F073FD638A15
:10FD4000228AEB186382094B551B4FF03002258243
:10FD50001A80094B4FF440521A80024B1B681E72E6
:10FD6000F8BD00BF580E0020E4060020BC0E0020A5
:10FD7000505C004002300020BA0E002008B5144B41
:10FD80001B681A7A022A01D0042A05D1FFF7A0FFC6
:10FD90000F4B1B681B7A14E0062A11D15A78052AEA
:10FDA0000AD11A7812F07F0F06D1D878FFF7E2FE59
:10FDB000084B1B681B6A9847074B1B689B68984752
:10FDC0000823034A12681372FFF7F8FE08BD00BF4C
:10FDD000580E0020140E0020F00D002038B5324BD4
:10FDE0001B68187810F07F0004D15A7A22F02002A4
:10FDF0005A7258E0022855D15A88002A52D11A79ED
:10FE0000002A4FD15A7912F0800F22F0800405D0D9
:10FE1000264951F8241001F0300104E0234951F83B
:10FE2000241001F440512248007884423AD200293B
:10FE300038D09B7A002B35D012F0800F0FD01B4B9F
:10FE400053F8243003F03003102B25D1E4B22046C0
:10FE500000F082FC2046302100F05EFB1CE0134DD8
:10FE600055F8243003F44053B3F5805F14D134B90E
:10FE7000104B204693F82C1000F0F6FC02E02046D0
:10FE800000F056FC55F824204BF68F7302EA03036A
:10FE900083F4405345F82430074B1B685B6998474F
:10FEA000002000E0022038BD580E0020005C004019
:10FEB0000401002080000020140E0020F7B58D4BB7
:10FEC0008D4E1A6835688D4B92B2D3182A7A5B0032
:10FED000092A1B681BD09BB203F1005303F5405362
:10FEE0005B001C4614F8012B03F10A072A705B78AB
:10FEF0006B70B4F8030000F063FE6880B4F807008C
:10FF0000346800F05DFEA08033687F88DF807A4C23
:10FF100001212368DA8819725D78002A62D11A7883
:10FF200012F07F022ED1092D02D1FFF715FD3BE023
:10FF3000052D0DD193F90320002A4EDB9A78002A73
:10FF40004BD19A88002A48D19B7A002B37D044E0C5
:10FF5000032D0BD1DA78012A27D19A882ABB5B7A44
:10FF600013F0200F21D0FFF7E5FD1DE0012D1CD17E
:10FF7000DA78012A19D19A88BAB95B7A13F0200F7E
:10FF800013D00AE0012A04D10B2D0ED1FFF714FD86
:10FF90000AE0022A09D1012D02D1FFF71FFF03E079
:10FFA000032D02D1FFF780FD48B1554B28461B6851
:10FFB0005B699847032801D109230FE068B94D4ACE
:10FFC000504B12684FF0300192B2D3185B00002200
:10FFD0001A604D4B1980062300E00823464A126838
:10FFE0001372E3E0062D18D11A7812F07F0F40F05B
:10FFF00097809B78012B03D1414B1B68DB696EE036
:020000040801F1
:10000000022B03D13E4B1B681B6A68E0032B40F0B8
:1000100087803B4B1B685B6A61E0002D3CD15988AF
:1000200000297DD15A6822F47F42B2F5003F77D192
:100030001A7812F07F0203D19B88002B70D129E03F
:10004000012A0BD158792E4B1B689B6998470028D1
:1000500066D123689B7A002B62D01BE0022A5FD115
:100060005B7913F0800F03F00F0205D0274951F898
:10007000221001F0300104E0244951F8221001F46B
:1000800040512348007882424AD213F0700F47D182
:10009000002945D01F4B23E0082D05D11B7813F014
:1000A0007F0F3DD11C4B1BE00A2D39D11A7802F08D
:1000B0007F02012A34D19A7A002A31D05988002946
:1000C0002ED15A6822F47F42B2F5803F28D1587968
:1000D0000B4B1B689B69984710BB104B00E0FBB1B2
:1000E000054A4FF000011268002093615182984741
:1000F000002020E0505C0040580E0020043000201A
:10010000F00D002002300020BC0E0020005C0040FA
:100110000401002001FA000831F9000891F90008F3
:10012000244C254B22681B6850781B69984703288C
:1001300001D1236806E01F4B4FF6FF711B681A8A36
:100140008A4201D1092203E0022800D012B9082214
:100150001A722BE093F90010002921DAD988019155
:100160000198824202D9019A1A8211E08A420FD282
:100170001149096891F82C108A4201D2002105E04A
:1001800092FBF1F001FB102212B901210B4A117010
:10019000094A126892F82C209A82FFF799FD05E02F
:1001A00003221A72064B4FF440521A80FFF706FDE5
:1001B000FEBD00BF580E0020F00D0020E406002018
:1001C000BA0E0020074A022108B5074811720749F4
:1001D000074B086007490A60074A13601B68984785
:1001E00008BD00BFF80D002008010020140E0020FB
:1001F00080000020580E0020F00D002008B529E0F6
:1002000047F6FF700860198801F00F018B0003F1B9
:100210008043117003F5B843196889B211F4004F97
:1002200009D0186840F68F7100EA01011960127850
:100230000E4B013A0BE011F0800F0BD0186848F616
:100240000F7100EA010119601278094B013A53F865
:10025000223098470749084B0868084A80B218803E
:10026000188800B20028CBDB08BD00BFE8000020E2
:10027000CC000020445C0040EE0D0020F40D002076
:10028000F8B59AE047F6FF761E601688564F06F0DE
:100290000F06B30003F1804303F5B8433E70002E10
:1002A00064D127682668236807F4405C03EA0000ED
:1002B00080F400502060236806F0300003EA01015A
:1002C00081F0200121601388484A13F0100F10803C
:1002D000A5F800C004D023689BB213F0800F08D0AB
:1002E000226848F60F7302EA03032360FFF746FD16
:1002F00016E013F4006F08D0226840F68F7302EA0C
:1003000003032360FFF7DAFD0AE013F4004F54D033
:10031000226840F68F7302EA03032360FFF770FC44
:1003200021682A884BF68F7301EA030312F4805F79
:1003300018BF83F4805312F4005F2D4A18BF83F472
:1003400000531360294B11681A8848F6BF7301EAFD
:10035000030312F0100F18BF83F0100312F0200FE8
:10036000234A18BF83F0200313603BE01C68A4B24B
:1003700014F4004F0BD0196840F68F7201EA0202A4
:100380001A603A781B4B013A53F82230984714F020
:10039000800F12D0144948F60F720B789B0003F1BE
:1003A000804303F5B843186800EA02021A600A782D
:1003B000114B013A53F822309847104B104A1D68F0
:1003C0000B4C1FFA85FCA2F800C0B2F800C04BF637
:1003D0008F700FFA8CFCBCF1000F48F6BF71094D0D
:1003E000FFF650AFF8BD00BFF40D0020BC0E00209A
:1003F000005C0040E8000020CC000020445C00408D
:10040000EE0D0020BA0E002001F10051013201F57D
:10041000405110B549005208002308E010F803C00D
:100420006478013A4CEA042C21F813C00233C41852
:10043000002AF3D110BD00BF01F10051013201F5D6
:10044000405110B549005208002304E031F8134030
:10045000013AC4520233002AF8D110BD014B186092
:10046000704700BF405C0040014B186880B2704785
:10047000405C0040014B1860704700BF445C004086
:10048000014B186880B27047445C0040014B18680B
:1004900080B27047485C0040014B1860704700BF55
:1004A0004C5C0040014B186880B270474C5C0040C7
:1004B0004FF6F873024A00EA03031360704700BF67
:1004C000505C0040014B186880B27047505C00409F
:1004D000014B43F820107047005C0040024B53F87A
:1004E000200080B2704700BF005C0040054B10B593
:1004F00053F8204048F68F1204EA02020A4343F8F8
:10050000202010BD005C0040024B53F8200000F496
:10051000C0607047005C00400A4B10B553F82020C3
:1005200048F6BF7402EA040411F0100F18BF84F0FB
:10053000100411F0200F18BF84F0200443F820406D
:1005400010BD00BF005C00400A4B10B553F82020DE
:100550004BF68F7402EA040411F4805F18BF84F430
:10056000805411F4005F18BF84F4005443F8204015
:1005700010BD00BF005C004038B50D460446FFF7D3
:10058000ADFF012D02D120F4805003E0022D04D1F3
:1005900020F01000014B43F8240038BD005C0040FF
:1005A000024B53F8200000F030007047005C004020
:1005B000024B53F8200000F440507047005C0040AC
:1005C000054B48F6BF7253F8201001EA020282F090
:1005D000300243F820207047005C0040054B4BF68A
:1005E0008F7253F8201001EA020282F4405243F85D
:1005F00020207047005C0040054B48F68F6253F89E
:10060000201001EA020242F4807243F82020704771
:10061000005C0040044B48F68F6253F8201001EA5A
:10062000020243F820207047005C0040044B48F66B
:100630008F6253F8201001EA020243F8202070472D
:10064000005C0040054B48F68F6253F8201001EA29
:10065000020242F4807243F820207047005C0040A0
:10066000054B48F68F6253F8201001EA020242F46B
:10067000807243F820207047005C0040044B48F62D
:100680008F6253F8201001EA020243F820207047DD
:10069000005C0040044B53F8200000F030001028AC
:1006A00014BF002001207047005C0040054B53F848
:1006B000200000F44050B0F5805F14BF00200120FE
:1006C000704700BF005C0040044B40F68F7253F847
:1006D000201001EA020243F820207047005C00402D
:1006E000044B48F60F7253F8201001EA020243F857
:1006F00020207047005C0040054B48F68F7253F88D
:10070000201001EA020242F4804243F820207047A0
:10071000005C0040054B48F68F7253F8201001EA48
:10072000020242F0400243F820207047005C004083
:10073000084B53F8202012F4804F09D053F82010B2
:1007400048F68F7201EA020242F4804243F8202008
:10075000704700BF005C0040084B53F8202012F0A7
:10076000400F09D053F8201048F68F7201EA0202B8
:1007700042F0400243F82020704700BF005C004078
:10078000054B10B553F8204048F68F7204EA020278
:100790000A4343F8202010BD005C0040024B53F890
:1007A000200000F00F007047005C0040064B490835
:1007B0001B6849009BB203EBC00303F1005303F530
:1007C00040535B0019607047505C0040054A064B7F
:1007D0001268490892B202EBC002D3185B004900CC
:1007E00019607047505C004004300020054B1B68C6
:1007F0009BB203EBC00303F1005303F540535B00CE
:1008000018887047505C0040044A054B126892B249
:1008100002EBC002D3185B0018887047505C0040A0
:1008200004300020044A054B126892B202EBC00269
:10083000D3185B0019607047505C00400230002004
:100840003E2909D94B0911F01F0F01D1013B9BB281
:100850009B0243F4004305E04B0811F0010F18BF61
:1008600001339B02036070470D4A0E4B126892B22F
:10087000D31803EBC0035B003E2909D94A0911F0E4
:100880001F0F01D1013A92B2920242F4004205E0F8
:100890004A0811F0010F18BF013292021A60704726
:1008A000505C004006300020054A064B126892B2A8
:1008B00002EBC002D3185B0018688005800D7047FA
:1008C000505C004002300020054A064B126892B28C
:1008D00002EBC002D3185B0018688005800D7047DA
:1008E000505C0040063000200C4B30B51D681C6881
:1008F000C0001FFA85FC8444A4B2094B00190CF116
:10090000005CC3180CF5405C490852084FEA4C00E3
:1009100049005B00520001601A6030BD505C00402D
:1009200004300020064B49081B6849009BB203EBCA
:10093000C00303F1005303F540535B001960704797
:10094000505C0040054A064B1268490892B202EB1F
:10095000C002D3185B00490019607047505C00402A
:1009600004300020054B1B689BB203EBC00303F16E
:10097000005303F540535B0018887047505C0040FB
:10098000044A054B126892B202EBC002D3185B0016
:1009900018887047505C004004300020012910B5D1
:1009A00024D1254B25491B68C0009BB25918091852
:1009B0004B003E2A09D9510912F01F0F01D101390C
:1009C00089B2890241F4004105E0510812F0010F9B
:1009D00018BF0131890219601749194B096889B29A
:1009E000CB18181840003E2A1ED913E0022922D144
:1009F000114BC0001C681B68A4B21FFA83FC0F498E
:100A00000F4B844400194118634449005B000A609D
:100A10001A6010E0530912F01F0F01D1013B9BB285
:100A20009B0243F4004305E0530812F0010F18BF86
:100A300001339B02036010BD505C00400230002077
:100A40000630002001291BD11349144B096889B2D3
:100A5000CB1803EBC00040003E2A09D9530912F01D
:100A60001F0F01D1013B9BB29B0243F4004305E001
:100A7000530812F0010F18BF01339B0203600AE014
:100A8000022908D10449054B096889B201EBC0006D
:100A9000C3185B001A607047505C004002300020B1
:100AA00001291BD11349144B096889B2CB1803EBF8
:100AB000C00040003E2A09D9530912F01F0F01D18E
:100AC000013B9BB29B0243F4004305E0530812F044
:100AD000010F18BF01339B0203600AE0022908D10D
:100AE0000449054B096889B201EBC000C3185B00DB
:100AF0001A607047505C004006300020054A064BE3
:100B0000126892B202EBC002D3185B00186880052D
:100B1000800D7047505C004002300020054A064BB3
:100B2000126892B202EBC002D3185B00186880050D
:100B3000800D7047505C0040063000200D4BC00017
:100B400019680D4A89B241188A185200128812F4A5
:100B50007C4F01D001200CE01A68084B92B280183B
:100B6000C3185B0018888005800D002814BF022080
:100B700000207047505C004006300020023000200A
:100B8000012909D10B4A48F68F7352F8201001EA67
:100B9000030343F040030AE002290AD1054A48F65C
:100BA0008F7352F8201001EA030343F4804342F8A4
:100BB00020307047005C004041EA0020704700BFD1
:100BC000030AC0B243EA0020704700BF08B5002204
:100BD0000A2300F045F808BD08B500210A2200F0FC
:100BE000DFF808BDF0B40378002B2DD040F23412AA
:100BF000C2F20002156802E010F8013FEBB15A1989
:100C000003F12004527812F001070A7808BF1C464D
:100C100001F10101561C9446AE5D16F0010F18BF9C
:100C200002F1200C6445E7D007B1203316F0010F24
:100C300018BF2032981AF0BC70470A786F78561C9B
:100C400007F00107AE5DEFE740F234100A78C2F218
:100C50000000561C05686F78AE5D07F00107E3E7FA
:100C60002DE9F04F40F23415C2F2000583B00C4676
:100C70001F46D5F800800E460190009216F8015BE1
:100C800008EB050393F801B01BF0080BF6D12D2DEE
:100C900065D02B2D08BF16F8015BD7F1010338BFD3
:100CA0000023102F14BF1A4643F0010232B1302D39
:100CB00066D01BB1302D0CBF08270A27BBF1000FEF
:100CC000394614BF4FF000496FF00049484600F024
:100CD00059FC48468A46394600F026FB00218C46DE
:100CE00008EB0502A5F13003527812F0040F08D189
:100CF00012F0030F20D012F0010F14BF3723572337
:100D0000EB1A9F4218DD844594BF0022012252EA6B
:100D1000D1714FF0FF310CD1844514BF0022012264
:100D20005345D4BF002202F0010212B907FB0C3C6C
:100D3000012116F8015BD3E7B1F1FF3F14D0BBF1FD
:100D4000000F09D16046009B1BB101B1741E009ACF
:100D5000146003B0BDE8F08FCCF10000F3E716F8A3
:100D6000015B4FF0010B98E7019ABBF1000F4FF0C8
:100D7000220314BF4FF000406FF000401360E2E721
:100D80003278782A14BF00210121582A14BF0A465C
:100D900041F00102002A8CD07578102702368DE7C9
:100DA00010B540F23814C2F200048C4613460146D6
:100DB00062462068FFF754FF10BD00BF2DE9F043E5
:100DC0008BB006460F4600F07BF840F22C24C2F2AE
:100DD000000494F90030B3F1FF3F8046894638D0D3
:100DE0003046394600F084FA0546002831D13046B5
:100DF00039460022002301F01DF8002829D124786B
:100E000042F64873C0F6010308950193CDE90267E5
:100E1000CDE90467002C21D040F200030022CFF678
:100E2000F0733046CDE9062339460022002300F056
:100E3000D9FF002822D0022300939C4234D0684678
:100E400000F064FA00282FD0089B002B27D1DDE9A1
:100E50000689404649460BB0BDE8F0834FF6FF7364
:100E60004FF06042CCF2EF733046CDE906233946AD
:100E70000022002300F0B6FF0028DCD10123022C61
:100E8000009316D0684600F041FA90B142F64C70DB
:100E9000C0F6010000F03CFACDE90601D4E700F00D
:100EA0003DFA089B0360D2E700F038FA2223036082
:100EB000CAE700F033FA21230360E7E700000000EF
:100EC000B1F5801F0B462DE9F04F804687B089466B
:100ED00004460D463EDB4FF6FF720026C7F6EF7262
:100EE000934251DC23F07F4445F6647C24F4700483
:100EF000C0F2090CA44440F20002A6F57E760CF480
:100F0000801C073EC3F6F0728CEA020206EB235601
:100F100040F20003404642EA0401C3F6F0730022A7
:100F200006EB1C5600F042FBA31C23F07F4323F486
:100F30007003022B804689462FDC0022002300F03C
:100F400051FF002800F0CA80002E40F07C81002074
:100F500000211FE021F00043034300F0B580002989
:100F6000C0F2468140F200030022C4F250336FF019
:100F7000350600F0CFFC4FF6FF72C7F6EF720B4656
:100F8000804693428946ADDD4046494642464B463F
:100F900000F00EFB07B0BDE8F08F00224FF0804359
:100FA00000F006FB4EF68635CFF6F9756519024658
:100FB0000B464046494600F0D7FDCDE902013046D8
:100FC00000F042FCCDE90401DDE9020102460B46D6
:100FD00000F0A0FC02460B46CDE9000100F09AFCAF
:100FE000A7A3D3E9002382468B4600F093FCA6A377
:100FF000D3E9002300F0DCFA52465B4600F08AFC9D
:10100000A3A3D3E9002300F0D3FA52465B4600F0D5
:1010100081FCA1A3D3E9002300F0CAFADDE9002393
:1010200000F078FC9EA3D3E90023CDE900015046EF
:10103000594600F06FFC9CA3D3E9002300F0B8FAF6
:1010400052465B4600F066FC99A3D3E9002300F00A
:10105000AFFA52465B4600F05DFC0B460246DDE906
:10106000000100F0A5FA4BF65103C0F206031B1B6A
:1010700043EA0505002D82468B4656DD40F200030B
:101080000022C3F6E0734046494600F043FC424666
:101090004B4600F03FFC04460D46002E75D15246EB
:1010A0005B4600F085FADDE9022300F033FC0246DE
:1010B0000B462046294600F079FA02460B46404688
:1010C000494600F073FA65E740F200010020002273
:1010D0000023CCF2503100F047FD5BE742464B461F
:1010E0004046494600F016FC73A3D3E900230446AA
:1010F0000D464046494600F00DFC40F20003002238
:10110000C3F6E07300F054FA02460B462046294627
:1011100000F000FC04460D46002E72D140464946C0
:1011200022462B4600F042FA34E7002E00F0D4802D
:1011300063A3D3E90023DDE9040100F0EBFB524691
:101140005B4606460F464046494600F02FFADDE969
:10115000022300F0DFFB5CA3D3E9002304460D4625
:10116000DDE9040100F0D6FB02460B462046294685
:1011700000F01EFA42464B4600F018FA02460B46B3
:101180003046394600F012FA04E74DA3D3E90023B4
:10119000DDE9040100F0BEFB52465B46CDE90001EB
:1011A0002046294600F004FADDE9022300F0B2FBF4
:1011B00047A3D3E9002306460F46DDE9040100F00A
:1011C000A9FB02460B463046394600F0F1F90246CB
:1011D0000B462046294600F0E9F942464B4600F00E
:1011E000E5F902460B46DDE9000100F0DFF9D1E642
:1011F00002460B4600F0DAF90022002300F0B4FCAE
:10120000C8E6304600F020FB2DA3D3E900230646B4
:101210000F4600F07FFB2CA3D3E9002382468B46C8
:101220003046394600F076FB22462B4600F0C0F9E6
:1012300042464B4600F0BAF902460B465046594624
:1012400000F0B4F9A6E6304600F0FEFA1CA3D3E99C
:10125000002306460F4600F05DFB1DA3D3E90023E3
:1012600004460D463046394600F054FB02460B4614
:101270002046294600F09CF98CE600BFAFF30080C1
:1012800044523EDF12F1C23FDE03CB966446C73FB5
:10129000599322942449D23F935555555555E53FCE
:1012A0009FC678D0099AC33FAF788E1DC571CC3FD9
:1012B00004FA97999999D93F555555555555D5BF24
:1012C0000000E0FE422EE63F763C7935EF39EABD7C
:1012D000763C7935EF39EA3D02460B4640464946B1
:1012E00000F064F9DDE9022300F014FBE5E600BF3D
:1012F00002464042104321F0004141EAD070C0F163
:10130000FE4000F57000C00F704700BF002070471E
:1013100040F200010020C7F6F871704740F2381320
:10132000C2F20003186870474A1E08BF7047C0F039
:101330002481884240F21681114200F01781B0FAF0
:1013400080F3B1FA81F2A2EB0303C3F11F0304A2FD
:1013500002EB03134FF000029F4600BFAFF3008083
:10136000B0EBC17F00BF42EB020228BFA0EBC1700F
:10137000B0EB817F00BF42EB020228BFA0EB81707F
:10138000B0EB417F00BF42EB020228BFA0EB4170EF
:10139000B0EB017F00BF42EB020228BFA0EB01705F
:1013A000B0EBC16F00BF42EB020228BFA0EBC160EF
:1013B000B0EB816F00BF42EB020228BFA0EB81605F
:1013C000B0EB416F00BF42EB020228BFA0EB4160CF
:1013D000B0EB016F00BF42EB020228BFA0EB01603F
:1013E000B0EBC15F00BF42EB020228BFA0EBC150CF
:1013F000B0EB815F00BF42EB020228BFA0EB81503F
:10140000B0EB415F00BF42EB020228BFA0EB4150AE
:10141000B0EB015F00BF42EB020228BFA0EB01501E
:10142000B0EBC14F00BF42EB020228BFA0EBC140AE
:10143000B0EB814F00BF42EB020228BFA0EB81401E
:10144000B0EB414F00BF42EB020228BFA0EB41408E
:10145000B0EB014F00BF42EB020228BFA0EB0140FE
:10146000B0EBC13F00BF42EB020228BFA0EBC1308E
:10147000B0EB813F00BF42EB020228BFA0EB8130FE
:10148000B0EB413F00BF42EB020228BFA0EB41306E
:10149000B0EB013F00BF42EB020228BFA0EB0130DE
:1014A000B0EBC12F00BF42EB020228BFA0EBC1206E
:1014B000B0EB812F00BF42EB020228BFA0EB8120DE
:1014C000B0EB412F00BF42EB020228BFA0EB41204E
:1014D000B0EB012F00BF42EB020228BFA0EB0120BE
:1014E000B0EBC11F00BF42EB020228BFA0EBC1104E
:1014F000B0EB811F00BF42EB020228BFA0EB8110BE
:10150000B0EB411F00BF42EB020228BFA0EB41102D
:10151000B0EB011F00BF42EB020228BFA0EB01109D
:10152000B0EBC10F00BF42EB020228BFA0EBC1002D
:10153000B0EB810F00BF42EB020228BFA0EB81009D
:10154000B0EB410F00BF42EB020228BFA0EB41000D
:10155000B0EB010F00BF42EB020228BFA0EB01007D
:10156000104670470CBF012000207047B1FA81F28D
:10157000C2F11F0220FA02F0704708B14FF0FF30AD
:1015800000F00EB80029F8D02DE90340FFF7CCFE9B
:10159000BDE8064002FB00F3A1EB0301704700BF6A
:1015A000704700BF81F0004102E000BF83F00043BC
:1015B00030B54FEA41044FEA430594EA050F08BFEE
:1015C00090EA020F1FBF54EA000C55EA020C7FEAB2
:1015D000645C7FEA655C00F0E2804FEA5454D4EB2F
:1015E0005555B8BF6D420CDD2C4480EA020281EAF9
:1015F000030382EA000083EA010180EA020281EA31
:101600000303362D88BF30BD11F0004F4FEA013182
:101610004FF4801C4CEA113102D0404261EB410191
:1016200013F0004F4FEA03334CEA133302D0524217
:1016300063EB430394EA050F00F0A780A4F10104D3
:10164000D5F1200E0DDB02FA0EFC22FA05F280180D
:1016500041F1000103FA0EF2801843FA05F35941F3
:101660000EE0A5F120050EF1200E012A03FA0EFC72
:1016700028BF4CF0020C43FA05F3C01851EBE3719C
:1016800001F0004507D54FF0000EDCF1000C7EEBB9
:1016900000006EEB0101B1F5801F1BD3B1F5001FF7
:1016A0000CD349085FEA30004FEA3C0C04F1010416
:1016B0004FEA445212F5800F80F09A80BCF1004F3F
:1016C00008BF5FEA500C50F1000041EB045141EAC1
:1016D000050130BD5FEA4C0C404141EB010111F4C2
:1016E000801FA4F10104E9D191F0000F04BF01466D
:1016F0000020B1FA81F308BF2033A3F10B03B3F14B
:1017000020020CDA0C3208DD02F1140CC2F10C02DA
:1017100001FA0CF021FA02F10CE002F11402D8BF38
:10172000C2F1200C01FA02F120FA0CFCDCBF41EA04
:101730000C019040E41AA2BF01EB0451294330BDD3
:101740006FEA04041F3C1CDA0C340EDC04F11404B0
:10175000C4F1200220FA04F001FA02F340EA030087
:1017600021FA04F345EA030130BDC4F10C04C4F1CD
:10177000200220FA02F001FA04F340EA03002946AD
:1017800030BD21FA04F0294630BD94F0000F83F4F7
:10179000801306BF81F480110134013D4EE77FEADA
:1017A000645C18BF7FEA655C29D094EA050F08BF26
:1017B00090EA020F05D054EA000C04BF1946104607
:1017C00030BD91EA030F1EBF0021002030BD5FEA4B
:1017D000545C05D14000494128BF41F0004130BD73
:1017E00014F580043CBF01F5801130BD01F00045C7
:1017F00045F0FE4141F470014FF0000030BD7FEA3A
:10180000645C1ABF194610467FEA655C1CBF0B4634
:10181000024650EA013406BF52EA033591EA030F4B
:1018200041F4002130BD00BF90F0000F04BF002143
:10183000704730B54FF4806404F132044FF0000576
:101840004FF0000150E700BF90F0000F04BF0021EF
:10185000704730B54FF4806404F1320410F0004555
:1018600048BF40424FF000013EE700BF42004FEA50
:10187000E2014FEA31014FEA02701FBF12F07F43CD
:1018800093F07F4F81F06051704792F0000F14BFCA
:1018900093F07F4F704730B54FF4607401F000450E
:1018A00021F0004120E700BF50EA010208BF704765
:1018B00030B54FF000050AE050EA010208BF70475A
:1018C00030B511F0004502D5404261EB41014FF4C3
:1018D000806404F132045FEA915C3FF4DCAE4FF0C7
:1018E00003025FEADC0C18BF03325FEADC0C18BFAE
:1018F000033202EBDC02C2F1200300FA03FC20FAFF
:1019000002F001FA03FE40EA0E0021FA02F114444B
:10191000C1E600BF70B54FF0FF0C4CF4E06C1CEA60
:1019200011541DBF1CEA135594EA0C0F95EA0C0FD5
:1019300000F0DEF82C4481EA030621EA4C5123EA48
:101940004C5350EA013518BF52EA033541F4801177
:1019500043F4801338D0A0FB02CE4FF00005E1FB2A
:1019600002E506F00042E0FB03E54FF00006E1FB74
:1019700003569CF0000F18BF4EF0010EA4F1FF04B7
:10198000B6F5007F64F5407404D25FEA4E0E6D41F7
:1019900046EB060642EAC62141EA55514FEAC52008
:1019A00040EA5E504FEACE2EB4F1FD0C88BFBCF584
:1019B000E06F1ED8BEF1004F08BF5FEA500E50F135
:1019C000000041EB045170BD06F0004646EA0101FB
:1019D00040EA020081EA0301B4EB5C04C2BFD4EB2D
:1019E0000C0541EA045170BD41F480114FF0000E26
:1019F000013C00F3AB8014F1360FDEBF002001F094
:101A0000004170BDC4F10004203C35DA0C341BDC0D
:101A100004F11404C4F1200500FA05F320FA04F0DF
:101A200001FA05F240EA020001F0004221F0004113
:101A300010EBD37021FA04F642EB06015EEA430E86
:101A400008BF20EAD37070BDC4F10C04C4F12005B6
:101A500000FA04F320FA05F001FA04F240EA020069
:101A600001F0004110EBD37041F100015EEA430E3A
:101A700008BF20EAD37070BDC4F1200500FA05F25A
:101A80004EEA020E20FA04F301FA05F243EA0203D9
:101A900021FA04F001F0004121FA04F220EA0200E8
:101AA00000EBD3705EEA430E08BF20EAD37070BD2E
:101AB00094F0000F0FD101F00046400041EB01010E
:101AC00011F4801F08BF013CF7D041EA060195F0F0
:101AD000000F18BF704703F00046520043EB0303AA
:101AE00013F4801F08BF013DF7D043EA0603704797
:101AF00094EA0C0F0CEA135518BF95EA0C0F0CD0A2
:101B000050EA410618BF52EA4306D1D181EA0301E7
:101B100001F000414FF0000070BD50EA410606BFE1
:101B20001046194652EA430619D094EA0C0F02D126
:101B300050EA013613D195EA0C0F05D152EA03366B
:101B40001CBF104619460AD181EA030101F0004189
:101B500041F0FE4141F470014FF0000070BD41F0D2
:101B6000FE4141F4780170BD70B54FF0FF0C4CF4AC
:101B7000E06C1CEA11541DBF1CEA135594EA0C0FCB
:101B800095EA0C0F00F0A7F8A4EB050481EA030E18
:101B900052EA03354FEA013100F088804FEA0333FF
:101BA0004FF0805545EA131343EA12634FEA0222CD
:101BB00045EA111545EA10654FEA00260EF000418E
:101BC0009D4208BF964244F1FD0404F5407402D2E0
:101BD0005B084FEA3202B61A65EB03055B084FEA71
:101BE00032024FF480104FF4002CB6EB020E75EB6E
:101BF000030E22BFB61A754640EA0C005B084FEA96
:101C00003202B6EB020E75EB030E22BFB61A754612
:101C100040EA5C005B084FEA3202B6EB020E75EB5D
:101C2000030E22BFB61A754640EA9C005B084FEAD5
:101C30003202B6EB020E75EB030E22BFB61A7546E2
:101C400040EADC0055EA060E18D04FEA051545EAD1
:101C500016754FEA06164FEAC30343EA52734FEA7A
:101C6000C2025FEA1C1CC0D111F4801F0BD141EAF3
:101C700000014FF000004FF0004CB6E711F4801F58
:101C800004BF01430020B4F1FD0C88BFBCF5E06F38
:101C90003FF6AFAEB5EB030C04BFB6EB020C5FEA48
:101CA000500C50F1000041EB045170BD0EF0004E9D
:101CB0004EEA113114EB5C04C2BFD4EB0C0541EACF
:101CC000045170BD41F480114FF0000E013C90E6CC
:101CD00045EA060E8DE60CEA135594EA0C0F08BF90
:101CE00095EA0C0F3FF43BAF94EA0C0F0AD150EA8F
:101CF00001347FF434AF95EA0C0F7FF425AF104622
:101D000019462CE795EA0C0F06D152EA03353FF449
:101D1000FDAE1046194622E750EA410618BF52EAC6
:101D200043067FF4C5AE50EA41047FF40DAF52EA9A
:101D300043057FF4EBAE12E74FF0FF3C06E000BF37
:101D40004FF0010C02E000BF4FF0010C4DF804CD44
:101D50004FEA410C7FEA6C5C4FEA430C18BF7FEA04
:101D60006C5C1BD001B050EA410C0CBF52EA430C32
:101D700091EA030F02BF90EA020F0020704710F1B2
:101D8000000F91EA030F58BF994208BF90422CBF41
:101D9000D8176FEAE37040F0010070474FEA410C3A
:101DA0007FEA6C5C02D150EA013C07D14FEA430C58
:101DB0007FEA6C5CD6D152EA033CD3D05DF8040BC9
:101DC000704700BF8446104662468C4619466346FB
:101DD00000E000BF01B5FFF7B7FF002848BF10F1D2
:101DE000000F01BD4DF808EDFFF7F4FF0CBF012017
:101DF00000205DF808FB00BF4DF808EDFFF7EAFF93
:101E000034BF012000205DF808FB00BF4DF808ED4D
:101E1000FFF7E0FF94BF012000205DF808FB00BF42
:101E20004DF808EDFFF7CEFF94BF012000205DF8CC
:101E300008FB00BF4DF808EDFFF7C4FF34BF0120D9
:101E400000205DF808FB00BF4FEA410212F50012C6
:101E500015D211D56FF47873B3EB625212D94FEAF1
:101E6000C12343F0004343EA505311F0004F23FADB
:101E700002F018BF404270474FF00000704750EA30
:101E8000013005D111F0004008BF6FF000407047ED
:101E90004FF00000704700BF4FEA4102B2F1E0434B
:101EA00024BFB3F5001CDCF1FE5C0DD901F0004C41
:101EB0004FEAC0024CEA5070B2F1004F40EB830091
:101EC00008BF20F00100704711F0804F21D113F1BD
:101ED0003872BCBF01F00040704741F480114FEAF6
:101EE0005252C2F11802C2F1200C10FA0CF320FA7F
:101EF00002F018BF40F001004FEAC1234FEAD3239C
:101F000003FA0CFC40EA0C0023FA02F34FEA430305
:101F1000CCE77FEA625307D150EA01331EBF4FF08E
:101F2000FE4040F44000704701F0004040F0FE40A9
:101F300040F40000704700BF80F0004002E000BFA6
:101F400081F0004142001FBF5FEA410392EA030FA4
:101F50007FEA226C7FEA236C6AD04FEA1262D2EBEE
:101F60001363C1BFD218414048404140B8BF5B42F3
:101F7000192B88BF704710F0004F40F4000020F08C
:101F80007F4018BF404211F0004F41F4000121F0A2
:101F90007F4118BF494292EA030F3FD0A2F10102EC
:101FA00041FA03FC10EB0C00C3F1200301FA03F12A
:101FB00000F0004302D5494260EB4000B0F5000F4D
:101FC00013D3B0F1807F06D340084FEA310102F10C
:101FD0000102FE2A51D2B1F1004F40EBC25008BFBE
:101FE00020F0010040EA03007047490040EB000088
:101FF00010F4000FA2F10102EDD1B0FA80FCACF1B7
:10200000080CB2EB0C0200FA0CF0AABF00EBC250B5
:1020100052421843BCBFD0401843704792F0000FA3
:1020200081F4000106BF80F400000132013BB5E7F6
:102030004FEA41037FEA226C18BF7FEA236C21D06C
:1020400092EA030F04D092F0000F08BF08467047D1
:1020500090EA010F1CBF0020704712F07F4F04D19F
:10206000400028BF40F00040704712F100723CBFB2
:1020700000F50000704700F0004343F0FE4040F4DC
:10208000000070477FEA226216BF08467FEA23639A
:102090000146420206BF5FEA412390EA010F40F485
:1020A000800070474FF0000304E000BF10F00043D1
:1020B00048BF40425FEA000C08BF704743F09643B8
:1020C00001464FF000001CE050EA010208BF7047D3
:1020D0004FF000030AE000BF50EA010208BF70475A
:1020E00011F0004302D5404261EB41015FEA010C6F
:1020F00002BF84460146002043F0B64308BFA3F167
:102100008053A3F50003BCFA8CF2083AA3EBC25348
:1021100010DB01FA02FC634400FA02FCC2F1200267
:10212000BCF1004F20FA02F243EB020008BF20F09E
:102130000100704702F1200201FA02FCC2F1200204
:1021400050EA4C0021FA02F243EB020008BF20EAF9
:10215000DC7070474FF0FF0C1CEAD0521EBF1CEA27
:10216000D15392EA0C0F93EA0C0F6FD01A4480EA15
:10217000010C400218BF5FEA41211ED04FF00063FE
:1021800043EA501043EA5111A0FB01310CF000402A
:10219000B1F5000F3EBF490041EAD3715B0040EA50
:1021A000010062F17F02FD2A1DD8B3F1004F40EB20
:1021B000C25008BF20F00100704790F0000F0CF0F3
:1021C000004C08BF49024CEA502040EA51207F3AB7
:1021D000C2BFD2F1FF0340EAC250704740F4000092
:1021E0004FF00003013A5DDC12F1190FDCBF00F083
:1021F00000407047C2F10002410021FA02F1C2F131
:10220000200200FA02FC5FEA310040F1000053EACC
:102210004C0308BF20EADC70704792F0000F00F01A
:10222000004C02BF400010F4000F013AF9D040EA20
:102230000C0093F0000F01F0004C02BF490011F4B4
:10224000000F013BF9D041EA0C018FE70CEAD153B2
:1022500092EA0C0F18BF93EA0C0F0AD030F0004C32
:1022600018BF31F0004CD8D180EA010000F00040E6
:10227000704790F0000F17BF90F0004F084691F0A4
:10228000000F91F0004F14D092EA0C0F01D14202DE
:102290000FD193EA0C0F03D14B0218BF084608D1A7
:1022A00080EA010000F0004040F0FE4040F40000F1
:1022B000704740F0FE4040F4400070474FF0FF0C84
:1022C0001CEAD0521EBF1CEAD15392EA0C0F93EACB
:1022D0000C0F69D0A2EB030280EA010C49024FEA1D
:1022E000402037D04FF0805343EA111143EA1013D6
:1022F0000CF000408B4238BF5B0042F17D024FF48E
:10230000000C8B4224BF5B1A40EA0C00B3EB510F68
:1023100024BFA3EB510340EA5C00B3EB910F24BF51
:10232000A3EB910340EA9C00B3EBD10F24BFA3EBD6
:10233000D10340EADC001B0118BF5FEA1C1CE0D19E
:10234000FD2A3FF650AF8B4240EBC25008BF20F051
:10235000010070470CF0004C4CEA50207F32C2BFA5
:10236000D2F1FF0340EAC250704740F400004FF042
:102370000003013A37E792F0000F00F0004C02BF73
:10238000400010F4000F013AF9D040EA0C0093F03D
:10239000000F01F0004C02BF490011F4000F013B97
:1023A000F9D041EA0C0195E70CEAD15392EA0C0FFF
:1023B00008D142027FF47DAF93EA0C0F7FF470AF37
:1023C000084676E793EA0C0F04D14B023FF44CAF7A
:1023D00008466EE730F0004C18BF31F0004CCAD10F
:1023E00030F000427FF45CAF31F000437FF43CAF4B
:1023F0005FE700BF4FF0FF3C06E000BF4FF0010C6D
:1024000002E000BF4FF0010C4DF804CD4FEA40024E
:102410004FEA41037FEA226C18BF7FEA236C11D098
:1024200001B052EA530C18BF90EA010F58BFB2EB4B
:10243000030088BFC81738BF6FEAE17018BF40F0CB
:10244000010070477FEA226C02D15FEA402C05D17F
:102450007FEA236CE4D15FEA412CE1D05DF8040B04
:10246000704700BF844608466146FFE70FB5FFF797
:10247000C9FF002848BF10F1000F0FBD4DF808ED4F
:10248000FFF7F4FF0CBF012000205DF808FB00BF40
:102490004DF808EDFFF7EAFF34BF012000205DF89A
:1024A00008FB00BF4DF808EDFFF7E0FF94BF0120E7
:1024B00000205DF808FB00BF4DF808EDFFF7D2FFE4
:1024C00094BF012000205DF808FB00BF4DF808ED27
:1024D000FFF7C8FF34BF012000205DF808FB00BFF4
:1024E00042000ED2B2F1FE4F0BD34FF09E03B3EB7E
:1024F000126209D44FEA002343F0004323FA02F0AA
:1025000070474FF00000704712F1610F01D1420295
:1025100002D14FF0FF3070474FF00000704700BF0E
:1025200073B96AB9002908BF0028BCBF00204FF06A
:102530000041C4BF6FF000414FF0FF30FFF730B8EB
:1025400082B0EC462DE9005000F01CF8DDF804E004
:1025500002B00CBC704700BFF8B514461D460646D5
:102560000F4600F0D3F900FB05F5A0FB042304FBA4
:102570000154E318B61A67EB0307069BC3E900672B
:10258000F8BD00BFF8B514461D4606460F4600F0DC
:102590000FF800FB05F5A0FB042304FB0154E3182E
:1025A000B61A67EB0307069BC3E90067F8BD00BFD7
:1025B00000292DE9F04F85B0C0F2C9800026002B1C
:1025C000C0F2C0808946144605469B46002B4BD17D
:1025D0008A4258D9B2FA82F353B1C3F1200001FA0A
:1025E00003F925FA00F812FA03F49D4048EA0909B4
:1025F000270C484639461FFA84FBFEF795FE3946FC
:1026000082464846FEF7BEFF4FEA15420BFB0AF32F
:1026100042EA01494B4509D919EB04090AF1FF3A8D
:1026200004D24B4584BF0AF1FF3AA144C3EB090928
:1026300039464846ADB2FEF777FE394680464846F1
:10264000FEF7A0FF0BFB08FB45EA0145AB4507D9A8
:102650002D1908F1FF3803D2AB4588BF08F1FF38C8
:1026600048EA0A48002703E08B4257D90027B846BA
:1026700042463B4616B1524263EB430319461046AD
:1026800005B0BDE8F08F22B911460120FEF74CFEDF
:102690000446B4FA84F8B8F1000F5ED1C4EB09081F
:1026A000270C1FFA84F90121029139464046FEF7B2
:1026B0003BFE394682464046FEF764FF4FEA154826
:1026C00009FB0AF348EA014B5B4509D91BEB040BF4
:1026D0000AF1FF3A04D25B4584BF0AF1FF3AA344F2
:1026E000C3EB0B0B39465846ADB2FEF71DFE39461B
:1026F00080465846FEF746FF09FB08F945EA0145C2
:10270000A94507D92D1908F1FF3803D2A94588BF7B
:1027100008F1FF3848EA0A48029FA9E7B3FA83F7AD
:10272000002F67D18B422CBF4FF000094FF00109F9
:1027300082428CBF4C4649F00104002C96D04FF0E9
:10274000010895E7524263EB4303F6433AE7404200
:1027500061EB41014FF0FF3631E704FA08F4C8F1AC
:10276000200735FA07F329FA07FA270C09FA08FBBC
:102770003946504643EA0B020292FEF7D5FD394630
:102780001FFA84F983465046FEF7FCFE029809FBC7
:102790000BF2030C43EA01439A4204D91B190BF1D3
:1027A000FF3BC0F0AD809B1A394618460193FEF7F7
:1027B000BBFD0199824608463946FEF7E3FE0298C2
:1027C00009FB0AF31FFA80FC4CEA0142934208D944
:1027D00012190AF1FF3A04D2934284BF0AF1FF3A78
:1027E000121905FA08F54AEA0B4EC3EB0208CDF8B8
:1027F00008E05AE7C7F1200003FA07FAC24035FAA9
:1028000000F342EA0A0B21FA00F801FA07F9404600
:102810004FEA1B4A43EA0901029151461FFA8BF223
:102820000392FEF781FD514681464046FEF7AAFE1F
:102830000398029B00FB09F2180C14FA07F340EA14
:102840000144A24204D914EB0B0409F1FF3951D31E
:10285000A41A514620460193FEF766FD5146804674
:102860002046FEF78FFE039C019B04FB08F2029CAE
:102870001FFA84FC4CEA0140824204D910EB0B00A1
:1028800008F1FF3830D348EA09481FFA83FC1B0CD3
:10289000801A1FFA88FE4FEA184A0CFB0EF90CFB4F
:1028A0000AF203FB0E2103FB0AF301EB19418A42F2
:1028B00088BF03F5803303EB114E704510D31FFA28
:1028C00089F905FA07F709EB014014BF002201223C
:1028D00087422CBF002702F00107002F3FF4C8AE4B
:1028E00008F1FF380027C3E6824284BF584408F14C
:1028F000FF38C8E7A24284BF09F1FF395C44A7E76B
:102900009A4284BF0BF1FF3B1B194CE72DE9F04FB6
:102910000C4683B08046164689461F4615468A46B1
:10292000002B4BD18A425CD9B2FA82F35BB1C3F17E
:10293000200001FA03FA28FA00F216FA03F508FA61
:1029400003F842EA0A0A2E0C50463146AFB2FEF7AF
:10295000EBFC31464FEA184481465046FEF712FE22
:1029600007FB09F344EA014A534509D91AEB050A62
:1029700009F1FF3904D2534584BF09F1FF39AA4454
:10298000C3EB0A0A314650461FFA88F8FEF7CCFC22
:10299000314604465046FEF7F5FD07FB04F748EACA
:1029A0000148474506D9013C18EB050802D24745C6
:1029B00088BF013C44EA094400265CE08B4258D8B9
:1029C000B3FA83F6002E5BD18B422CBF002201228A
:1029D00085428CBF154642F00105002D49D00124E7
:1029E00049E022B911460120FEF79EFC0546B5FAE2
:1029F00085F6002E40F0BB80641B2F0C1FFA85FA71
:102A0000012639462046FEF78FFC39464FEA184B1F
:102A100081462046FEF7B6FD0AFB09F34BEA014B5F
:102A20005B4509D91BEB050B09F1FF3904D25B4566
:102A300084BF09F1FF39AB44C3EB0B0B3946584651
:102A40001FFA88F8FEF770FC394604465846FEF730
:102A500099FD0AFB04FA48EA0148C24506D9013C3F
:102A600018EB050802D2C24588BF013C44EA09447C
:102A700001E0002634463146204603B0BDE8F08F21
:102A8000C6F12000B34032FA00F721FA00FB1F43E1
:102A900014FA06F228FA00F158464FEA174A114391
:102AA00000915146BBB20193FEF73EFC5146B54042
:102AB00081465846FEF766FD019C009804FB09F329
:102AC0004FEA104C4CEA014B5B4505D91BEB070B59
:102AD00009F1FF39C0F08F80C3EB0B0B514658460C
:102AE000FEF722FC514604465846FEF74BFD01987E
:102AF000009A00FB04F31FFA82FC4CEA0142934265
:102B000006D9013CD21903D2934201D9D219013C12
:102B100044EA0944A8B2D21A2D0C1FFA84FC4FEAE9
:102B2000144300FB0CF700FB03FE05FB0CE105FB67
:102B300003F501EB17418E4588BF05F5803505EBA0
:102B40001145AA4210D3BFB208FA06F607EB0142BC
:102B500014BF4FF0000E4FF0010E96422CBF00261E
:102B60000EF00106002E86D0013C002683E7B5401A
:102B7000C6F1200124FA01F928FA01F22F0CB44021
:102B80003946484622430092FEF7CEFB39461FFAEB
:102B900085FA83464846FEF7F5FC009B1A0C0AFBB3
:102BA0000BF342EA0144A34203D964190BF1FF3B42
:102BB00027D3E41A39462046FEF7B6FB394681464C
:102BC0002046FEF7DFFC00980AFB09F31FFA80FCA1
:102BD0004CEA0144A34208D9641909F1FF3904D22F
:102BE000A34284BF09F1FF39641908FA06F8E41A10
:102BF00049EA0B4605E75B4584BF09F1FF39BB4451
:102C00006AE7A34284BF0BF1FF3B6419D1E700BF21
:102C10000000000000000000010003E800000000C8
:102C200000000003E800000000000200FA060003B4
:102C30000000000000370600000000000000000057
:102C4000F40100006400000001800808000000009A
:102C5000006400000000000000000000C800000048
:102C60001201100102000040D0165106011B0102A2
:102C70000301000009024300020100C03209040000
:102C800000010202010005240010010524010001D9
:102C9000042402020524060001070582030800FF40
:102CA00009040100020A00000007050302400000B9
:102CB00007058102400000000403090426035400B4
:102CC000720069006E0061006D00690063004D00D4
:102CD0006F00740069006F006E00200043007400F4
:102CE0006C000000320354004D0043004D002D00E5
:102CF00031003100360030002000280076006900E5
:102D000072007400750061006C00200043004F00E9
:102D10004D00290020000000524F520000010652D1
:102D20004F4C000002064D5354000003024D565014
:102D300000000407534150000005074741500000C0
:102D400006035354415000070352534150000803F7
:102D50005347500000090747475000000A035354E7
:102D60004750000B0352534750000C035246530088
:102D7000000D0353494F00000E0747494F00000F55
:102D80000353414300001D0753434F00001E0747F4
:102D9000434F00001F0343434F0000200341434FB4
:102DA000000027035546300000400755463100001B
:102DB000410755463200004207554633000043079D
:102DC0005546340000440755463500004507554632
:102DD00036000046075546370000470752554E005B
:102DE00000810553544F5000800042494E00008B33
:102DF00000000000000000000200000000000001D0
:102E00000000000001020304010203040607080990
:102E1000020406080020202020202020202028282E
:102E2000282828202020202020202020202020208A
:102E300020202020208810101010101010101010CA
:102E400010101010100404040404040404040410FA
:102E50001010101010104141414141410101010188
:102E60000101010101010101010101010101010152
:102E7000101010101010424242424242020202025E
:102E80000202020202020202020202020202020222
:102E900010101010200000000000000000000000D2
:102EA0000000000000000000000000000000000022
:102EB0000000000000000000000000000000000012
:102EC0000000000000000000000000000000000002
:102ED00000000000000000000000000000000000F2
:102EE00000000000000000000000000000000000E2
:102EF00000000000000000000000000000000000D2
:102F000000000000000000000000000000000000C1
:102F100000000000000000003131363056313237F9
:102F2000004142530052454C00434F4F524400531E
:102F3000544152540053544F50005354415455532C
:102F400000000000430000006C6F670000000000FC
:082F500060F6FF7F01000000A4
:102F5800182F01080001000000010200000800000D
:102F68000100000002000000000000000000000056
:102F78000000000000000000000000000000000049
:102F88000000000000000000000000000000000039
:102F9800000000000000000000C20100000008005E
:102FA800B82C010804000000BC2C01082600000011
:102FB800E42C010832000000B00000201A000000D4
:102FC800742C010843000000602C01081200000066
:102FD80011A100081D9F00082D9D0008419D0008B3
:102FE800459D0008A59D0008C99D00080D9F000883
:102FF800FD9E0008D99E0008000000004000000067
:103008001A0354004D0043003100310036003000EF
:103018000000000000000000000000002D9C0008D7
:10302800B9FB0008B9FB0008B9FB0008B9FB0008A8
:10303800B9FB0008B9FB0008B9FB0008B9FB000898
:103048006DA00008B9FB0008B9FB0008B9FB00082F
:10305800B9FB000804010000B9FB0008099D00083D
:10306800B9FB0008B9FB0008B9FB0008B9FB000868
:10307800B9FB0008B9FB0008219D00080100000009
:10308800152E0108142E01083C0100200000000044
:103098000000000000000000000000000000000028
:1030A800000000000000000000000000442F01089C
:1030B8000000000000000000000000000000000008
:1030C80000000000000000000000000000000000F8
:1030D80000000000000000000000000000000000E8
:1030E80000000000000000000000000000000000D8
:1030F80000000000000000000000000000000000C8
:1031080000000000000000000000000000000000B7
:1031180000000000000000000000000000000000A7
:103128000000000000000000000000000000000097
:103138000000000000000000000000000000000087
:103148000000000000000000000000000000000077
:103158000000000000000000000000000000000067
:103168000000000000000000000000000000000057
:103178000000000000000000000000000100000046
:04000005080041109E
:00000001FF
